 Localizer

 Timestamp is 54e2a5c5 (Mon Feb 16 20:21:57 2015)

 Preferred load address is 10000000

 Start         Length     Name                   Class
 0001:00000000 000089baH .text                   CODE
 0001:000089ba 00000375H .text$x                 CODE
 0001:00008d2f 00000040H .text$yc                CODE
 0001:00008d6f 0000002cH .text$yd                CODE
 0002:00000000 000001a8H .idata$5                DATA
 0002:000001a8 00000004H .CRT$XCA                DATA
 0002:000001ac 00000014H .CRT$XCU                DATA
 0002:000001c0 00000004H .CRT$XCZ                DATA
 0002:000001c4 00000004H .CRT$XIA                DATA
 0002:000001c8 00000004H .CRT$XIAA               DATA
 0002:000001cc 00000004H .CRT$XIC                DATA
 0002:000001d0 00000004H .CRT$XIZ                DATA
 0002:000001e0 00000838H .rdata                  DATA
 0002:00000a18 00000070H .rdata$debug            DATA
 0002:00000a88 00000370H .rdata$r                DATA
 0002:00000e00 00000088H .rdata$sxdata           DATA
 0002:00000e88 00000004H .rtc$IAA                DATA
 0002:00000e8c 00000004H .rtc$IZZ                DATA
 0002:00000e90 00000004H .rtc$TAA                DATA
 0002:00000e94 00000004H .rtc$TZZ                DATA
 0002:00000e98 0000092cH .xdata$x                DATA
 0002:000017c4 0000008cH .idata$2                DATA
 0002:00001850 00000014H .idata$3                DATA
 0002:00001864 000001a8H .idata$4                DATA
 0002:00001a0c 0000082cH .idata$6                DATA
 0002:00002240 00000c17H .edata                  DATA
 0003:00000000 0000028cH .data                   DATA
 0003:00000290 00004394H .bss                    DATA
 0004:00000000 00000058H .rsrc$01                DATA
 0004:00000060 00000180H .rsrc$02                DATA

  Address         Publics by Value              Rva+Base       Lib:Object

 0000:00000022       ___safe_se_handler_count   00000022     <absolute>
 0000:00000000       ___ImageBase               10000000     <linker-defined>
 0001:00000000       ??$?APB_W@?$list1@AA_W@_bi@boost@@QBEABQB_WABV?$value@PB_W@12@@Z 10001000 f i Localizer.obj
 0001:00000007       ??$?R_NP6G_N_WPB_W@ZV?$list1@AA_W@_bi@boost@@@?$list2@V?$arg@$00@boost@@V?$value@PB_W@_bi@2@@_bi@boost@@QBE_NV?$type@_N@12@P6G_N_WPB_W@ZAAV?$list1@AA_W@12@@Z 10001007 f i Localizer.obj
 0001:0000001b       ??$?R_W@?$bind_t@_NP6G_N_WPB_W@ZV?$list2@V?$arg@$00@boost@@V?$value@PB_W@_bi@2@@_bi@boost@@@_bi@boost@@QAE_NAA_W@Z 1000101b f i Localizer.obj
 0001:0000002d       ??$_Allocate@D@std@@YGPADIPAD@Z 1000102d f i Localizer.obj
 0001:00000054       ??$_Allocate@_W@std@@YGPA_WIPA_W@Z 10001054 f i Localizer.obj
 0001:0000007f       ??$_Destroy_range@U?$_Wrap_alloc@V?$allocator@V?$basic_string@DU?$char_traits@D@std@@V?$allocator@D@2@@std@@@std@@@std@@@std@@YGXPAV?$basic_string@DU?$char_traits@D@std@@V?$allocator@D@2@@0@0AAU?$_Wrap_alloc@V?$allocator@V?$basic_string@DU?$char_traits@D@std@@V?$allocator@D@2@@std@@@std@@@0@@Z 1000107f f i Localizer.obj
 0001:0000009a       ??$_Destroy_range@U?$_Wrap_alloc@V?$allocator@V?$basic_string@DU?$char_traits@D@std@@V?$allocator@D@2@@std@@@std@@@std@@@std@@YGXPAV?$basic_string@DU?$char_traits@D@std@@V?$allocator@D@2@@0@0AAU?$_Wrap_alloc@V?$allocator@V?$basic_string@DU?$char_traits@D@std@@V?$allocator@D@2@@std@@@std@@@0@U_Nonscalar_ptr_iterator_tag@0@@Z 1000109a f i Localizer.obj
 0001:000000b5       ??$_Fill@PAII@std@@YGXPAI0ABI@Z 100010b5 f i Localizer.obj
 0001:000000d3       ??$_Fill@PAPB_WPB_W@std@@YGXPAPB_W0ABQB_W@Z 100010d3 f i Localizer.obj
 0001:000000f1       ??$_Find_if@PA_WV?$bind_t@_NP6G_N_WPB_W@ZV?$list2@V?$arg@$00@boost@@V?$value@PB_W@_bi@2@@_bi@boost@@@_bi@boost@@@std@@YGPA_WPA_W0V?$bind_t@_NP6G_N_WPB_W@ZV?$list2@V?$arg@$00@boost@@V?$value@PB_W@_bi@2@@_bi@boost@@@_bi@boost@@@Z 100010f1 f i Localizer.obj
 0001:00000117       ??$_Max_element@PBI@std@@YGPBIPBI0@Z 10001117 f i Localizer.obj
 0001:00000138       ??$_Move@AA_W@std@@YG$$QA_WAA_W@Z 10001138 f i Localizer.obj
 0001:0000013f       ??$_Ptr_cat@V?$basic_string@DU?$char_traits@D@std@@V?$allocator@D@2@@std@@V12@@std@@YG?AU_Nonscalar_ptr_iterator_tag@0@PAV?$basic_string@DU?$char_traits@D@std@@V?$allocator@D@2@@0@0@Z 1000113f f i Localizer.obj
 0001:00000148       ??$_Rechecked@PBIPBI@std@@YGAAPBIAAPBIPBI@Z 10001148 f i Localizer.obj
 0001:00000155       ??$_Rechecked@V?$_String_val@U?$_Simple_types@_W@std@@@std@@@std@@YG?AV?$_String_iterator@V?$_String_val@U?$_Simple_types@_W@std@@@std@@@0@AAV10@PA_W@Z 10001155 f i Localizer.obj
 0001:00000168       ??$_Remove_if@PA_WV?$bind_t@_NP6G_N_WPB_W@ZV?$list2@V?$arg@$00@boost@@V?$value@PB_W@_bi@2@@_bi@boost@@@_bi@boost@@@std@@YGPA_WPA_W0V?$bind_t@_NP6G_N_WPB_W@ZV?$list2@V?$arg@$00@boost@@V?$value@PB_W@_bi@2@@_bi@boost@@@_bi@boost@@@Z 10001168 f i Localizer.obj
 0001:0000019b       ??$_Unchecked@PAI@std@@YGPAIPAI@Z 1000119b f i Localizer.obj
 0001:000001a2       ??$_Unchecked@PAPB_W@std@@YGPAPB_WPAPB_W@Z 100011a2 f i Localizer.obj
 0001:000001a9       ??$_Unchecked@PBI@std@@YGPBIPBI@Z 100011a9 f i Localizer.obj
 0001:000001b0       ??$_Unchecked@V?$_String_val@U?$_Simple_types@_W@std@@@std@@@std@@YGPA_WV?$_String_iterator@V?$_String_val@U?$_Simple_types@_W@std@@@std@@@0@@Z 100011b0 f i Localizer.obj
 0001:000001b7       ??$addressof@D@std@@YGPADAAD@Z 100011b7 f i Localizer.obj
 0001:000001be       ??$addressof@_W@std@@YGPA_WAA_W@Z 100011be f i Localizer.obj
 0001:000001c5       ??$bind@_N_WPB_WV?$arg@$00@boost@@PB_W@boost@@YG?AV?$bind_t@_NP6G_N_WPB_W@ZV?$list2@V?$arg@$00@boost@@V?$value@PB_W@_bi@2@@_bi@boost@@@_bi@0@P6G_N_WPB_W@ZV?$arg@$00@0@1@Z 100011c5 f i Localizer.obj
 0001:000001e2       ??$checked_array_delete@G@boost@@YGXPAG@Z 100011e2 f i Localizer.obj
 0001:000001ef       ??$construct@PADAAPAD@?$_Wrap_alloc@V?$allocator@D@std@@@std@@QAEXPAPADAAPAD@Z 100011ef f i Localizer.obj
 0001:00000202       ??$construct@PADAAPAD@?$allocator@D@std@@QAEXPAPADAAPAD@Z 10001202 f i Localizer.obj
 0001:00000215       ??$construct@PADAAPAD@?$allocator_traits@V?$allocator@D@std@@@std@@SGXAAV?$allocator@D@1@PAPADAAPAD@Z 10001215 f i Localizer.obj
 0001:00000228       ??$construct@PA_WAAPA_W@?$_Wrap_alloc@V?$allocator@_W@std@@@std@@QAEXPAPA_WAAPA_W@Z 10001228 f i Localizer.obj
 0001:0000023b       ??$construct@PA_WAAPA_W@?$allocator@_W@std@@QAEXPAPA_WAAPA_W@Z 1000123b f i Localizer.obj
 0001:0000024e       ??$construct@PA_WAAPA_W@?$allocator_traits@V?$allocator@_W@std@@@std@@SGXAAV?$allocator@_W@1@PAPA_WAAPA_W@Z 1000124e f i Localizer.obj
 0001:00000261       ??$destroy@PAD@?$_Wrap_alloc@V?$allocator@D@std@@@std@@QAEXPAPAD@Z 10001261 f i Localizer.obj
 0001:00000264       ??$destroy@PAD@?$allocator@D@std@@QAEXPAPAD@Z 10001264 f i Localizer.obj
 0001:00000267       ??$destroy@PAD@?$allocator_traits@V?$allocator@D@std@@@std@@SGXAAV?$allocator@D@1@PAPAD@Z 10001267 f i Localizer.obj
 0001:0000026a       ??$destroy@PA_W@?$_Wrap_alloc@V?$allocator@_W@std@@@std@@QAEXPAPA_W@Z 1000126a f i Localizer.obj
 0001:0000026d       ??$destroy@PA_W@?$allocator@_W@std@@QAEXPAPA_W@Z 1000126d f i Localizer.obj
 0001:00000270       ??$destroy@PA_W@?$allocator_traits@V?$allocator@_W@std@@@std@@SGXAAV?$allocator@_W@1@PAPA_W@Z 10001270 f i Localizer.obj
 0001:00000273       ??$destroy@V?$basic_string@DU?$char_traits@D@std@@V?$allocator@D@2@@std@@@?$_Wrap_alloc@V?$allocator@V?$basic_string@DU?$char_traits@D@std@@V?$allocator@D@2@@std@@@std@@@std@@QAEXPAV?$basic_string@DU?$char_traits@D@std@@V?$allocator@D@2@@1@@Z 10001273 f i Localizer.obj
 0001:0000027f       ??$destroy@V?$basic_string@DU?$char_traits@D@std@@V?$allocator@D@2@@std@@@?$allocator@V?$basic_string@DU?$char_traits@D@std@@V?$allocator@D@2@@std@@@std@@QAEXPAV?$basic_string@DU?$char_traits@D@std@@V?$allocator@D@2@@1@@Z 1000127f f i Localizer.obj
 0001:0000028b       ??$destroy@V?$basic_string@DU?$char_traits@D@std@@V?$allocator@D@2@@std@@@?$allocator_traits@V?$allocator@V?$basic_string@DU?$char_traits@D@std@@V?$allocator@D@2@@std@@@std@@@std@@SGXAAV?$allocator@V?$basic_string@DU?$char_traits@D@std@@V?$allocator@D@2@@std@@@1@PAV?$basic_string@DU?$char_traits@D@std@@V?$allocator@D@2@@1@@Z 1000128b f i Localizer.obj
 0001:00000297       ??$fill@QAII@std@@YGXPAI0ABI@Z 10001297 f i Localizer.obj
 0001:0000029c       ??$fill@QAPB_WPB_W@std@@YGXPAPB_W0ABQB_W@Z 1000129c f i Localizer.obj
 0001:000002a1       ??$find_if@V?$_String_iterator@V?$_String_val@U?$_Simple_types@_W@std@@@std@@@std@@V?$bind_t@_NP6G_N_WPB_W@ZV?$list2@V?$arg@$00@boost@@V?$value@PB_W@_bi@2@@_bi@boost@@@_bi@boost@@@std@@YG?AV?$_String_iterator@V?$_String_val@U?$_Simple_types@_W@std@@@std@@@0@V10@0V?$bind_t@_NP6G_N_WPB_W@ZV?$list2@V?$arg@$00@boost@@V?$value@PB_W@_bi@2@@_bi@boost@@@_bi@boost@@@Z 100012a1 f i Localizer.obj
 0001:000002c9       ??$forward@AAPAD@std@@YGAAPADAAPAD@Z 100012c9 f i Localizer.obj
 0001:000002d0       ??$forward@AAPA_W@std@@YGAAPA_WAAPA_W@Z 100012d0 f i Localizer.obj
 0001:000002d7       ??$max_element@QBI@std@@YGPBIPBI0@Z 100012d7 f i Localizer.obj
 0001:000002dc       ??$remove_if@V?$_String_iterator@V?$_String_val@U?$_Simple_types@_W@std@@@std@@@std@@V?$bind_t@_NP6G_N_WPB_W@ZV?$list2@V?$arg@$00@boost@@V?$value@PB_W@_bi@2@@_bi@boost@@@_bi@boost@@@std@@YG?AV?$_String_iterator@V?$_String_val@U?$_Simple_types@_W@std@@@std@@@0@V10@0V?$bind_t@_NP6G_N_WPB_W@ZV?$list2@V?$arg@$00@boost@@V?$value@PB_W@_bi@2@@_bi@boost@@@_bi@boost@@@Z 100012dc f i Localizer.obj
 0001:0000032e       ??$unwrap@P6G_N_WPB_W@Z@_bi@boost@@YGAAP6G_N_WPB_W@ZAAP6G_N01@ZJ@Z 1000132e f i Localizer.obj
 0001:00000335       ??0?$_String_alloc@$0A@U?$_String_base_types@DV?$allocator@D@std@@@std@@@std@@QAE@ABV?$allocator@D@1@@Z 10001335 f i Localizer.obj
 0001:00000342       ??0?$_String_alloc@$0A@U?$_String_base_types@_WV?$allocator@_W@std@@@std@@@std@@QAE@ABV?$allocator@_W@1@@Z 10001342 f i Localizer.obj
 0001:0000034f       ??0?$_String_const_iterator@V?$_String_val@U?$_Simple_types@_W@std@@@std@@@std@@QAE@PB_WPBU_Container_base0@1@@Z 1000134f f i Localizer.obj
 0001:0000035a       ??0?$_String_iterator@V?$_String_val@U?$_Simple_types@_W@std@@@std@@@std@@QAE@PA_WPBU_Container_base0@1@@Z 1000135a f i Localizer.obj
 0001:00000365       ??0?$_String_val@U?$_Simple_types@D@std@@@std@@QAE@XZ 10001365 f i Localizer.obj
 0001:00000370       ??0?$_String_val@U?$_Simple_types@_W@std@@@std@@QAE@XZ 10001370 f i Localizer.obj
 0001:0000037b       ??0?$_Wrap_alloc@V?$allocator@D@std@@@std@@QAE@XZ 1000137b f i Localizer.obj
 0001:0000037e       ??0?$_Wrap_alloc@V?$allocator@V?$basic_string@DU?$char_traits@D@std@@V?$allocator@D@2@@std@@@std@@@std@@QAE@XZ 1000137e f i Localizer.obj
 0001:00000381       ??0?$_Wrap_alloc@V?$allocator@_W@std@@@std@@QAE@XZ 10001381 f i Localizer.obj
 0001:00000384       ??0?$allocator@D@std@@QAE@XZ 10001384 f i Localizer.obj
 0001:00000387       ??0?$allocator@V?$basic_string@DU?$char_traits@D@std@@V?$allocator@D@2@@std@@@std@@QAE@XZ 10001387 f i Localizer.obj
 0001:0000038a       ??0?$allocator@_W@std@@QAE@XZ 1000138a f i Localizer.obj
 0001:0000038d       ??0?$basic_string@DU?$char_traits@D@std@@V?$allocator@D@2@@std@@QAE@PBD@Z 1000138d f i Localizer.obj
 0001:000003ba       ??0?$basic_string@_WU?$char_traits@_W@std@@V?$allocator@_W@2@@std@@QAE@PB_W@Z 100013ba f i Localizer.obj
 0001:000003e9       ??0?$bind_t@_NP6G_N_WPB_W@ZV?$list2@V?$arg@$00@boost@@V?$value@PB_W@_bi@2@@_bi@boost@@@_bi@boost@@QAE@P6G_N_WPB_W@ZABV?$list2@V?$arg@$00@boost@@V?$value@PB_W@_bi@2@@12@@Z 100013e9 f i Localizer.obj
 0001:00000403       ??0?$list1@AA_W@_bi@boost@@QAE@AA_W@Z 10001403 f i Localizer.obj
 0001:0000040e       ??0?$list2@V?$arg@$00@boost@@V?$value@PB_W@_bi@2@@_bi@boost@@QAE@V?$arg@$00@2@V?$value@PB_W@12@@Z 1000140e f i Localizer.obj
 0001:0000041a       ??0?$scoped_array@G@boost@@QAE@PAG@Z 1000141a f i Localizer.obj
 0001:00000425       ??0?$value@PB_W@_bi@boost@@QAE@ABQB_W@Z 10001425 f i Localizer.obj
 0001:00000432       ??0Resource@LocalizerImp@@QAE@ABV01@@Z 10001432 f i Localizer.obj
 0001:0000043d       ??0Resource@LocalizerImp@@QAE@XZ 1000143d f i Localizer.obj
 0001:00000446       ??1?$basic_string@DU?$char_traits@D@std@@V?$allocator@D@2@@std@@QAE@XZ 10001446 f i Localizer.obj
 0001:00000467       ??1?$basic_string@_WU?$char_traits@_W@std@@V?$allocator@_W@2@@std@@QAE@XZ 10001467 f i Localizer.obj
 0001:00000471       ??1?$scoped_array@G@boost@@QAE@XZ 10001471 f i Localizer.obj
 0001:0000047a       ??1?$vector@V?$basic_string@DU?$char_traits@D@std@@V?$allocator@D@2@@std@@V?$allocator@V?$basic_string@DU?$char_traits@D@std@@V?$allocator@D@2@@std@@@2@@std@@QAE@XZ 1000147a f i Localizer.obj
 0001:0000047f       ??2@YAPAXIPAX@Z            1000147f f i Localizer.obj
 0001:00000484       ??3@YAXPAX0@Z              10001484 f i Localizer.obj
 0001:00000485       ??4?$basic_string@_WU?$char_traits@_W@std@@V?$allocator@_W@2@@std@@QAEAAV01@PB_W@Z 10001485 f i Localizer.obj
 0001:000004a2       ??4Resource@LocalizerImp@@QAEAAV01@ABV01@@Z 100014a2 f i Localizer.obj
 0001:000004a7       ??8?$_String_const_iterator@V?$_String_val@U?$_Simple_types@_W@std@@@std@@@std@@QBE_NABV01@@Z 100014a7 f i Localizer.obj
 0001:000004b7       ??A?$list1@AA_W@_bi@boost@@QBEAA_WV?$arg@$00@2@@Z 100014b7 f i Localizer.obj
 0001:000004bc       ??G?$_String_const_iterator@V?$_String_val@U?$_Simple_types@_W@std@@@std@@@std@@QBEHABV01@@Z 100014bc f i Localizer.obj
 0001:000004c9       ??_EResource@LocalizerImp@@UAEPAXI@Z 100014c9 f i Localizer.obj
 0001:00000512       ??_G?$basic_string@DU?$char_traits@D@std@@V?$allocator@D@2@@std@@QAEPAXI@Z 10001512 f i Localizer.obj
 0001:0000052e       ??_GResource@LocalizerImp@@UAEPAXI@Z 1000152e f i Localizer.obj
 0001:0000054a       ?CheckString@Localizer@@SG_NPB_WK0@Z 1000154a f   Localizer.obj
 0001:000006b1       ?CompareEqual@Localizer@@SG_NABV?$basic_string@_WU?$char_traits@_W@std@@V?$allocator@_W@2@@std@@0@Z 100016b1 f   Localizer.obj
 0001:000006d3       ?CompareEqual@Localizer@@SG_NPB_W0@Z 100016d3 f   Localizer.obj
 0001:00000748       ?CompareSort@Localizer@@SGHABV?$basic_string@_WU?$char_traits@_W@std@@V?$allocator@_W@2@@std@@0@Z 10001748 f   Localizer.obj
 0001:0000076a       ?CompareSort@Localizer@@SGHPB_W0@Z 1000176a f   Localizer.obj
 0001:000007f6       ?CompareStrict@Localizer@@SG_NABV?$basic_string@_WU?$char_traits@_W@std@@V?$allocator@_W@2@@std@@0@Z 100017f6 f   Localizer.obj
 0001:00000818       ?CompareStrict@Localizer@@SG_NPB_W0@Z 10001818 f   Localizer.obj
 0001:00000830       ?ConvertLocIDToLocalized@Localizer@@SG_NHPA_WI@Z 10001830 f   Localizer.obj
 0001:0000087e       ?ConvertLocIDToLocalized@Localizer@@SG_NPBDPA_WI@Z 1000187e f   Localizer.obj
 0001:000008b5       ?ConvertLocIDToLocalized@Localizer@@SG_NPB_WPA_WI@Z 100018b5 f   Localizer.obj
 0001:00000945       ?ConvertLocalizedToLocID@Localizer@@SG_NPB_WAAH@Z 10001945 f   Localizer.obj
 0001:000009a2       ?ConvertNumber2Localized@Localizer@@SG_NPA_WIJ@Z 100019a2 f   Localizer.obj
 0001:00000c0e       ?FormatText@Localizer@@SA_NPA_WIHZZ 10001c0e f   Localizer.obj
 0001:00000cf9       ?GetLocalizedDate@Localizer@@SG_NPA_WI@Z 10001cf9 f   Localizer.obj
 0001:00000d5a       ?GetLocalizedTime@Localizer@@SG_NPA_WI@Z 10001d5a f   Localizer.obj
 0001:00000dbb       ?GetString@Localizer@@SG?AV?$basic_string@_WU?$char_traits@_W@std@@V?$allocator@_W@2@@std@@H@Z 10001dbb f   Localizer.obj
 0001:00000df6       ?GetString@Localizer@@SG_NAAV?$basic_string@_WU?$char_traits@_W@std@@V?$allocator@_W@2@@std@@H@Z 10001df6 f   Localizer.obj
 0001:00000e66       ?GetString@Localizer@@SG_NPA_WIH@Z 10001e66 f   Localizer.obj
 0001:00000eb1       ?Initialize@Localizer@@SG_NXZ 10001eb1 f   Localizer.obj
 0001:00000f41       ?LocString2String@Localizer@@SG?AV?$basic_string@DU?$char_traits@D@std@@V?$allocator@D@2@@std@@ABV?$basic_string@_WU?$char_traits@_W@std@@V?$allocator@_W@2@@3@@Z 10001f41 f   Localizer.obj
 0001:00000f64       ?LocString2String@Localizer@@SG?AV?$basic_string@DU?$char_traits@D@std@@V?$allocator@D@2@@std@@PB_W@Z 10001f64 f   Localizer.obj
 0001:00000f9f       ?LocString2String@Localizer@@SGXPADIPB_W@Z 10001f9f f   Localizer.obj
 0001:00000fe1       ?ResLoadFolder@Localizer@@SG?AV?$vector@V?$basic_string@DU?$char_traits@D@std@@V?$allocator@D@2@@std@@V?$allocator@V?$basic_string@DU?$char_traits@D@std@@V?$allocator@D@2@@std@@@2@@std@@PBD@Z 10001fe1 f   Localizer.obj
 0001:00001002       ?ResUnload@Localizer@@SGXABV?$vector@V?$basic_string@DU?$char_traits@D@std@@V?$allocator@D@2@@std@@V?$allocator@V?$basic_string@DU?$char_traits@D@std@@V?$allocator@D@2@@std@@@2@@std@@@Z 10002002 f   Localizer.obj
 0001:00001015       ?ResUnload@Localizer@@SG_NPBD@Z 10002015 f   Localizer.obj
 0001:00001028       ?Shutdown@Localizer@@SG_NXZ 10002028 f   Localizer.obj
 0001:00001030       ?String2LocString@Localizer@@SG?AV?$basic_string@_WU?$char_traits@_W@std@@V?$allocator@_W@2@@std@@ABV?$basic_string@DU?$char_traits@D@std@@V?$allocator@D@2@@3@@Z 10002030 f   Localizer.obj
 0001:00001053       ?String2LocString@Localizer@@SG?AV?$basic_string@_WU?$char_traits@_W@std@@V?$allocator@_W@2@@std@@PBD@Z 10002053 f   Localizer.obj
 0001:0000108e       ?String2LocString@Localizer@@SGXPA_WIPBD@Z 1000208e f   Localizer.obj
 0001:000010d2       ?TxtAdd@Localizer@@SGHPBDHHPB_WH@Z 100020d2 f   Localizer.obj
 0001:000010f4       ?TxtAddRange@Localizer@@SG_NPBDI0AAH1@Z 100020f4 f   Localizer.obj
 0001:00001116       ?TxtGetRange@Localizer@@SG_NPBDAAH1@Z 10002116 f   Localizer.obj
 0001:00001131       ?TxtLoad@Localizer@@SG_NPBD@Z 10002131 f   Localizer.obj
 0001:00001144       ?TxtResetRange@Localizer@@SG_NPBDHH@Z 10002144 f   Localizer.obj
 0001:0000115f       ?TxtSave@Localizer@@SG_NPBD@Z 1000215f f   Localizer.obj
 0001:00001172       ?TxtUnload@Localizer@@SG_NPBD@Z 10002172 f   Localizer.obj
 0001:00001185       ?UCSLoad@Localizer@@SG_NPBD@Z 10002185 f   Localizer.obj
 0001:00001198       ?UCSUnload@Localizer@@SG_NPBD@Z 10002198 f   Localizer.obj
 0001:000011ab       ?_Adopt@_Iterator_base0@std@@QAEXPBX@Z 100021ab f i Localizer.obj
 0001:000011ae       ?_Compat@?$_String_const_iterator@V?$_String_val@U?$_Simple_types@_W@std@@@std@@@std@@QBEXABV12@@Z 100021ae f i Localizer.obj
 0001:000011b1       ?_Copy@?$basic_string@DU?$char_traits@D@std@@V?$allocator@D@2@@std@@QAEXII@Z 100021b1 f i Localizer.obj
 0001:000012c6       ?_Copy@?$basic_string@_WU?$char_traits@_W@std@@V?$allocator@_W@2@@std@@QAEXII@Z 100022c6 f i Localizer.obj
 0001:000013be       ?_Destroy@?$vector@V?$basic_string@DU?$char_traits@D@std@@V?$allocator@D@2@@std@@V?$allocator@V?$basic_string@DU?$char_traits@D@std@@V?$allocator@D@2@@std@@@2@@std@@IAEXPAV?$basic_string@DU?$char_traits@D@std@@V?$allocator@D@2@@2@0@Z 100023be f i Localizer.obj
 0001:000013d9       ?_Eos@?$basic_string@DU?$char_traits@D@std@@V?$allocator@D@2@@std@@QAEXI@Z 100023d9 f i Localizer.obj
 0001:000013ef       ?_Eos@?$basic_string@_WU?$char_traits@_W@std@@V?$allocator@_W@2@@std@@QAEXI@Z 100023ef f i Localizer.obj
 0001:00001407       ?_Getal@?$_String_alloc@$0A@U?$_String_base_types@DV?$allocator@D@std@@@std@@@std@@QBE?AU?$_Wrap_alloc@V?$allocator@D@std@@@2@XZ 10002407 f i Localizer.obj
 0001:0000140e       ?_Getal@?$_String_alloc@$0A@U?$_String_base_types@_WV?$allocator@_W@std@@@std@@@std@@QBE?AU?$_Wrap_alloc@V?$allocator@_W@std@@@2@XZ 1000240e f i Localizer.obj
 0001:00001415       ?_Getal@?$_Vector_alloc@$0A@U?$_Vec_base_types@V?$basic_string@DU?$char_traits@D@std@@V?$allocator@D@2@@std@@V?$allocator@V?$basic_string@DU?$char_traits@D@std@@V?$allocator@D@2@@std@@@2@@std@@@std@@QBE?AU?$_Wrap_alloc@V?$allocator@V?$basic_string@DU?$char_traits@D@std@@V?$allocator@D@2@@std@@@std@@@2@XZ 10002415 f i Localizer.obj
 0001:0000141c       ?_Grow@?$basic_string@DU?$char_traits@D@std@@V?$allocator@D@2@@std@@QAE_NI_N@Z 1000241c f i Localizer.obj
 0001:0000147d       ?_Grow@?$basic_string@_WU?$char_traits@_W@std@@V?$allocator@_W@2@@std@@QAE_NI_N@Z 1000247d f i Localizer.obj
 0001:000014e3       ?_Inside@?$basic_string@DU?$char_traits@D@std@@V?$allocator@D@2@@std@@QAE_NPBD@Z 100024e3 f i Localizer.obj
 0001:0000151b       ?_Inside@?$basic_string@_WU?$char_traits@_W@std@@V?$allocator@_W@2@@std@@QAE_NPB_W@Z 1000251b f i Localizer.obj
 0001:00001554       ?_Myptr@?$_String_val@U?$_Simple_types@D@std@@@std@@QAEPADXZ 10002554 f i Localizer.obj
 0001:0000155f       ?_Myptr@?$_String_val@U?$_Simple_types@D@std@@@std@@QBEPBDXZ 1000255f f i Localizer.obj
 0001:0000156a       ?_Myptr@?$_String_val@U?$_Simple_types@_W@std@@@std@@QAEPA_WXZ 1000256a f i Localizer.obj
 0001:00001575       ?_Myptr@?$_String_val@U?$_Simple_types@_W@std@@@std@@QBEPB_WXZ 10002575 f i Localizer.obj
 0001:00001580       ?_Pdif@?$basic_string@_WU?$char_traits@_W@std@@V?$allocator@_W@2@@std@@SGIV?$_String_const_iterator@V?$_String_val@U?$_Simple_types@_W@std@@@std@@@2@0@Z 10002580 f i Localizer.obj
 0001:00001591       ?_Rechecked@?$_String_iterator@V?$_String_val@U?$_Simple_types@_W@std@@@std@@@std@@QAEAAV12@PA_W@Z 10002591 f i Localizer.obj
 0001:0000159c       ?_Tidy@?$basic_string@DU?$char_traits@D@std@@V?$allocator@D@2@@std@@QAEX_NI@Z 1000259c f i Localizer.obj
 0001:000015de       ?_Tidy@?$basic_string@_WU?$char_traits@_W@std@@V?$allocator@_W@2@@std@@QAEX_NI@Z 100025de f i Localizer.obj
 0001:00001621       ?_Tidy@?$vector@V?$basic_string@DU?$char_traits@D@std@@V?$allocator@D@2@@std@@V?$allocator@V?$basic_string@DU?$char_traits@D@std@@V?$allocator@D@2@@std@@@2@@std@@IAEXXZ 10002621 f i Localizer.obj
 0001:00001650       ?_Unchecked@?$_String_iterator@V?$_String_val@U?$_Simple_types@_W@std@@@std@@@std@@QBEPA_WXZ 10002650 f i Localizer.obj
 0001:00001653       ?_Xlen@?$basic_string@DU?$char_traits@D@std@@V?$allocator@D@2@@std@@QBEXXZ 10002653 f i Localizer.obj
 0001:0000165f       ?_Xlen@?$basic_string@_WU?$char_traits@_W@std@@V?$allocator@_W@2@@std@@QBEXXZ 1000265f f i Localizer.obj
 0001:0000166b       ?_Xran@?$basic_string@DU?$char_traits@D@std@@V?$allocator@D@2@@std@@QBEXXZ 1000266b f i Localizer.obj
 0001:00001677       ?_Xran@?$basic_string@_WU?$char_traits@_W@std@@V?$allocator@_W@2@@std@@QBEXXZ 10002677 f i Localizer.obj
 0001:00001683       ?allocate@?$_Wrap_alloc@V?$allocator@D@std@@@std@@QAEPADI@Z 10002683 f i Localizer.obj
 0001:00001691       ?allocate@?$_Wrap_alloc@V?$allocator@_W@std@@@std@@QAEPA_WI@Z 10002691 f i Localizer.obj
 0001:0000169f       ?allocate@?$allocator@D@std@@QAEPADI@Z 1000269f f i Localizer.obj
 0001:000016ad       ?allocate@?$allocator@_W@std@@QAEPA_WI@Z 100026ad f i Localizer.obj
 0001:000016bb       ?assign@?$basic_string@DU?$char_traits@D@std@@V?$allocator@D@2@@std@@QAEAAV12@ABV12@II@Z 100026bb f i Localizer.obj
 0001:0000174d       ?assign@?$basic_string@DU?$char_traits@D@std@@V?$allocator@D@2@@std@@QAEAAV12@PBD@Z 1000274d f i Localizer.obj
 0001:0000176a       ?assign@?$basic_string@DU?$char_traits@D@std@@V?$allocator@D@2@@std@@QAEAAV12@PBDI@Z 1000276a f i Localizer.obj
 0001:000017e2       ?assign@?$basic_string@_WU?$char_traits@_W@std@@V?$allocator@_W@2@@std@@QAEAAV12@ABV12@II@Z 100027e2 f i Localizer.obj
 0001:00001869       ?assign@?$basic_string@_WU?$char_traits@_W@std@@V?$allocator@_W@2@@std@@QAEAAV12@PB_W@Z 10002869 f i Localizer.obj
 0001:00001886       ?assign@?$basic_string@_WU?$char_traits@_W@std@@V?$allocator@_W@2@@std@@QAEAAV12@PB_WI@Z 10002886 f i Localizer.obj
 0001:000018f5       ?assign@?$char_traits@D@std@@SAXAADABD@Z 100028f5 f i Localizer.obj
 0001:00001902       ?assign@?$char_traits@_W@std@@SAXAA_WAB_W@Z 10002902 f i Localizer.obj
 0001:00001911       ?begin@?$basic_string@_WU?$char_traits@_W@std@@V?$allocator@_W@2@@std@@QAE?AV?$_String_iterator@V?$_String_val@U?$_Simple_types@_W@std@@@std@@@2@XZ 10002911 f i Localizer.obj
 0001:00001922       ?c_str@?$basic_string@DU?$char_traits@D@std@@V?$allocator@D@2@@std@@QBEPBDXZ 10002922 f i Localizer.obj
 0001:0000192d       ?c_str@?$basic_string@_WU?$char_traits@_W@std@@V?$allocator@_W@2@@std@@QBEPB_WXZ 1000292d f i Localizer.obj
 0001:00001938       ?clear@?$basic_string@_WU?$char_traits@_W@std@@V?$allocator@_W@2@@std@@QAEXXZ 10002938 f i Localizer.obj
 0001:0000194a       ?copy@?$char_traits@D@std@@SAPADPADPBDI@Z 1000294a f i Localizer.obj
 0001:0000195e       ?copy@?$char_traits@_W@std@@SAPA_WPA_WPB_WI@Z 1000295e f i Localizer.obj
 0001:00001972       ?deallocate@?$_Wrap_alloc@V?$allocator@D@std@@@std@@QAEXPADI@Z 10002972 f i Localizer.obj
 0001:0000197f       ?deallocate@?$_Wrap_alloc@V?$allocator@V?$basic_string@DU?$char_traits@D@std@@V?$allocator@D@2@@std@@@std@@@std@@QAEXPAV?$basic_string@DU?$char_traits@D@std@@V?$allocator@D@2@@2@I@Z 1000297f f i Localizer.obj
 0001:0000198c       ?deallocate@?$_Wrap_alloc@V?$allocator@_W@std@@@std@@QAEXPA_WI@Z 1000298c f i Localizer.obj
 0001:00001999       ?deallocate@?$allocator@D@std@@QAEXPADI@Z 10002999 f i Localizer.obj
 0001:000019a6       ?deallocate@?$allocator@V?$basic_string@DU?$char_traits@D@std@@V?$allocator@D@2@@std@@@std@@QAEXPAV?$basic_string@DU?$char_traits@D@std@@V?$allocator@D@2@@2@I@Z 100029a6 f i Localizer.obj
 0001:000019b3       ?deallocate@?$allocator@_W@std@@QAEXPA_WI@Z 100029b3 f i Localizer.obj
 0001:000019c0       ?empty@?$basic_string@_WU?$char_traits@_W@std@@V?$allocator@_W@2@@std@@QBE_NXZ 100029c0 f i Localizer.obj
 0001:000019c9       ?end@?$basic_string@_WU?$char_traits@_W@std@@V?$allocator@_W@2@@std@@QAE?AV?$_String_iterator@V?$_String_val@U?$_Simple_types@_W@std@@@std@@@2@XZ 100029c9 f i Localizer.obj
 0001:000019e4       ?erase@?$basic_string@DU?$char_traits@D@std@@V?$allocator@D@2@@std@@QAEAAV12@I@Z 100029e4 f i Localizer.obj
 0001:00001a10       ?erase@?$basic_string@DU?$char_traits@D@std@@V?$allocator@D@2@@std@@QAEAAV12@II@Z 10002a10 f i Localizer.obj
 0001:00001a91       ?erase@?$basic_string@_WU?$char_traits@_W@std@@V?$allocator@_W@2@@std@@QAE?AV?$_String_iterator@V?$_String_val@U?$_Simple_types@_W@std@@@std@@@2@V?$_String_const_iterator@V?$_String_val@U?$_Simple_types@_W@std@@@std@@@2@0@Z 10002a91 f i Localizer.obj
 0001:00001ae2       ?erase@?$basic_string@_WU?$char_traits@_W@std@@V?$allocator@_W@2@@std@@QAEAAV12@I@Z 10002ae2 f i Localizer.obj
 0001:00001b05       ?erase@?$basic_string@_WU?$char_traits@_W@std@@V?$allocator@_W@2@@std@@QAEAAV12@II@Z 10002b05 f i Localizer.obj
 0001:00001b6f       ?get@?$scoped_array@G@boost@@QBEPAGXZ 10002b6f f i Localizer.obj
 0001:00001b72       ?get@?$value@PB_W@_bi@boost@@QBEABQB_WXZ 10002b72 f i Localizer.obj
 0001:00001b75       ?length@?$basic_string@DU?$char_traits@D@std@@V?$allocator@D@2@@std@@QBEIXZ 10002b75 f i Localizer.obj
 0001:00001b79       ?length@?$char_traits@D@std@@SAIPBD@Z 10002b79 f i Localizer.obj
 0001:00001b8d       ?length@?$char_traits@_W@std@@SAIPB_W@Z 10002b8d f i Localizer.obj
 0001:00001ba1       ?max_size@?$_Wrap_alloc@V?$allocator@D@std@@@std@@QBEIXZ 10002ba1 f i Localizer.obj
 0001:00001ba5       ?max_size@?$_Wrap_alloc@V?$allocator@_W@std@@@std@@QBEIXZ 10002ba5 f i Localizer.obj
 0001:00001bab       ?max_size@?$allocator@D@std@@QBEIXZ 10002bab f i Localizer.obj
 0001:00001baf       ?max_size@?$allocator@_W@std@@QBEIXZ 10002baf f i Localizer.obj
 0001:00001bb5       ?max_size@?$allocator_traits@V?$allocator@D@std@@@std@@SGIABV?$allocator@D@2@@Z 10002bb5 f i Localizer.obj
 0001:00001bbb       ?max_size@?$allocator_traits@V?$allocator@_W@std@@@std@@SGIABV?$allocator@_W@2@@Z 10002bbb f i Localizer.obj
 0001:00001bc3       ?max_size@?$basic_string@DU?$char_traits@D@std@@V?$allocator@D@2@@std@@QBEIXZ 10002bc3 f i Localizer.obj
 0001:00001bc7       ?max_size@?$basic_string@_WU?$char_traits@_W@std@@V?$allocator@_W@2@@std@@QBEIXZ 10002bc7 f i Localizer.obj
 0001:00001bcd       ?move@?$char_traits@D@std@@SAPADPADPBDI@Z 10002bcd f i Localizer.obj
 0001:00001be2       ?move@?$char_traits@_W@std@@SAPA_WPA_WPB_WI@Z 10002be2 f i Localizer.obj
 0001:00001bf6       ?size@?$basic_string@DU?$char_traits@D@std@@V?$allocator@D@2@@std@@QBEIXZ 10002bf6 f i Localizer.obj
 0001:00001bfa       ?size@?$basic_string@_WU?$char_traits@_W@std@@V?$allocator@_W@2@@std@@QBEIXZ 10002bfa f i Localizer.obj
 0001:00001bfe       _wmemcpy                   10002bfe f i Localizer.obj
 0001:00001c16       _wmemmove                  10002c16 f i Localizer.obj
 0001:00001c2f       ??$?0PAVResource@LocalizerImp@@U?$checked_deleter@VResource@LocalizerImp@@@boost@@@shared_count@detail@boost@@QAE@PAVResource@LocalizerImp@@U?$checked_deleter@VResource@LocalizerImp@@@2@@Z 10002c2f f i LocalizerImp.obj
 0001:00001ca0       ??$?0VResource@LocalizerImp@@@?$shared_ptr@VResource@LocalizerImp@@@boost@@QAE@PAVResource@LocalizerImp@@@Z 10002ca0 f i LocalizerImp.obj
 0001:00001cc2       ??$?APBD@?$list1@AAVResEntry@LocalizerImp@@@_bi@boost@@QBEABQBDABV?$value@PBD@12@@Z 10002cc2 f i LocalizerImp.obj
 0001:00001cc9       ??$?RVResEntry@LocalizerImp@@@?$bind_t@_NP6G_NABVResEntry@LocalizerImp@@PBD@ZV?$list2@V?$arg@$00@boost@@V?$value@PBD@_bi@2@@_bi@boost@@@_bi@boost@@QAE_NAAVResEntry@LocalizerImp@@@Z 10002cc9 f i LocalizerImp.obj
 0001:00001cd7       ??$?R_NP6G_NABVResEntry@LocalizerImp@@PBD@ZV?$list1@AAVResEntry@LocalizerImp@@@_bi@boost@@@?$list2@V?$arg@$00@boost@@V?$value@PBD@_bi@2@@_bi@boost@@QBE_NV?$type@_N@12@P6G_NABVResEntry@LocalizerImp@@PBD@ZAAV?$list1@AAVResEntry@LocalizerImp@@@12@@Z 10002cd7 f i LocalizerImp.obj
 0001:00001ce7       ??$_Allocate@V?$basic_string@DU?$char_traits@D@std@@V?$allocator@D@2@@std@@@std@@YGPAV?$basic_string@DU?$char_traits@D@std@@V?$allocator@D@2@@0@IPAV10@@Z 10002ce7 f i LocalizerImp.obj
 0001:00001d13       ??$_Allocate@VResEntry@LocalizerImp@@@std@@YGPAVResEntry@LocalizerImp@@IPAV12@@Z 10002d13 f i LocalizerImp.obj
 0001:00001d3f       ??$_Destroy_range@U?$_Wrap_alloc@V?$allocator@VResEntry@LocalizerImp@@@std@@@std@@@std@@YGXPAVResEntry@LocalizerImp@@0AAU?$_Wrap_alloc@V?$allocator@VResEntry@LocalizerImp@@@std@@@0@@Z 10002d3f f i LocalizerImp.obj
 0001:00001d57       ??$_Destroy_range@U?$_Wrap_alloc@V?$allocator@VResEntry@LocalizerImp@@@std@@@std@@@std@@YGXPAVResEntry@LocalizerImp@@0AAU?$_Wrap_alloc@V?$allocator@VResEntry@LocalizerImp@@@std@@@0@U_Nonscalar_ptr_iterator_tag@0@@Z 10002d57 f i LocalizerImp.obj
 0001:00001d74       ??$_Find_if@PAVResEntry@LocalizerImp@@V?$bind_t@_NP6G_NABVResEntry@LocalizerImp@@PBD@ZV?$list2@V?$arg@$00@boost@@V?$value@PBD@_bi@2@@_bi@boost@@@_bi@boost@@@std@@YGPAVResEntry@LocalizerImp@@PAV12@0V?$bind_t@_NP6G_NABVResEntry@LocalizerImp@@PBD@ZV?$list2@V?$arg@$00@boost@@V?$value@PBD@_bi@2@@_bi@boost@@@_bi@boost@@@Z 10002d74 f i LocalizerImp.obj
 0001:00001d97       ??$_Move@AAPAVResource@LocalizerImp@@@std@@YG$$QAPAVResource@LocalizerImp@@AAPAV12@@Z 10002d97 f i LocalizerImp.obj
 0001:00001d9e       ??$_Move@PAVResEntry@LocalizerImp@@PAV12@@std@@YGPAVResEntry@LocalizerImp@@PAV12@00@Z 10002d9e f i LocalizerImp.obj
 0001:00001db6       ??$_Move@PAVResEntry@LocalizerImp@@PAV12@@std@@YGPAVResEntry@LocalizerImp@@PAV12@00U_Nonscalar_ptr_iterator_tag@0@@Z 10002db6 f i LocalizerImp.obj
 0001:00001de6       ??$_Ptr_cat@VResEntry@LocalizerImp@@V12@@std@@YG?AU_Nonscalar_ptr_iterator_tag@0@PAVResEntry@LocalizerImp@@0@Z 10002de6 f i LocalizerImp.obj
 0001:00001def       ??$_Rechecked@V?$_Vector_val@U?$_Simple_types@VResEntry@LocalizerImp@@@std@@@std@@@std@@YGAAV?$_Vector_iterator@V?$_Vector_val@U?$_Simple_types@VResEntry@LocalizerImp@@@std@@@std@@@0@AAV10@PAVResEntry@LocalizerImp@@@Z 10002def f i LocalizerImp.obj
 0001:00001dfc       ??$_Umove@PAV?$basic_string@DU?$char_traits@D@std@@V?$allocator@D@2@@std@@@?$vector@V?$basic_string@DU?$char_traits@D@std@@V?$allocator@D@2@@std@@V?$allocator@V?$basic_string@DU?$char_traits@D@std@@V?$allocator@D@2@@std@@@2@@std@@IAEPAV?$basic_string@DU?$char_traits@D@std@@V?$allocator@D@2@@1@PAV21@00@Z 10002dfc f i LocalizerImp.obj
 0001:00001e1b       ??$_Umove@PAVResEntry@LocalizerImp@@@?$vector@VResEntry@LocalizerImp@@V?$allocator@VResEntry@LocalizerImp@@@std@@@std@@IAEPAVResEntry@LocalizerImp@@PAV23@00@Z 10002e1b f i LocalizerImp.obj
 0001:00001e3a       ??$_Unchecked@V?$_Vector_val@U?$_Simple_types@VResEntry@LocalizerImp@@@std@@@std@@@std@@YGPAVResEntry@LocalizerImp@@V?$_Vector_iterator@V?$_Vector_val@U?$_Simple_types@VResEntry@LocalizerImp@@@std@@@std@@@0@@Z 10002e3a f i LocalizerImp.obj
 0001:00001e41       ??$_Uninit_move@PAV?$basic_string@DU?$char_traits@D@std@@V?$allocator@D@2@@std@@PAV12@V?$allocator@V?$basic_string@DU?$char_traits@D@std@@V?$allocator@D@2@@std@@@2@V12@@std@@YGPAV?$basic_string@DU?$char_traits@D@std@@V?$allocator@D@2@@0@PAV10@00AAU?$_Wrap_alloc@V?$allocator@V?$basic_string@DU?$char_traits@D@std@@V?$allocator@D@2@@std@@@std@@@0@0U_Nonscalar_ptr_iterator_tag@0@@Z 10002e41 f i LocalizerImp.obj
 0001:00001e6d       ??$_Uninit_move@PAVResEntry@LocalizerImp@@PAV12@V?$allocator@VResEntry@LocalizerImp@@@std@@V12@@std@@YGPAVResEntry@LocalizerImp@@PAV12@00AAU?$_Wrap_alloc@V?$allocator@VResEntry@LocalizerImp@@@std@@@0@0U_Nonscalar_ptr_iterator_tag@0@@Z 10002e6d f i LocalizerImp.obj
 0001:00001ed6       ??$_Uninitialized_move@PAV?$basic_string@DU?$char_traits@D@std@@V?$allocator@D@2@@std@@PAV12@U?$_Wrap_alloc@V?$allocator@V?$basic_string@DU?$char_traits@D@std@@V?$allocator@D@2@@std@@@std@@@2@@std@@YGPAV?$basic_string@DU?$char_traits@D@std@@V?$allocator@D@2@@0@PAV10@00AAU?$_Wrap_alloc@V?$allocator@V?$basic_string@DU?$char_traits@D@std@@V?$allocator@D@2@@std@@@std@@@0@@Z 10002ed6 f i LocalizerImp.obj
 0001:00001ef3       ??$_Uninitialized_move@PAVResEntry@LocalizerImp@@PAV12@U?$_Wrap_alloc@V?$allocator@VResEntry@LocalizerImp@@@std@@@std@@@std@@YGPAVResEntry@LocalizerImp@@PAV12@00AAU?$_Wrap_alloc@V?$allocator@VResEntry@LocalizerImp@@@std@@@0@@Z 10002ef3 f i LocalizerImp.obj
 0001:00001f10       ??$_Val_type@PAV?$basic_string@DU?$char_traits@D@std@@V?$allocator@D@2@@std@@@std@@YGPAV?$basic_string@DU?$char_traits@D@std@@V?$allocator@D@2@@0@PAV10@@Z 10002f10 f i LocalizerImp.obj
 0001:00001f15       ??$_Val_type@PAVResEntry@LocalizerImp@@@std@@YGPAVResEntry@LocalizerImp@@PAV12@@Z 10002f15 f i LocalizerImp.obj
 0001:00001f1a       ??$addressof@$$CBV?$basic_string@DU?$char_traits@D@std@@V?$allocator@D@2@@std@@@std@@YGPBV?$basic_string@DU?$char_traits@D@std@@V?$allocator@D@2@@0@ABV10@@Z 10002f1a f i LocalizerImp.obj
 0001:00001f21       ??$addressof@$$CBVResEntry@LocalizerImp@@@std@@YGPBVResEntry@LocalizerImp@@ABV12@@Z 10002f21 f i LocalizerImp.obj
 0001:00001f28       ??$addressof@VResEntry@LocalizerImp@@@std@@YGPAVResEntry@LocalizerImp@@AAV12@@Z 10002f28 f i LocalizerImp.obj
 0001:00001f2f       ??$bind@_NABVResEntry@LocalizerImp@@PBDV?$arg@$00@boost@@PBD@boost@@YG?AV?$bind_t@_NP6G_NABVResEntry@LocalizerImp@@PBD@ZV?$list2@V?$arg@$00@boost@@V?$value@PBD@_bi@2@@_bi@boost@@@_bi@0@P6G_NABVResEntry@LocalizerImp@@PBD@ZV?$arg@$00@0@1@Z 10002f2f f i LocalizerImp.obj
 0001:00001f4c       ??$checked_delete@VResource@LocalizerImp@@@boost@@YGXPAVResource@LocalizerImp@@@Z 10002f4c f i LocalizerImp.obj
 0001:00001f5d       ??$construct@V?$basic_string@DU?$char_traits@D@std@@V?$allocator@D@2@@std@@AAV12@@?$_Wrap_alloc@V?$allocator@V?$basic_string@DU?$char_traits@D@std@@V?$allocator@D@2@@std@@@std@@@std@@QAEXPAV?$basic_string@DU?$char_traits@D@std@@V?$allocator@D@2@@1@AAV21@@Z 10002f5d f i LocalizerImp.obj
 0001:00001f8c       ??$construct@V?$basic_string@DU?$char_traits@D@std@@V?$allocator@D@2@@std@@AAV12@@?$allocator@V?$basic_string@DU?$char_traits@D@std@@V?$allocator@D@2@@std@@@std@@QAEXPAV?$basic_string@DU?$char_traits@D@std@@V?$allocator@D@2@@1@AAV21@@Z 10002f8c f i LocalizerImp.obj
 0001:00001fbb       ??$construct@V?$basic_string@DU?$char_traits@D@std@@V?$allocator@D@2@@std@@AAV12@@?$allocator_traits@V?$allocator@V?$basic_string@DU?$char_traits@D@std@@V?$allocator@D@2@@std@@@std@@@std@@SGXAAV?$allocator@V?$basic_string@DU?$char_traits@D@std@@V?$allocator@D@2@@std@@@1@PAV?$basic_string@DU?$char_traits@D@std@@V?$allocator@D@2@@1@AAV31@@Z 10002fbb f i LocalizerImp.obj
 0001:00001fea       ??$construct@V?$basic_string@DU?$char_traits@D@std@@V?$allocator@D@2@@std@@ABV12@@?$_Wrap_alloc@V?$allocator@V?$basic_string@DU?$char_traits@D@std@@V?$allocator@D@2@@std@@@std@@@std@@QAEXPAV?$basic_string@DU?$char_traits@D@std@@V?$allocator@D@2@@1@ABV21@@Z 10002fea f i LocalizerImp.obj
 0001:00002019       ??$construct@V?$basic_string@DU?$char_traits@D@std@@V?$allocator@D@2@@std@@ABV12@@?$allocator_traits@V?$allocator@V?$basic_string@DU?$char_traits@D@std@@V?$allocator@D@2@@std@@@std@@@std@@SGXAAV?$allocator@V?$basic_string@DU?$char_traits@D@std@@V?$allocator@D@2@@std@@@1@PAV?$basic_string@DU?$char_traits@D@std@@V?$allocator@D@2@@1@ABV31@@Z 10003019 f i LocalizerImp.obj
 0001:00002048       ??$construct@V?$basic_string@DU?$char_traits@D@std@@V?$allocator@D@2@@std@@V12@@?$_Wrap_alloc@V?$allocator@V?$basic_string@DU?$char_traits@D@std@@V?$allocator@D@2@@std@@@std@@@std@@QAEXPAV?$basic_string@DU?$char_traits@D@std@@V?$allocator@D@2@@1@$$QAV21@@Z 10003048 f i LocalizerImp.obj
 0001:0000205c       ??$construct@V?$basic_string@DU?$char_traits@D@std@@V?$allocator@D@2@@std@@V12@@?$allocator@V?$basic_string@DU?$char_traits@D@std@@V?$allocator@D@2@@std@@@std@@QAEXPAV?$basic_string@DU?$char_traits@D@std@@V?$allocator@D@2@@1@$$QAV21@@Z 1000305c f i LocalizerImp.obj
 0001:00002070       ??$construct@V?$basic_string@DU?$char_traits@D@std@@V?$allocator@D@2@@std@@V12@@?$allocator_traits@V?$allocator@V?$basic_string@DU?$char_traits@D@std@@V?$allocator@D@2@@std@@@std@@@std@@SGXAAV?$allocator@V?$basic_string@DU?$char_traits@D@std@@V?$allocator@D@2@@std@@@1@PAV?$basic_string@DU?$char_traits@D@std@@V?$allocator@D@2@@1@$$QAV31@@Z 10003070 f i LocalizerImp.obj
 0001:00002084       ??$construct@VResEntry@LocalizerImp@@AAV12@@?$_Wrap_alloc@V?$allocator@VResEntry@LocalizerImp@@@std@@@std@@QAEXPAVResEntry@LocalizerImp@@AAV23@@Z 10003084 f i LocalizerImp.obj
 0001:00002089       ??$construct@VResEntry@LocalizerImp@@AAV12@@?$allocator@VResEntry@LocalizerImp@@@std@@QAEXPAVResEntry@LocalizerImp@@AAV23@@Z 10003089 f i LocalizerImp.obj
 0001:000020c6       ??$construct@VResEntry@LocalizerImp@@AAV12@@?$allocator_traits@V?$allocator@VResEntry@LocalizerImp@@@std@@@std@@SGXAAV?$allocator@VResEntry@LocalizerImp@@@1@PAVResEntry@LocalizerImp@@AAV34@@Z 100030c6 f i LocalizerImp.obj
 0001:000020da       ??$construct@VResEntry@LocalizerImp@@ABV12@@?$_Wrap_alloc@V?$allocator@VResEntry@LocalizerImp@@@std@@@std@@QAEXPAVResEntry@LocalizerImp@@ABV23@@Z 100030da f i LocalizerImp.obj
 0001:000020df       ??$construct@VResEntry@LocalizerImp@@ABV12@@?$allocator_traits@V?$allocator@VResEntry@LocalizerImp@@@std@@@std@@SGXAAV?$allocator@VResEntry@LocalizerImp@@@1@PAVResEntry@LocalizerImp@@ABV34@@Z 100030df f i LocalizerImp.obj
 0001:000020f3       ??$construct@VResEntry@LocalizerImp@@V12@@?$_Wrap_alloc@V?$allocator@VResEntry@LocalizerImp@@@std@@@std@@QAEXPAVResEntry@LocalizerImp@@$$QAV23@@Z 100030f3 f i LocalizerImp.obj
 0001:000020f8       ??$construct@VResEntry@LocalizerImp@@V12@@?$allocator@VResEntry@LocalizerImp@@@std@@QAEXPAVResEntry@LocalizerImp@@$$QAV23@@Z 100030f8 f i LocalizerImp.obj
 0001:00002135       ??$construct@VResEntry@LocalizerImp@@V12@@?$allocator_traits@V?$allocator@VResEntry@LocalizerImp@@@std@@@std@@SGXAAV?$allocator@VResEntry@LocalizerImp@@@1@PAVResEntry@LocalizerImp@@$$QAV34@@Z 10003135 f i LocalizerImp.obj
 0001:00002149       ??$destroy@VResEntry@LocalizerImp@@@?$_Wrap_alloc@V?$allocator@VResEntry@LocalizerImp@@@std@@@std@@QAEXPAVResEntry@LocalizerImp@@@Z 10003149 f i LocalizerImp.obj
 0001:00002157       ??$destroy@VResEntry@LocalizerImp@@@?$allocator@VResEntry@LocalizerImp@@@std@@QAEXPAVResEntry@LocalizerImp@@@Z 10003157 f i LocalizerImp.obj
 0001:00002165       ??$destroy@VResEntry@LocalizerImp@@@?$allocator_traits@V?$allocator@VResEntry@LocalizerImp@@@std@@@std@@SGXAAV?$allocator@VResEntry@LocalizerImp@@@1@PAVResEntry@LocalizerImp@@@Z 10003165 f i LocalizerImp.obj
 0001:00002173       ??$find_if@V?$_Vector_iterator@V?$_Vector_val@U?$_Simple_types@VResEntry@LocalizerImp@@@std@@@std@@@std@@V?$bind_t@_NP6G_NABVResEntry@LocalizerImp@@PBD@ZV?$list2@V?$arg@$00@boost@@V?$value@PBD@_bi@2@@_bi@boost@@@_bi@boost@@@std@@YG?AV?$_Vector_iterator@V?$_Vector_val@U?$_Simple_types@VResEntry@LocalizerImp@@@std@@@std@@@0@V10@0V?$bind_t@_NP6G_NABVResEntry@LocalizerImp@@PBD@ZV?$list2@V?$arg@$00@boost@@V?$value@PBD@_bi@2@@_bi@boost@@@_bi@boost@@@Z 10003173 f i LocalizerImp.obj
 0001:0000219b       ??$forward@AAV?$basic_string@DU?$char_traits@D@std@@V?$allocator@D@2@@std@@@std@@YGAAV?$basic_string@DU?$char_traits@D@std@@V?$allocator@D@2@@0@AAV10@@Z 1000319b f i LocalizerImp.obj
 0001:000021a2       ??$forward@AAVResEntry@LocalizerImp@@@std@@YGAAVResEntry@LocalizerImp@@AAV12@@Z 100031a2 f i LocalizerImp.obj
 0001:000021a9       ??$forward@ABV?$basic_string@DU?$char_traits@D@std@@V?$allocator@D@2@@std@@@std@@YGABV?$basic_string@DU?$char_traits@D@std@@V?$allocator@D@2@@0@ABV10@@Z 100031a9 f i LocalizerImp.obj
 0001:000021b0       ??$forward@ABVResEntry@LocalizerImp@@@std@@YGABVResEntry@LocalizerImp@@ABV12@@Z 100031b0 f i LocalizerImp.obj
 0001:000021b7       ??$forward@V?$basic_string@DU?$char_traits@D@std@@V?$allocator@D@2@@std@@@std@@YG$$QAV?$basic_string@DU?$char_traits@D@std@@V?$allocator@D@2@@0@AAV10@@Z 100031b7 f i LocalizerImp.obj
 0001:000021be       ??$forward@V?$vector@V?$basic_string@DU?$char_traits@D@std@@V?$allocator@D@2@@std@@V?$allocator@V?$basic_string@DU?$char_traits@D@std@@V?$allocator@D@2@@std@@@2@@std@@@std@@YG$$QAV?$vector@V?$basic_string@DU?$char_traits@D@std@@V?$allocator@D@2@@std@@V?$allocator@V?$basic_string@DU?$char_traits@D@std@@V?$allocator@D@2@@std@@@2@@0@AAV10@@Z 100031be f i LocalizerImp.obj
 0001:000021c5       ??$forward@VResEntry@LocalizerImp@@@std@@YG$$QAVResEntry@LocalizerImp@@AAV12@@Z 100031c5 f i LocalizerImp.obj
 0001:000021cc       ??$move@AAVResEntry@LocalizerImp@@@std@@YG$$QAVResEntry@LocalizerImp@@AAV12@@Z 100031cc f i LocalizerImp.obj
 0001:000021d3       ??$reset@VResource@LocalizerImp@@@?$shared_ptr@VResource@LocalizerImp@@@boost@@QAEXPAVResource@LocalizerImp@@@Z 100031d3 f i LocalizerImp.obj
 0001:0000220d       ??$swap@PAVResource@LocalizerImp@@@std@@YGXAAPAVResource@LocalizerImp@@0@Z 1000320d f i LocalizerImp.obj
 0001:00002222       ??$throw_exception@Vbad_weak_ptr@boost@@@boost@@YGXABVbad_weak_ptr@0@@Z 10003222 f i LocalizerImp.obj
 0001:0000224a       ??$unwrap@P6G_NABVResEntry@LocalizerImp@@PBD@Z@_bi@boost@@YGAAP6G_NABVResEntry@LocalizerImp@@PBD@ZAAP6G_N01@ZJ@Z 1000324a f i LocalizerImp.obj
 0001:00002251       ??0?$Scoped@USTH@?A0x592ce793@@@@QAE@PAXABUSTH@?A0x592ce793@@@Z 10003251 f i LocalizerImp.obj
 0001:0000225c       ??0?$_Vector_alloc@$0A@U?$_Vec_base_types@V?$basic_string@DU?$char_traits@D@std@@V?$allocator@D@2@@std@@V?$allocator@V?$basic_string@DU?$char_traits@D@std@@V?$allocator@D@2@@std@@@2@@std@@@std@@QAE@ABV?$allocator@V?$basic_string@DU?$char_traits@D@std@@V?$allocator@D@2@@std@@@1@@Z 1000325c f i LocalizerImp.obj
 0001:0000226b       ??0?$_Vector_alloc@$0A@U?$_Vec_base_types@VResEntry@LocalizerImp@@V?$allocator@VResEntry@LocalizerImp@@@std@@@std@@@std@@QAE@ABV?$allocator@VResEntry@LocalizerImp@@@1@@Z 1000326b f i LocalizerImp.obj
 0001:0000227a       ??0?$_Vector_const_iterator@V?$_Vector_val@U?$_Simple_types@V?$basic_string@DU?$char_traits@D@std@@V?$allocator@D@2@@std@@@std@@@std@@@std@@QAE@PAV?$basic_string@DU?$char_traits@D@std@@V?$allocator@D@2@@1@PBU_Container_base0@1@@Z 1000327a f i LocalizerImp.obj
 0001:00002285       ??0?$_Vector_const_iterator@V?$_Vector_val@U?$_Simple_types@VResEntry@LocalizerImp@@@std@@@std@@@std@@QAE@PAVResEntry@LocalizerImp@@PBU_Container_base0@1@@Z 10003285 f i LocalizerImp.obj
 0001:00002290       ??0?$_Vector_iterator@V?$_Vector_val@U?$_Simple_types@V?$basic_string@DU?$char_traits@D@std@@V?$allocator@D@2@@std@@@std@@@std@@@std@@QAE@PAV?$basic_string@DU?$char_traits@D@std@@V?$allocator@D@2@@1@PBU_Container_base0@1@@Z 10003290 f i LocalizerImp.obj
 0001:0000229b       ??0?$_Vector_iterator@V?$_Vector_val@U?$_Simple_types@VResEntry@LocalizerImp@@@std@@@std@@@std@@QAE@PAVResEntry@LocalizerImp@@PBU_Container_base0@1@@Z 1000329b f i LocalizerImp.obj
 0001:000022a6       ??0?$_Vector_val@U?$_Simple_types@V?$basic_string@DU?$char_traits@D@std@@V?$allocator@D@2@@std@@@std@@@std@@QAE@XZ 100032a6 f i LocalizerImp.obj
 0001:000022b3       ??0?$_Vector_val@U?$_Simple_types@VResEntry@LocalizerImp@@@std@@@std@@QAE@XZ 100032b3 f i LocalizerImp.obj
 0001:000022c0       ??0?$_Wrap_alloc@V?$allocator@D@std@@@std@@QAE@ABV?$allocator@D@1@@Z 100032c0 f i LocalizerImp.obj
 0001:000022c5       ??0?$_Wrap_alloc@V?$allocator@VResEntry@LocalizerImp@@@std@@@std@@QAE@XZ 100032c5 f i LocalizerImp.obj
 0001:000022c8       ??0?$allocator@D@std@@QAE@ABV01@@Z 100032c8 f i LocalizerImp.obj
 0001:000022cd       ??0?$allocator@VResEntry@LocalizerImp@@@std@@QAE@XZ 100032cd f i LocalizerImp.obj
 0001:000022d0       ??0?$auto_ptr@VResource@LocalizerImp@@@std@@QAE@PAVResource@LocalizerImp@@@Z 100032d0 f i LocalizerImp.obj
 0001:000022db       ??0?$basic_string@DU?$char_traits@D@std@@V?$allocator@D@2@@std@@QAE@$$QAV01@@Z 100032db f i LocalizerImp.obj
 0001:000022fb       ??0?$basic_string@DU?$char_traits@D@std@@V?$allocator@D@2@@std@@QAE@ABV01@@Z 100032fb f i LocalizerImp.obj
 0001:0000231e       ??0?$basic_string@DU?$char_traits@D@std@@V?$allocator@D@2@@std@@QAE@XZ 1000331e f i LocalizerImp.obj
 0001:0000232f       ??0?$bind_t@_NP6G_NABVResEntry@LocalizerImp@@PBD@ZV?$list2@V?$arg@$00@boost@@V?$value@PBD@_bi@2@@_bi@boost@@@_bi@boost@@QAE@P6G_NABVResEntry@LocalizerImp@@PBD@ZABV?$list2@V?$arg@$00@boost@@V?$value@PBD@_bi@2@@12@@Z 1000332f f i LocalizerImp.obj
 0001:00002349       ??0?$list1@AAVResEntry@LocalizerImp@@@_bi@boost@@QAE@AAVResEntry@LocalizerImp@@@Z 10003349 f i LocalizerImp.obj
 0001:00002354       ??0?$list2@V?$arg@$00@boost@@V?$value@PBD@_bi@2@@_bi@boost@@QAE@V?$arg@$00@2@V?$value@PBD@12@@Z 10003354 f i LocalizerImp.obj
 0001:00002360       ??0?$shared_ptr@VResource@LocalizerImp@@@boost@@QAE@ABV01@@Z 10003360 f i LocalizerImp.obj
 0001:00002380       ??0?$shared_ptr@VResource@LocalizerImp@@@boost@@QAE@XZ 10003380 f i LocalizerImp.obj
 0001:0000238a       ??0?$sp_counted_base_impl@PAVResource@LocalizerImp@@U?$checked_deleter@VResource@LocalizerImp@@@boost@@@detail@boost@@QAE@PAVResource@LocalizerImp@@U?$checked_deleter@VResource@LocalizerImp@@@2@@Z 1000338a f i LocalizerImp.obj
 0001:000023a9       ??0?$value@PBD@_bi@boost@@QAE@ABQBD@Z 100033a9 f i LocalizerImp.obj
 0001:000023b6       ??0?$vector@V?$basic_string@DU?$char_traits@D@std@@V?$allocator@D@2@@std@@V?$allocator@V?$basic_string@DU?$char_traits@D@std@@V?$allocator@D@2@@std@@@2@@std@@QAE@$$QAV01@@Z 100033b6 f i LocalizerImp.obj
 0001:000023d2       ??0?$vector@V?$basic_string@DU?$char_traits@D@std@@V?$allocator@D@2@@std@@V?$allocator@V?$basic_string@DU?$char_traits@D@std@@V?$allocator@D@2@@std@@@2@@std@@QAE@XZ 100033d2 f i LocalizerImp.obj
 0001:000023df       ??0?$vector@VResEntry@LocalizerImp@@V?$allocator@VResEntry@LocalizerImp@@@std@@@std@@QAE@XZ 100033df f i LocalizerImp.obj
 0001:000023ec       ??0LocalizerImp@@AAE@XZ    100033ec f   LocalizerImp.obj
 0001:000023f9       ??0ResEntry@LocalizerImp@@QAE@ABV01@@Z 100033f9 f i LocalizerImp.obj
 0001:00002419       ??0ResEntry@LocalizerImp@@QAE@XZ 10003419 f i LocalizerImp.obj
 0001:00002423       ??0bad_weak_ptr@boost@@QAE@ABV01@@Z 10003423 f i LocalizerImp.obj
 0001:0000243c       ??0bad_weak_ptr@boost@@QAE@XZ 1000343c f i LocalizerImp.obj
 0001:0000244f       ??0lightweight_mutex@detail@boost@@QAE@XZ 1000344f f i LocalizerImp.obj
 0001:00002455       ??0scoped_lock@lightweight_mutex@detail@boost@@QAE@AAV123@@Z 10003455 f i LocalizerImp.obj
 0001:0000247f       ??0shared_count@detail@boost@@QAE@ABV012@@Z 1000347f f i LocalizerImp.obj
 0001:00002499       ??0shared_count@detail@boost@@QAE@XZ 10003499 f i LocalizerImp.obj
 0001:0000249f       ??0sp_counted_base@detail@boost@@QAE@XZ 1000349f f i LocalizerImp.obj
 0001:000024b5       ??1?$Scoped@USTH@?A0x592ce793@@@@QAE@XZ 100034b5 f i LocalizerImp.obj
 0001:000024da       ??1?$auto_ptr@VResource@LocalizerImp@@@std@@QAE@XZ 100034da f i LocalizerImp.obj
 0001:000024e7       ??1?$shared_ptr@VResource@LocalizerImp@@@boost@@QAE@XZ 100034e7 f i LocalizerImp.obj
 0001:000024f3       ??1?$sp_counted_base_impl@PAVResource@LocalizerImp@@U?$checked_deleter@VResource@LocalizerImp@@@boost@@@detail@boost@@UAE@XZ 100034f3 f i LocalizerImp.obj
 0001:000024fa       ??1?$vector@VResEntry@LocalizerImp@@V?$allocator@VResEntry@LocalizerImp@@@std@@@std@@QAE@XZ 100034fa f i LocalizerImp.obj
 0001:000024ff       ??1LocalizerImp@@AAE@XZ    100034ff f   LocalizerImp.obj
 0001:0000250f       ??1ResEntry@LocalizerImp@@QAE@XZ 1000350f f i LocalizerImp.obj
 0001:0000251b       ??1Resource@LocalizerImp@@UAE@XZ 1000351b f   LocalizerImp.obj
 0001:00002522       ??1bad_weak_ptr@boost@@UAE@XZ 10003522 f i LocalizerImp.obj
 0001:00002528       ??1scoped_lock@lightweight_mutex@detail@boost@@QAE@XZ 10003528 f i LocalizerImp.obj
 0001:00002533       ??1shared_count@detail@boost@@QAE@XZ 10003533 f i LocalizerImp.obj
 0001:0000253e       ??1sp_counted_base@detail@boost@@UAE@XZ 1000353e f i LocalizerImp.obj
 0001:00002545       ??4?$shared_ptr@VResource@LocalizerImp@@@boost@@QAEAAV01@ABV01@@Z 10003545 f i LocalizerImp.obj
 0001:00002562       ??4ResEntry@LocalizerImp@@QAEAAV01@ABV01@@Z 10003562 f i LocalizerImp.obj
 0001:0000257f       ??4shared_count@detail@boost@@QAEAAV012@ABV012@@Z 1000357f f i LocalizerImp.obj
 0001:000025a8       ??8?$_Vector_const_iterator@V?$_Vector_val@U?$_Simple_types@V?$basic_string@DU?$char_traits@D@std@@V?$allocator@D@2@@std@@@std@@@std@@@std@@QBE_NABV01@@Z 100035a8 f i LocalizerImp.obj
 0001:000025b8       ??8?$_Vector_const_iterator@V?$_Vector_val@U?$_Simple_types@VResEntry@LocalizerImp@@@std@@@std@@@std@@QBE_NABV01@@Z 100035b8 f i LocalizerImp.obj
 0001:000025c8       ??9?$_Vector_const_iterator@V?$_Vector_val@U?$_Simple_types@V?$basic_string@DU?$char_traits@D@std@@V?$allocator@D@2@@std@@@std@@@std@@@std@@QBE_NABV01@@Z 100035c8 f i LocalizerImp.obj
 0001:000025d8       ??9?$_Vector_const_iterator@V?$_Vector_val@U?$_Simple_types@VResEntry@LocalizerImp@@@std@@@std@@@std@@QBE_NABV01@@Z 100035d8 f i LocalizerImp.obj
 0001:000025e8       ??A?$list1@AAVResEntry@LocalizerImp@@@_bi@boost@@QBEAAVResEntry@LocalizerImp@@V?$arg@$00@2@@Z 100035e8 f i LocalizerImp.obj
 0001:000025ed       ??B?$Scoped@USTH@?A0x592ce793@@@@QBEQ6GXXZXZ 100035ed f i LocalizerImp.obj
 0001:000025fe       ??C?$_Vector_const_iterator@V?$_Vector_val@U?$_Simple_types@V?$basic_string@DU?$char_traits@D@std@@V?$allocator@D@2@@std@@@std@@@std@@@std@@QBEPBV?$basic_string@DU?$char_traits@D@std@@V?$allocator@D@2@@1@XZ 100035fe f i LocalizerImp.obj
 0001:00002601       ??C?$_Vector_const_iterator@V?$_Vector_val@U?$_Simple_types@VResEntry@LocalizerImp@@@std@@@std@@@std@@QBEPBVResEntry@LocalizerImp@@XZ 10003601 f i LocalizerImp.obj
 0001:00002604       ??C?$_Vector_iterator@V?$_Vector_val@U?$_Simple_types@VResEntry@LocalizerImp@@@std@@@std@@@std@@QBEPAVResEntry@LocalizerImp@@XZ 10003604 f i LocalizerImp.obj
 0001:00002607       ??C?$auto_ptr@VResource@LocalizerImp@@@std@@QBEPAVResource@LocalizerImp@@XZ 10003607 f i LocalizerImp.obj
 0001:0000260a       ??C?$shared_ptr@VResource@LocalizerImp@@@boost@@QBEPAVResource@LocalizerImp@@XZ 1000360a f i LocalizerImp.obj
 0001:0000260d       ??D?$_Vector_const_iterator@V?$_Vector_val@U?$_Simple_types@V?$basic_string@DU?$char_traits@D@std@@V?$allocator@D@2@@std@@@std@@@std@@@std@@QBEABV?$basic_string@DU?$char_traits@D@std@@V?$allocator@D@2@@1@XZ 1000360d f i LocalizerImp.obj
 0001:00002610       ??D?$_Vector_const_iterator@V?$_Vector_val@U?$_Simple_types@VResEntry@LocalizerImp@@@std@@@std@@@std@@QBEABVResEntry@LocalizerImp@@XZ 10003610 f i LocalizerImp.obj
 0001:00002613       ??D?$_Vector_iterator@V?$_Vector_val@U?$_Simple_types@VResEntry@LocalizerImp@@@std@@@std@@@std@@QBEAAVResEntry@LocalizerImp@@XZ 10003613 f i LocalizerImp.obj
 0001:00002616       ??E?$_Vector_const_iterator@V?$_Vector_val@U?$_Simple_types@V?$basic_string@DU?$char_traits@D@std@@V?$allocator@D@2@@std@@@std@@@std@@@std@@QAEAAV01@XZ 10003616 f i LocalizerImp.obj
 0001:0000261c       ??E?$_Vector_const_iterator@V?$_Vector_val@U?$_Simple_types@VResEntry@LocalizerImp@@@std@@@std@@@std@@QAEAAV01@XZ 1000361c f i LocalizerImp.obj
 0001:00002622       ??E?$_Vector_iterator@V?$_Vector_val@U?$_Simple_types@VResEntry@LocalizerImp@@@std@@@std@@@std@@QAEAAV01@XZ 10003622 f i LocalizerImp.obj
 0001:00002628       ??R?$checked_deleter@VResource@LocalizerImp@@@boost@@QBEXPAVResource@LocalizerImp@@@Z 10003628 f i LocalizerImp.obj
 0001:00002639       ??Y?$basic_string@DU?$char_traits@D@std@@V?$allocator@D@2@@std@@QAEAAV01@D@Z 10003639 f i LocalizerImp.obj
 0001:00002647       ??Y?$basic_string@DU?$char_traits@D@std@@V?$allocator@D@2@@std@@QAEAAV01@PBD@Z 10003647 f i LocalizerImp.obj
 0001:00002664       ??_E?$sp_counted_base_impl@PAVResource@LocalizerImp@@U?$checked_deleter@VResource@LocalizerImp@@@boost@@@detail@boost@@UAEPAXI@Z 10003664 f i LocalizerImp.obj
 0001:00002664       ??_G?$sp_counted_base_impl@PAVResource@LocalizerImp@@U?$checked_deleter@VResource@LocalizerImp@@@boost@@@detail@boost@@UAEPAXI@Z 10003664 f i LocalizerImp.obj
 0001:00002681       ??_GLocalizerImp@@AAEPAXI@Z 10003681 f i LocalizerImp.obj
 0001:0000269d       ??_GResEntry@LocalizerImp@@QAEPAXI@Z 1000369d f i LocalizerImp.obj
 0001:000026c0       ??_Gbad_weak_ptr@boost@@UAEPAXI@Z 100036c0 f i LocalizerImp.obj
 0001:000026c0       ??_Ebad_weak_ptr@boost@@UAEPAXI@Z 100036c0 f i LocalizerImp.obj
 0001:000026dd       ??_Esp_counted_base@detail@boost@@UAEPAXI@Z 100036dd f i LocalizerImp.obj
 0001:000026dd       ??_Gsp_counted_base@detail@boost@@UAEPAXI@Z 100036dd f i LocalizerImp.obj
 0001:000026fa       ?Allocator@LocalizerImp@@SGPAU_HMEMPOOL@@XZ 100036fa f   LocalizerImp.obj
 0001:00002768       ?GetString@LocalizerImp@@QBE_NPA_WIH@Z 10003768 f   LocalizerImp.obj
 0001:000027bb       ?GetTxtResourceByFileName@LocalizerImp@@AAEPAVResource@1@PBD@Z 100037bb f   LocalizerImp.obj
 0001:0000280d       ?Initialize@LocalizerImp@@SGXXZ 1000380d f   LocalizerImp.obj
 0001:0000283c       ?Instance@LocalizerImp@@SGPAV1@XZ 1000383c f   LocalizerImp.obj
 0001:00002842       ?InternalResLoad@LocalizerImp@@AAE_NPBDP6GPAVResource@1@0@Z@Z 10003842 f   LocalizerImp.obj
 0001:00002a14       ?InternalResUnload@LocalizerImp@@AAE_NPBD@Z 10003a14 f   LocalizerImp.obj
 0001:00002a7b       ?IsNull@STH@?A0x592ce793@@QBE_NPAX@Z 10003a7b f i LocalizerImp.obj
 0001:00002cbd       ?Release@STH@?A0x592ce793@@QAEXPAX@Z 10003cbd f i LocalizerImp.obj
 0001:00002cd3       ?ResLoadFolder@LocalizerImp@@QAE?AV?$vector@V?$basic_string@DU?$char_traits@D@std@@V?$allocator@D@2@@std@@V?$allocator@V?$basic_string@DU?$char_traits@D@std@@V?$allocator@D@2@@std@@@2@@std@@PBD@Z 10003cd3 f   LocalizerImp.obj
 0001:00002e17       ?ResUnload@LocalizerImp@@QAEXABV?$vector@V?$basic_string@DU?$char_traits@D@std@@V?$allocator@D@2@@std@@V?$allocator@V?$basic_string@DU?$char_traits@D@std@@V?$allocator@D@2@@std@@@2@@std@@@Z 10003e17 f   LocalizerImp.obj
 0001:00002e48       ?ResUnload@LocalizerImp@@QAE_NPBD@Z 10003e48 f   LocalizerImp.obj
 0001:00002ec8       ?Shutdown@LocalizerImp@@SGXXZ 10003ec8 f   LocalizerImp.obj
 0001:00002efb       ?TxtAdd@LocalizerImp@@QAEHPBDHHPB_WH@Z 10003efb f   LocalizerImp.obj
 0001:00002f21       ?TxtAddRange@LocalizerImp@@QAE_NPBDI0AAH1@Z 10003f21 f   LocalizerImp.obj
 0001:00002f4b       ?TxtGetRange@LocalizerImp@@QAE_NPBDAAH1@Z 10003f4b f   LocalizerImp.obj
 0001:00002f89       ?TxtLoad@LocalizerImp@@QAE_NPBD@Z 10003f89 f   LocalizerImp.obj
 0001:00002f9a       ?TxtResetRange@LocalizerImp@@QAE_NPBDHH@Z 10003f9a f   LocalizerImp.obj
 0001:00002fbd       ?TxtSave@LocalizerImp@@QAE_NPBD@Z 10003fbd f   LocalizerImp.obj
 0001:00002fe4       ?TxtUnload@LocalizerImp@@QAE_NPBD@Z 10003fe4 f   LocalizerImp.obj
 0001:00002fe9       ?UCSLoad@LocalizerImp@@QAE_NPBD@Z 10003fe9 f   LocalizerImp.obj
 0001:00002ffa       ?UCSUnload@LocalizerImp@@QAE_NPBD@Z 10003ffa f   LocalizerImp.obj
 0001:00002fff       ?_Assign_rv@?$basic_string@DU?$char_traits@D@std@@V?$allocator@D@2@@std@@QAEX$$QAV12@@Z 10003fff f i LocalizerImp.obj
 0001:0000304b       ?_Assign_rv@?$vector@V?$basic_string@DU?$char_traits@D@std@@V?$allocator@D@2@@std@@V?$allocator@V?$basic_string@DU?$char_traits@D@std@@V?$allocator@D@2@@std@@@2@@std@@QAEX$$QAV12@@Z 1000404b f i LocalizerImp.obj
 0001:00003079       ?_Chassign@?$basic_string@DU?$char_traits@D@std@@V?$allocator@D@2@@std@@QAEXIID@Z 10004079 f i LocalizerImp.obj
 0001:000030b9       ?_Compat@?$_Vector_const_iterator@V?$_Vector_val@U?$_Simple_types@V?$basic_string@DU?$char_traits@D@std@@V?$allocator@D@2@@std@@@std@@@std@@@std@@QBEXABV12@@Z 100040b9 f i LocalizerImp.obj
 0001:000030bc       ?_Compat@?$_Vector_const_iterator@V?$_Vector_val@U?$_Simple_types@VResEntry@LocalizerImp@@@std@@@std@@@std@@QBEXABV12@@Z 100040bc f i LocalizerImp.obj
 0001:000030bf       ?_Destroy@?$vector@VResEntry@LocalizerImp@@V?$allocator@VResEntry@LocalizerImp@@@std@@@std@@IAEXPAVResEntry@LocalizerImp@@0@Z 100040bf f i LocalizerImp.obj
 0001:000030dc       ?_Getal@?$_Vector_alloc@$0A@U?$_Vec_base_types@VResEntry@LocalizerImp@@V?$allocator@VResEntry@LocalizerImp@@@std@@@std@@@std@@QBE?AU?$_Wrap_alloc@V?$allocator@VResEntry@LocalizerImp@@@std@@@2@XZ 100040dc f i LocalizerImp.obj
 0001:000030e3       ?_Grow_to@?$vector@V?$basic_string@DU?$char_traits@D@std@@V?$allocator@D@2@@std@@V?$allocator@V?$basic_string@DU?$char_traits@D@std@@V?$allocator@D@2@@std@@@2@@std@@IBEII@Z 100040e3 f i LocalizerImp.obj
 0001:00003113       ?_Grow_to@?$vector@VResEntry@LocalizerImp@@V?$allocator@VResEntry@LocalizerImp@@@std@@@std@@IBEII@Z 10004113 f i LocalizerImp.obj
 0001:0000313e       ?_Inside@?$vector@V?$basic_string@DU?$char_traits@D@std@@V?$allocator@D@2@@std@@V?$allocator@V?$basic_string@DU?$char_traits@D@std@@V?$allocator@D@2@@std@@@2@@std@@IBE_NPBV?$basic_string@DU?$char_traits@D@std@@V?$allocator@D@2@@2@@Z 1000413e f i LocalizerImp.obj
 0001:00003155       ?_Inside@?$vector@VResEntry@LocalizerImp@@V?$allocator@VResEntry@LocalizerImp@@@std@@@std@@IBE_NPBVResEntry@LocalizerImp@@@Z 10004155 f i LocalizerImp.obj
 0001:0000316c       ?_Make_iter@?$vector@VResEntry@LocalizerImp@@V?$allocator@VResEntry@LocalizerImp@@@std@@@std@@QBE?AV?$_Vector_iterator@V?$_Vector_val@U?$_Simple_types@VResEntry@LocalizerImp@@@std@@@std@@@2@V?$_Vector_const_iterator@V?$_Vector_val@U?$_Simple_types@VResEntry@LocalizerImp@@@std@@@std@@@2@@Z 1000416c f i LocalizerImp.obj
 0001:00003179       ?_Orphan_range@?$vector@V?$basic_string@DU?$char_traits@D@std@@V?$allocator@D@2@@std@@V?$allocator@V?$basic_string@DU?$char_traits@D@std@@V?$allocator@D@2@@std@@@2@@std@@IBEXPAV?$basic_string@DU?$char_traits@D@std@@V?$allocator@D@2@@2@0@Z 10004179 f i LocalizerImp.obj
 0001:0000317c       ?_Orphan_range@?$vector@VResEntry@LocalizerImp@@V?$allocator@VResEntry@LocalizerImp@@@std@@@std@@IBEXPAVResEntry@LocalizerImp@@0@Z 1000417c f i LocalizerImp.obj
 0001:0000317f       ?_Reallocate@?$vector@V?$basic_string@DU?$char_traits@D@std@@V?$allocator@D@2@@std@@V?$allocator@V?$basic_string@DU?$char_traits@D@std@@V?$allocator@D@2@@std@@@2@@std@@IAEXI@Z 1000417f f i LocalizerImp.obj
 0001:00003223       ?_Reallocate@?$vector@VResEntry@LocalizerImp@@V?$allocator@VResEntry@LocalizerImp@@@std@@@std@@IAEXI@Z 10004223 f i LocalizerImp.obj
 0001:000032c0       ?_Rechecked@?$_Vector_iterator@V?$_Vector_val@U?$_Simple_types@VResEntry@LocalizerImp@@@std@@@std@@@std@@QAEAAV12@PAVResEntry@LocalizerImp@@@Z 100042c0 f i LocalizerImp.obj
 0001:000032cb       ?_Reserve@?$vector@V?$basic_string@DU?$char_traits@D@std@@V?$allocator@D@2@@std@@V?$allocator@V?$basic_string@DU?$char_traits@D@std@@V?$allocator@D@2@@std@@@2@@std@@IAEXI@Z 100042cb f i LocalizerImp.obj
 0001:0000331b       ?_Reserve@?$vector@VResEntry@LocalizerImp@@V?$allocator@VResEntry@LocalizerImp@@@std@@@std@@IAEXI@Z 1000431b f i LocalizerImp.obj
 0001:00003363       ?_Tidy@?$vector@VResEntry@LocalizerImp@@V?$allocator@VResEntry@LocalizerImp@@@std@@@std@@IAEXXZ 10004363 f i LocalizerImp.obj
 0001:00003392       ?_Unchecked@?$_Vector_iterator@V?$_Vector_val@U?$_Simple_types@VResEntry@LocalizerImp@@@std@@@std@@@std@@QBEPAVResEntry@LocalizerImp@@XZ 10004392 f i LocalizerImp.obj
 0001:00003395       ?_Unused_capacity@?$vector@V?$basic_string@DU?$char_traits@D@std@@V?$allocator@D@2@@std@@V?$allocator@V?$basic_string@DU?$char_traits@D@std@@V?$allocator@D@2@@std@@@2@@std@@QBEIXZ 10004395 f i LocalizerImp.obj
 0001:000033a2       ?_Unused_capacity@?$vector@VResEntry@LocalizerImp@@V?$allocator@VResEntry@LocalizerImp@@@std@@@std@@QBEIXZ 100043a2 f i LocalizerImp.obj
 0001:000033ac       ?_Xlen@?$vector@V?$basic_string@DU?$char_traits@D@std@@V?$allocator@D@2@@std@@V?$allocator@V?$basic_string@DU?$char_traits@D@std@@V?$allocator@D@2@@std@@@2@@std@@IBEXXZ 100043ac f i LocalizerImp.obj
 0001:000033b8       ?_Xlen@?$vector@VResEntry@LocalizerImp@@V?$allocator@VResEntry@LocalizerImp@@@std@@@std@@IBEXXZ 100043b8 f i LocalizerImp.obj
 0001:000033c4       ?add_ref@sp_counted_base@detail@boost@@QAEXXZ 100043c4 f i LocalizerImp.obj
 0001:0000342c       ?allocate@?$_Wrap_alloc@V?$allocator@V?$basic_string@DU?$char_traits@D@std@@V?$allocator@D@2@@std@@@std@@@std@@QAEPAV?$basic_string@DU?$char_traits@D@std@@V?$allocator@D@2@@2@I@Z 1000442c f i LocalizerImp.obj
 0001:0000343a       ?allocate@?$_Wrap_alloc@V?$allocator@VResEntry@LocalizerImp@@@std@@@std@@QAEPAVResEntry@LocalizerImp@@I@Z 1000443a f i LocalizerImp.obj
 0001:00003448       ?allocate@?$allocator@V?$basic_string@DU?$char_traits@D@std@@V?$allocator@D@2@@std@@@std@@QAEPAV?$basic_string@DU?$char_traits@D@std@@V?$allocator@D@2@@2@I@Z 10004448 f i LocalizerImp.obj
 0001:00003456       ?allocate@?$allocator@VResEntry@LocalizerImp@@@std@@QAEPAVResEntry@LocalizerImp@@I@Z 10004456 f i LocalizerImp.obj
 0001:00003464       ?append@?$basic_string@DU?$char_traits@D@std@@V?$allocator@D@2@@std@@QAEAAV12@ABV12@II@Z 10004464 f i LocalizerImp.obj
 0001:00003505       ?append@?$basic_string@DU?$char_traits@D@std@@V?$allocator@D@2@@std@@QAEAAV12@ID@Z 10004505 f i LocalizerImp.obj
 0001:00003564       ?append@?$basic_string@DU?$char_traits@D@std@@V?$allocator@D@2@@std@@QAEAAV12@PBD@Z 10004564 f i LocalizerImp.obj
 0001:00003581       ?append@?$basic_string@DU?$char_traits@D@std@@V?$allocator@D@2@@std@@QAEAAV12@PBDI@Z 10004581 f i LocalizerImp.obj
 0001:0000361e       ?assign@?$char_traits@D@std@@SAPADPADID@Z 1000461e f i LocalizerImp.obj
 0001:00003635       ?begin@?$vector@V?$basic_string@DU?$char_traits@D@std@@V?$allocator@D@2@@std@@V?$allocator@V?$basic_string@DU?$char_traits@D@std@@V?$allocator@D@2@@std@@@2@@std@@QAE?AV?$_Vector_iterator@V?$_Vector_val@U?$_Simple_types@V?$basic_string@DU?$char_traits@D@std@@V?$allocator@D@2@@std@@@std@@@std@@@2@XZ 10004635 f i LocalizerImp.obj
 0001:00003640       ?begin@?$vector@V?$basic_string@DU?$char_traits@D@std@@V?$allocator@D@2@@std@@V?$allocator@V?$basic_string@DU?$char_traits@D@std@@V?$allocator@D@2@@std@@@2@@std@@QBE?AV?$_Vector_const_iterator@V?$_Vector_val@U?$_Simple_types@V?$basic_string@DU?$char_traits@D@std@@V?$allocator@D@2@@std@@@std@@@std@@@2@XZ 10004640 f i LocalizerImp.obj
 0001:0000364b       ?begin@?$vector@VResEntry@LocalizerImp@@V?$allocator@VResEntry@LocalizerImp@@@std@@@std@@QAE?AV?$_Vector_iterator@V?$_Vector_val@U?$_Simple_types@VResEntry@LocalizerImp@@@std@@@std@@@2@XZ 1000464b f i LocalizerImp.obj
 0001:00003656       ?begin@?$vector@VResEntry@LocalizerImp@@V?$allocator@VResEntry@LocalizerImp@@@std@@@std@@QBE?AV?$_Vector_const_iterator@V?$_Vector_val@U?$_Simple_types@VResEntry@LocalizerImp@@@std@@@std@@@2@XZ 10004656 f i LocalizerImp.obj
 0001:00003661       ?capacity@?$vector@V?$basic_string@DU?$char_traits@D@std@@V?$allocator@D@2@@std@@V?$allocator@V?$basic_string@DU?$char_traits@D@std@@V?$allocator@D@2@@std@@@2@@std@@QBEIXZ 10004661 f i LocalizerImp.obj
 0001:0000366d       ?capacity@?$vector@VResEntry@LocalizerImp@@V?$allocator@VResEntry@LocalizerImp@@@std@@@std@@QBEIXZ 1000466d f i LocalizerImp.obj
 0001:00003676       ?clear@?$basic_string@DU?$char_traits@D@std@@V?$allocator@D@2@@std@@QAEXXZ 10004676 f i LocalizerImp.obj
 0001:00003686       ?clear@?$vector@V?$basic_string@DU?$char_traits@D@std@@V?$allocator@D@2@@std@@V?$allocator@V?$basic_string@DU?$char_traits@D@std@@V?$allocator@D@2@@std@@@2@@std@@QAEXXZ 10004686 f i LocalizerImp.obj
 0001:000036a2       ?clear@?$vector@VResEntry@LocalizerImp@@V?$allocator@VResEntry@LocalizerImp@@@std@@@std@@QAEXXZ 100046a2 f i LocalizerImp.obj
 0001:000036be       ?construct@?$allocator@V?$basic_string@DU?$char_traits@D@std@@V?$allocator@D@2@@std@@@std@@QAEXPAV?$basic_string@DU?$char_traits@D@std@@V?$allocator@D@2@@2@ABV32@@Z 100046be f i LocalizerImp.obj
 0001:000036ed       ?construct@?$allocator@VResEntry@LocalizerImp@@@std@@QAEXPAVResEntry@LocalizerImp@@ABV34@@Z 100046ed f i LocalizerImp.obj
 0001:0000372a       ?deallocate@?$_Wrap_alloc@V?$allocator@VResEntry@LocalizerImp@@@std@@@std@@QAEXPAVResEntry@LocalizerImp@@I@Z 1000472a f i LocalizerImp.obj
 0001:00003737       ?deallocate@?$allocator@VResEntry@LocalizerImp@@@std@@QAEXPAVResEntry@LocalizerImp@@I@Z 10004737 f i LocalizerImp.obj
 0001:00003744       ?destruct@sp_counted_base@detail@boost@@UAEXXZ 10004744 f i LocalizerImp.obj
 0001:0000374f       ?dispose@?$sp_counted_base_impl@PAVResource@LocalizerImp@@U?$checked_deleter@VResource@LocalizerImp@@@boost@@@detail@boost@@UAEXXZ 1000474f f i LocalizerImp.obj
 0001:0000375d       ?empty@?$vector@V?$basic_string@DU?$char_traits@D@std@@V?$allocator@D@2@@std@@V?$allocator@V?$basic_string@DU?$char_traits@D@std@@V?$allocator@D@2@@std@@@2@@std@@QBE_NXZ 1000475d f i LocalizerImp.obj
 0001:00003768       ?end@?$vector@V?$basic_string@DU?$char_traits@D@std@@V?$allocator@D@2@@std@@V?$allocator@V?$basic_string@DU?$char_traits@D@std@@V?$allocator@D@2@@std@@@2@@std@@QAE?AV?$_Vector_iterator@V?$_Vector_val@U?$_Simple_types@V?$basic_string@DU?$char_traits@D@std@@V?$allocator@D@2@@std@@@std@@@std@@@2@XZ 10004768 f i LocalizerImp.obj
 0001:00003774       ?end@?$vector@V?$basic_string@DU?$char_traits@D@std@@V?$allocator@D@2@@std@@V?$allocator@V?$basic_string@DU?$char_traits@D@std@@V?$allocator@D@2@@std@@@2@@std@@QBE?AV?$_Vector_const_iterator@V?$_Vector_val@U?$_Simple_types@V?$basic_string@DU?$char_traits@D@std@@V?$allocator@D@2@@std@@@std@@@std@@@2@XZ 10004774 f i LocalizerImp.obj
 0001:00003780       ?end@?$vector@VResEntry@LocalizerImp@@V?$allocator@VResEntry@LocalizerImp@@@std@@@std@@QAE?AV?$_Vector_iterator@V?$_Vector_val@U?$_Simple_types@VResEntry@LocalizerImp@@@std@@@std@@@2@XZ 10004780 f i LocalizerImp.obj
 0001:0000378c       ?end@?$vector@VResEntry@LocalizerImp@@V?$allocator@VResEntry@LocalizerImp@@@std@@@std@@QBE?AV?$_Vector_const_iterator@V?$_Vector_val@U?$_Simple_types@VResEntry@LocalizerImp@@@std@@@std@@@2@XZ 1000478c f i LocalizerImp.obj
 0001:00003798       ?erase@?$vector@VResEntry@LocalizerImp@@V?$allocator@VResEntry@LocalizerImp@@@std@@@std@@QAE?AV?$_Vector_iterator@V?$_Vector_val@U?$_Simple_types@VResEntry@LocalizerImp@@@std@@@std@@@2@V?$_Vector_const_iterator@V?$_Vector_val@U?$_Simple_types@VResEntry@LocalizerImp@@@std@@@std@@@2@@Z 10004798 f i LocalizerImp.obj
 0001:000037d1       ?get@?$Scoped@USTH@?A0x592ce793@@@@QAEPAXXZ 100047d1 f i LocalizerImp.obj
 0001:000037d4       ?get@?$auto_ptr@VResource@LocalizerImp@@@std@@QBEPAVResource@LocalizerImp@@XZ 100047d4 f i LocalizerImp.obj
 0001:000037d7       ?get@?$shared_ptr@VResource@LocalizerImp@@@boost@@QBEPAVResource@LocalizerImp@@XZ 100047d7 f i LocalizerImp.obj
 0001:000037da       ?get@?$value@PBD@_bi@boost@@QBEABQBDXZ 100047da f i LocalizerImp.obj
 0001:000037dd       ?get_deleter@?$sp_counted_base_impl@PAVResource@LocalizerImp@@U?$checked_deleter@VResource@LocalizerImp@@@boost@@@detail@boost@@UAEPAXABVtype_info@@@Z 100047dd f i LocalizerImp.obj
 0001:000037ff       ?max_size@?$_Wrap_alloc@V?$allocator@V?$basic_string@DU?$char_traits@D@std@@V?$allocator@D@2@@std@@@std@@@std@@QBEIXZ 100047ff f i LocalizerImp.obj
 0001:00003805       ?max_size@?$_Wrap_alloc@V?$allocator@VResEntry@LocalizerImp@@@std@@@std@@QBEIXZ 10004805 f i LocalizerImp.obj
 0001:0000380b       ?max_size@?$allocator@V?$basic_string@DU?$char_traits@D@std@@V?$allocator@D@2@@std@@@std@@QBEIXZ 1000480b f i LocalizerImp.obj
 0001:00003811       ?max_size@?$allocator@VResEntry@LocalizerImp@@@std@@QBEIXZ 10004811 f i LocalizerImp.obj
 0001:00003817       ?max_size@?$allocator_traits@V?$allocator@V?$basic_string@DU?$char_traits@D@std@@V?$allocator@D@2@@std@@@std@@@std@@SGIABV?$allocator@V?$basic_string@DU?$char_traits@D@std@@V?$allocator@D@2@@std@@@2@@Z 10004817 f i LocalizerImp.obj
 0001:0000381f       ?max_size@?$allocator_traits@V?$allocator@VResEntry@LocalizerImp@@@std@@@std@@SGIABV?$allocator@VResEntry@LocalizerImp@@@2@@Z 1000481f f i LocalizerImp.obj
 0001:00003827       ?max_size@?$vector@V?$basic_string@DU?$char_traits@D@std@@V?$allocator@D@2@@std@@V?$allocator@V?$basic_string@DU?$char_traits@D@std@@V?$allocator@D@2@@std@@@2@@std@@QBEIXZ 10004827 f i LocalizerImp.obj
 0001:0000382d       ?max_size@?$vector@VResEntry@LocalizerImp@@V?$allocator@VResEntry@LocalizerImp@@@std@@@std@@QBEIXZ 1000482d f i LocalizerImp.obj
 0001:00003833       ?pointer_to@?$pointer_traits@PAVResEntry@LocalizerImp@@@std@@SGPAVResEntry@LocalizerImp@@AAV34@@Z 10004833 f i LocalizerImp.obj
 0001:0000383a       ?pointer_to@?$pointer_traits@PBV?$basic_string@DU?$char_traits@D@std@@V?$allocator@D@2@@std@@@std@@SGPBV?$basic_string@DU?$char_traits@D@std@@V?$allocator@D@2@@2@ABV32@@Z 1000483a f i LocalizerImp.obj
 0001:00003841       ?pointer_to@?$pointer_traits@PBVResEntry@LocalizerImp@@@std@@SGPBVResEntry@LocalizerImp@@ABV34@@Z 10004841 f i LocalizerImp.obj
 0001:00003848       ?push_back@?$vector@V?$basic_string@DU?$char_traits@D@std@@V?$allocator@D@2@@std@@V?$allocator@V?$basic_string@DU?$char_traits@D@std@@V?$allocator@D@2@@std@@@2@@std@@QAEXABV?$basic_string@DU?$char_traits@D@std@@V?$allocator@D@2@@2@@Z 10004848 f i LocalizerImp.obj
 0001:000038dc       ?push_back@?$vector@VResEntry@LocalizerImp@@V?$allocator@VResEntry@LocalizerImp@@@std@@@std@@QAEXABVResEntry@LocalizerImp@@@Z 100048dc f i LocalizerImp.obj
 0001:00003937       ?release@?$auto_ptr@VResource@LocalizerImp@@@std@@QAEPAVResource@LocalizerImp@@XZ 10004937 f i LocalizerImp.obj
 0001:0000393d       ?release@sp_counted_base@detail@boost@@QAEXXZ 1000493d f i LocalizerImp.obj
 0001:0000397c       ?select_on_container_copy_construction@?$_Wrap_alloc@V?$allocator@D@std@@@std@@QBE?AU12@XZ 1000497c f i LocalizerImp.obj
 0001:00003983       ?select_on_container_copy_construction@?$allocator@D@std@@QBE?AV12@XZ 10004983 f i LocalizerImp.obj
 0001:0000398a       ?select_on_container_copy_construction@?$allocator_traits@V?$allocator@D@std@@@std@@SG?AV?$allocator@D@2@ABV32@@Z 1000498a f i LocalizerImp.obj
 0001:00003991       ?size@?$vector@V?$basic_string@DU?$char_traits@D@std@@V?$allocator@D@2@@std@@V?$allocator@V?$basic_string@DU?$char_traits@D@std@@V?$allocator@D@2@@std@@@2@@std@@QBEIXZ 10004991 f i LocalizerImp.obj
 0001:0000399d       ?size@?$vector@VResEntry@LocalizerImp@@V?$allocator@VResEntry@LocalizerImp@@@std@@@std@@QBEIXZ 1000499d f i LocalizerImp.obj
 0001:000039a6       ?sp_enable_shared_from_this@detail@boost@@YGXPBX0ABVshared_count@12@@Z 100049a6 f i LocalizerImp.obj
 0001:000039a9       ?swap@?$shared_ptr@VResource@LocalizerImp@@@boost@@QAEXAAV12@@Z 100049a9 f i LocalizerImp.obj
 0001:000039c6       ?swap@shared_count@detail@boost@@QAEXAAV123@@Z 100049c6 f i LocalizerImp.obj
 0001:000039d7       ?weak_release@sp_counted_base@detail@boost@@QAEXXZ 100049d7 f i LocalizerImp.obj
 0001:00003a0b       ?what@bad_weak_ptr@boost@@UBEPBDXZ 10004a0b f i LocalizerImp.obj
 0001:00003a11       ??$?0AAHAAULine@LocalizerResourceTxt@@@?$pair@HULine@LocalizerResourceTxt@@@std@@QAE@AAHAAULine@LocalizerResourceTxt@@PAPAX@Z 10004a11 f i LocalizerTxt.obj
 0001:00003a2c       ??$?0AAPAU?$pair@HULine@LocalizerResourceTxt@@@std@@AAPAU01@@?$pair@PAU?$pair@HULine@LocalizerResourceTxt@@@std@@PAU12@@std@@QAE@AAPAU?$pair@HULine@LocalizerResourceTxt@@@1@0PAPAX@Z 10004a2c f i LocalizerTxt.obj
 0001:00003a42       ??$?0AAPAURange@LocalizerResourceTxt@@AAPAU01@@?$pair@PAURange@LocalizerResourceTxt@@PAU12@@std@@QAE@AAPAURange@LocalizerResourceTxt@@0PAPAX@Z 10004a42 f i LocalizerTxt.obj
 0001:00003a58       ??$?0AAPBU?$pair@HULine@LocalizerResourceTxt@@@std@@AAPBU01@@?$pair@PBU?$pair@HULine@LocalizerResourceTxt@@@std@@PBU12@@std@@QAE@AAPBU?$pair@HULine@LocalizerResourceTxt@@@1@0PAPAX@Z 10004a58 f i LocalizerTxt.obj
 0001:00003a6e       ??$?0AAV?$_Vector_const_iterator@V?$_Vector_val@U?$_Simple_types@U?$pair@HULine@LocalizerResourceTxt@@@std@@@std@@@std@@@std@@AAV01@@?$pair@V?$_Vector_const_iterator@V?$_Vector_val@U?$_Simple_types@U?$pair@HULine@LocalizerResourceTxt@@@std@@@std@@@std@@@std@@V12@@std@@QAE@AAV?$_Vector_const_iterator@V?$_Vector_val@U?$_Simple_types@U?$pair@HULine@LocalizerResourceTxt@@@std@@@std@@@std@@@1@0PAPAX@Z 10004a6e f i LocalizerTxt.obj
 0001:00003a84       ??$?0AAV?$_Vector_iterator@V?$_Vector_val@U?$_Simple_types@U?$pair@HULine@LocalizerResourceTxt@@@std@@@std@@@std@@@std@@AAV01@@?$pair@V?$_Vector_iterator@V?$_Vector_val@U?$_Simple_types@U?$pair@HULine@LocalizerResourceTxt@@@std@@@std@@@std@@@std@@V12@@std@@QAE@AAV?$_Vector_iterator@V?$_Vector_val@U?$_Simple_types@U?$pair@HULine@LocalizerResourceTxt@@@std@@@std@@@std@@@1@0PAPAX@Z 10004a84 f i LocalizerTxt.obj
 0001:00003a9a       ??$?0PAU?$pair@HULine@LocalizerResourceTxt@@@std@@PAU01@@?$pair@PAU?$pair@HULine@LocalizerResourceTxt@@@std@@PAU12@@std@@QAE@$$QAU01@PAPAX@Z 10004a9a f i LocalizerTxt.obj
 0001:00003aad       ??$?0PAURange@LocalizerResourceTxt@@PAU01@@?$pair@PAURange@LocalizerResourceTxt@@PAU12@@std@@QAE@$$QAU01@PAPAX@Z 10004aad f i LocalizerTxt.obj
 0001:00003ac0       ??$?0PBU?$pair@HULine@LocalizerResourceTxt@@@std@@PBU01@@?$pair@PBU?$pair@HULine@LocalizerResourceTxt@@@std@@PBU12@@std@@QAE@$$QAU01@PAPAX@Z 10004ac0 f i LocalizerTxt.obj
 0001:00003ad3       ??$?0U?$_Wrap_alloc@V?$mempool_alloc@U?$pair@HULine@LocalizerResourceTxt@@@std@@@@@std@@@?$_Wrap_alloc@V?$mempool_alloc@U?$pair@HULine@LocalizerResourceTxt@@@std@@@@@std@@QAE@AAU01@@Z 10004ad3 f i LocalizerTxt.obj
 0001:00003ae0       ??$?0U?$_Wrap_alloc@V?$mempool_alloc@URange@LocalizerResourceTxt@@@@@std@@@?$_Wrap_alloc@V?$mempool_alloc@URange@LocalizerResourceTxt@@@@@std@@QAE@AAU01@@Z 10004ae0 f i LocalizerTxt.obj
 0001:00003aed       ??$?0V?$_Vector_const_iterator@V?$_Vector_val@U?$_Simple_types@U?$pair@HULine@LocalizerResourceTxt@@@std@@@std@@@std@@@std@@V01@@?$pair@V?$_Vector_const_iterator@V?$_Vector_val@U?$_Simple_types@U?$pair@HULine@LocalizerResourceTxt@@@std@@@std@@@std@@@std@@V12@@std@@QAE@$$QAU01@PAPAX@Z 10004aed f i LocalizerTxt.obj
 0001:00003b00       ??$?0V?$_Vector_iterator@V?$_Vector_val@U?$_Simple_types@U?$pair@HULine@LocalizerResourceTxt@@@std@@@std@@@std@@@std@@V01@@?$pair@V?$_Vector_iterator@V?$_Vector_val@U?$_Simple_types@U?$pair@HULine@LocalizerResourceTxt@@@std@@@std@@@std@@@std@@V12@@std@@QAE@$$QAU01@PAPAX@Z 10004b00 f i LocalizerTxt.obj
 0001:00003b13       ??$?HDU?$char_traits@D@std@@V?$allocator@D@1@@std@@YG?AV?$basic_string@DU?$char_traits@D@std@@V?$allocator@D@2@@0@ABV10@PBD@Z 10004b13 f i LocalizerTxt.obj
 0001:00003b8b       ??$_Adjust_heap@PAURange@LocalizerResourceTxt@@HU12@VRangeArrayLess@?A0x10e53216@@@std@@YGXPAURange@LocalizerResourceTxt@@HH$$QAU12@VRangeArrayLess@?A0x10e53216@@@Z 10004b8b f i LocalizerTxt.obj
 0001:00003c07       ??$_Advance@PAU?$pair@HULine@LocalizerResourceTxt@@@std@@H@std@@YGXAAPAU?$pair@HULine@LocalizerResourceTxt@@@0@HUrandom_access_iterator_tag@0@@Z 10004c07 f i LocalizerTxt.obj
 0001:00003c17       ??$_Advance@PBU?$pair@HULine@LocalizerResourceTxt@@@std@@H@std@@YGXAAPBU?$pair@HULine@LocalizerResourceTxt@@@0@HUrandom_access_iterator_tag@0@@Z 10004c17 f i LocalizerTxt.obj
 0001:00003c27       ??$_Advance@V?$_Vector_iterator@V?$_Vector_val@U?$_Simple_types@U?$pair@HULine@LocalizerResourceTxt@@@std@@@std@@@std@@@std@@H@std@@YGXAAV?$_Vector_iterator@V?$_Vector_val@U?$_Simple_types@U?$pair@HULine@LocalizerResourceTxt@@@std@@@std@@@std@@@0@HUrandom_access_iterator_tag@0@@Z 10004c27 f i LocalizerTxt.obj
 0001:00003c37       ??$_Destroy_range@U?$_Wrap_alloc@V?$mempool_alloc@U?$pair@HULine@LocalizerResourceTxt@@@std@@@@@std@@@std@@YGXPAU?$pair@HULine@LocalizerResourceTxt@@@0@0AAU?$_Wrap_alloc@V?$mempool_alloc@U?$pair@HULine@LocalizerResourceTxt@@@std@@@@@0@@Z 10004c37 f i LocalizerTxt.obj
 0001:00003c3a       ??$_Destroy_range@U?$_Wrap_alloc@V?$mempool_alloc@U?$pair@HULine@LocalizerResourceTxt@@@std@@@@@std@@@std@@YGXPAU?$pair@HULine@LocalizerResourceTxt@@@0@0AAU?$_Wrap_alloc@V?$mempool_alloc@U?$pair@HULine@LocalizerResourceTxt@@@std@@@@@0@U_Nonscalar_ptr_iterator_tag@0@@Z 10004c3a f i LocalizerTxt.obj
 0001:00003c3d       ??$_Destroy_range@U?$_Wrap_alloc@V?$mempool_alloc@URange@LocalizerResourceTxt@@@@@std@@@std@@YGXPAURange@LocalizerResourceTxt@@0AAU?$_Wrap_alloc@V?$mempool_alloc@URange@LocalizerResourceTxt@@@@@0@@Z 10004c3d f i LocalizerTxt.obj
 0001:00003c40       ??$_Destroy_range@U?$_Wrap_alloc@V?$mempool_alloc@URange@LocalizerResourceTxt@@@@@std@@@std@@YGXPAURange@LocalizerResourceTxt@@0AAU?$_Wrap_alloc@V?$mempool_alloc@URange@LocalizerResourceTxt@@@@@0@U_Nonscalar_ptr_iterator_tag@0@@Z 10004c40 f i LocalizerTxt.obj
 0001:00003c43       ??$_Dist_type@PAU?$pair@HULine@LocalizerResourceTxt@@@std@@@std@@YGPAHPAU?$pair@HULine@LocalizerResourceTxt@@@0@@Z 10004c43 f i LocalizerTxt.obj
 0001:00003c48       ??$_Dist_type@PAURange@LocalizerResourceTxt@@@std@@YGPAHPAURange@LocalizerResourceTxt@@@Z 10004c48 f i LocalizerTxt.obj
 0001:00003c4d       ??$_Dist_type@PBU?$pair@HULine@LocalizerResourceTxt@@@std@@@std@@YGPAHPBU?$pair@HULine@LocalizerResourceTxt@@@0@@Z 10004c4d f i LocalizerTxt.obj
 0001:00003c52       ??$_Dist_type@V?$_Vector_const_iterator@V?$_Vector_val@U?$_Simple_types@U?$pair@HULine@LocalizerResourceTxt@@@std@@@std@@@std@@@std@@@std@@YGPAHV?$_Vector_const_iterator@V?$_Vector_val@U?$_Simple_types@U?$pair@HULine@LocalizerResourceTxt@@@std@@@std@@@std@@@0@@Z 10004c52 f i LocalizerTxt.obj
 0001:00003c57       ??$_Dist_type@V?$_Vector_iterator@V?$_Vector_val@U?$_Simple_types@U?$pair@HULine@LocalizerResourceTxt@@@std@@@std@@@std@@@std@@@std@@YGPAHV?$_Vector_iterator@V?$_Vector_val@U?$_Simple_types@U?$pair@HULine@LocalizerResourceTxt@@@std@@@std@@@std@@@0@@Z 10004c57 f i LocalizerTxt.obj
 0001:00003c5c       ??$_Distance2@PAU?$pair@HULine@LocalizerResourceTxt@@@std@@H@std@@YGXPAU?$pair@HULine@LocalizerResourceTxt@@@0@0AAHUrandom_access_iterator_tag@0@@Z 10004c5c f i LocalizerTxt.obj
 0001:00003c70       ??$_Distance2@PBU?$pair@HULine@LocalizerResourceTxt@@@std@@H@std@@YGXPBU?$pair@HULine@LocalizerResourceTxt@@@0@0AAHUrandom_access_iterator_tag@0@@Z 10004c70 f i LocalizerTxt.obj
 0001:00003c84       ??$_Distance2@V?$_Vector_iterator@V?$_Vector_val@U?$_Simple_types@U?$pair@HULine@LocalizerResourceTxt@@@std@@@std@@@std@@@std@@H@std@@YGXV?$_Vector_iterator@V?$_Vector_val@U?$_Simple_types@U?$pair@HULine@LocalizerResourceTxt@@@std@@@std@@@std@@@0@0AAHUrandom_access_iterator_tag@0@@Z 10004c84 f i LocalizerTxt.obj
 0001:00003c98       ??$_Distance@PAU?$pair@HULine@LocalizerResourceTxt@@@std@@H@std@@YGXPAU?$pair@HULine@LocalizerResourceTxt@@@0@0AAH@Z 10004c98 f i LocalizerTxt.obj
 0001:00003cac       ??$_Distance@PBU?$pair@HULine@LocalizerResourceTxt@@@std@@H@std@@YGXPBU?$pair@HULine@LocalizerResourceTxt@@@0@0AAH@Z 10004cac f i LocalizerTxt.obj
 0001:00003cc0       ??$_Equal_range@PAU?$pair@HULine@LocalizerResourceTxt@@@std@@HHVLineArrayLess@?A0x10e53216@@@std@@YG?AU?$pair@PAU?$pair@HULine@LocalizerResourceTxt@@@std@@PAU12@@0@PAU?$pair@HULine@LocalizerResourceTxt@@@0@0ABHVLineArrayLess@?A0x10e53216@@PAH@Z 10004cc0 f i LocalizerTxt.obj
 0001:00003d4a       ??$_Equal_range@PBU?$pair@HULine@LocalizerResourceTxt@@@std@@HHVLineArrayLess@?A0x10e53216@@@std@@YG?AU?$pair@PBU?$pair@HULine@LocalizerResourceTxt@@@std@@PBU12@@0@PBU?$pair@HULine@LocalizerResourceTxt@@@0@0ABHVLineArrayLess@?A0x10e53216@@PAH@Z 10004d4a f i LocalizerTxt.obj
 0001:00003dd4       ??$_Fn@V?$mempool_alloc@U?$pair@HULine@LocalizerResourceTxt@@@std@@@@@_Alloc_max_size@std@@SGIU_Wrap_int@1@ABV?$mempool_alloc@U?$pair@HULine@LocalizerResourceTxt@@@std@@@@@Z 10004dd4 f i LocalizerTxt.obj
 0001:00003dda       ??$_Fn@V?$mempool_alloc@U?$pair@HULine@LocalizerResourceTxt@@@std@@@@U?$pair@HULine@LocalizerResourceTxt@@@std@@@_Alloc_destroy@std@@SGXHAAV?$mempool_alloc@U?$pair@HULine@LocalizerResourceTxt@@@std@@@@PAU?$pair@HULine@LocalizerResourceTxt@@@1@@Z 10004dda f i LocalizerTxt.obj
 0001:00003ddd       ??$_Fn@V?$mempool_alloc@U?$pair@HULine@LocalizerResourceTxt@@@std@@@@U?$pair@HULine@LocalizerResourceTxt@@@std@@U23@@_Alloc_construct@std@@SGXHAAV?$mempool_alloc@U?$pair@HULine@LocalizerResourceTxt@@@std@@@@PAU?$pair@HULine@LocalizerResourceTxt@@@1@$$QAU31@@Z 10004ddd f i LocalizerTxt.obj
 0001:00003df4       ??$_Fn@V?$mempool_alloc@URange@LocalizerResourceTxt@@@@@_Alloc_max_size@std@@SGIU_Wrap_int@1@ABV?$mempool_alloc@URange@LocalizerResourceTxt@@@@@Z 10004df4 f i LocalizerTxt.obj
 0001:00003dfa       ??$_Fn@V?$mempool_alloc@URange@LocalizerResourceTxt@@@@URange@LocalizerResourceTxt@@@_Alloc_destroy@std@@SGXHAAV?$mempool_alloc@URange@LocalizerResourceTxt@@@@PAURange@LocalizerResourceTxt@@@Z 10004dfa f i LocalizerTxt.obj
 0001:00003dfd       ??$_Fn@V?$mempool_alloc@URange@LocalizerResourceTxt@@@@URange@LocalizerResourceTxt@@AAU23@@_Alloc_construct@std@@SGXHAAV?$mempool_alloc@URange@LocalizerResourceTxt@@@@PAURange@LocalizerResourceTxt@@AAU34@@Z 10004dfd f i LocalizerTxt.obj
 0001:00003e13       ??$_Fn@V?$mempool_alloc@URange@LocalizerResourceTxt@@@@URange@LocalizerResourceTxt@@ABU23@@_Alloc_construct@std@@SGXHAAV?$mempool_alloc@URange@LocalizerResourceTxt@@@@PAURange@LocalizerResourceTxt@@ABU34@@Z 10004e13 f i LocalizerTxt.obj
 0001:00003e29       ??$_Fn@V?$mempool_alloc@URange@LocalizerResourceTxt@@@@URange@LocalizerResourceTxt@@U23@@_Alloc_construct@std@@SGXHAAV?$mempool_alloc@URange@LocalizerResourceTxt@@@@PAURange@LocalizerResourceTxt@@$$QAU34@@Z 10004e29 f i LocalizerTxt.obj
 0001:00003e3f       ??$_For_each@PAU?$pair@HULine@LocalizerResourceTxt@@@std@@P6GXAAU12@@Z@std@@YGXPAU?$pair@HULine@LocalizerResourceTxt@@@0@0AAP6GXAAU10@@Z@Z 10004e3f f i LocalizerTxt.obj
 0001:00003e60       ??$_For_each@PAURange@LocalizerResourceTxt@@P6GXAAU12@@Z@std@@YGXPAURange@LocalizerResourceTxt@@0AAP6GXAAU12@@Z@Z 10004e60 f i LocalizerTxt.obj
 0001:00003e81       ??$_Insertion_sort1@PAURange@LocalizerResourceTxt@@VRangeArrayLess@?A0x10e53216@@U12@@std@@YGXPAURange@LocalizerResourceTxt@@0VRangeArrayLess@?A0x10e53216@@0@Z 10004e81 f i LocalizerTxt.obj
 0001:00003ef1       ??$_Insertion_sort@PAURange@LocalizerResourceTxt@@VRangeArrayLess@?A0x10e53216@@@std@@YGXPAURange@LocalizerResourceTxt@@0VRangeArrayLess@?A0x10e53216@@@Z 10004ef1 f i LocalizerTxt.obj
 0001:00003f07       ??$_Iter_cat@PAU?$pair@HULine@LocalizerResourceTxt@@@std@@@std@@YG?AUrandom_access_iterator_tag@0@ABQAU?$pair@HULine@LocalizerResourceTxt@@@0@@Z 10004f07 f i LocalizerTxt.obj
 0001:00003f0e       ??$_Iter_cat@PBU?$pair@HULine@LocalizerResourceTxt@@@std@@@std@@YG?AUrandom_access_iterator_tag@0@ABQBU?$pair@HULine@LocalizerResourceTxt@@@0@@Z 10004f0e f i LocalizerTxt.obj
 0001:00003f15       ??$_Iter_cat@V?$_Vector_iterator@V?$_Vector_val@U?$_Simple_types@U?$pair@HULine@LocalizerResourceTxt@@@std@@@std@@@std@@@std@@@std@@YG?AUrandom_access_iterator_tag@0@ABV?$_Vector_iterator@V?$_Vector_val@U?$_Simple_types@U?$pair@HULine@LocalizerResourceTxt@@@std@@@std@@@std@@@0@@Z 10004f15 f i LocalizerTxt.obj
 0001:00003f1c       ??$_Lower_bound@PAU?$pair@HULine@LocalizerResourceTxt@@@std@@HHVLineArrayLess@?A0x10e53216@@@std@@YGPAU?$pair@HULine@LocalizerResourceTxt@@@0@PAU10@0ABHVLineArrayLess@?A0x10e53216@@PAH@Z 10004f1c f i LocalizerTxt.obj
 0001:00003f63       ??$_Lower_bound@PBU?$pair@HULine@LocalizerResourceTxt@@@std@@HHVLineArrayLess@?A0x10e53216@@@std@@YGPBU?$pair@HULine@LocalizerResourceTxt@@@0@PBU10@0ABHVLineArrayLess@?A0x10e53216@@PAH@Z 10004f63 f i LocalizerTxt.obj
 0001:00003faa       ??$_Make_heap@PAURange@LocalizerResourceTxt@@HU12@VRangeArrayLess@?A0x10e53216@@@std@@YGXPAURange@LocalizerResourceTxt@@0VRangeArrayLess@?A0x10e53216@@PAH0@Z 10004faa f i LocalizerTxt.obj
 0001:0000400e       ??$_Med3@PAURange@LocalizerResourceTxt@@VRangeArrayLess@?A0x10e53216@@@std@@YGXPAURange@LocalizerResourceTxt@@00VRangeArrayLess@?A0x10e53216@@@Z 1000500e f i LocalizerTxt.obj
 0001:00004079       ??$_Median@PAURange@LocalizerResourceTxt@@VRangeArrayLess@?A0x10e53216@@@std@@YGXPAURange@LocalizerResourceTxt@@00VRangeArrayLess@?A0x10e53216@@@Z 10005079 f i LocalizerTxt.obj
 0001:00004110       ??$_Move@AAH@std@@YG$$QAHAAH@Z 10005110 f i LocalizerTxt.obj
 0001:00004117       ??$_Move@AAULine@LocalizerResourceTxt@@@std@@YG$$QAULine@LocalizerResourceTxt@@AAU12@@Z 10005117 f i LocalizerTxt.obj
 0001:0000411e       ??$_Move@AAURange@LocalizerResourceTxt@@@std@@YG$$QAURange@LocalizerResourceTxt@@AAU12@@Z 1000511e f i LocalizerTxt.obj
 0001:00004125       ??$_Move@PAU?$pair@HULine@LocalizerResourceTxt@@@std@@PAU12@@std@@YGPAU?$pair@HULine@LocalizerResourceTxt@@@0@PAU10@00@Z 10005125 f i LocalizerTxt.obj
 0001:0000413d       ??$_Move@PAU?$pair@HULine@LocalizerResourceTxt@@@std@@PAU12@@std@@YGPAU?$pair@HULine@LocalizerResourceTxt@@@0@PAU10@00U_Nonscalar_ptr_iterator_tag@0@@Z 1000513d f i LocalizerTxt.obj
 0001:0000416d       ??$_Move_backward@PAURange@LocalizerResourceTxt@@PAU12@@std@@YGPAURange@LocalizerResourceTxt@@PAU12@00@Z 1000516d f i LocalizerTxt.obj
 0001:00004185       ??$_Move_backward@PAURange@LocalizerResourceTxt@@PAU12@@std@@YGPAURange@LocalizerResourceTxt@@PAU12@00U_Nonscalar_ptr_iterator_tag@0@@Z 10005185 f i LocalizerTxt.obj
 0001:000041ad       ??$_Pop_heap@PAURange@LocalizerResourceTxt@@HU12@VRangeArrayLess@?A0x10e53216@@@std@@YGXPAURange@LocalizerResourceTxt@@00$$QAU12@VRangeArrayLess@?A0x10e53216@@PAH@Z 100051ad f i LocalizerTxt.obj
 0001:000041de       ??$_Pop_heap@PAURange@LocalizerResourceTxt@@VRangeArrayLess@?A0x10e53216@@@std@@YGXPAURange@LocalizerResourceTxt@@0VRangeArrayLess@?A0x10e53216@@@Z 100051de f i LocalizerTxt.obj
 0001:000041f4       ??$_Pop_heap_0@PAURange@LocalizerResourceTxt@@U12@VRangeArrayLess@?A0x10e53216@@@std@@YGXPAURange@LocalizerResourceTxt@@0VRangeArrayLess@?A0x10e53216@@0@Z 100051f4 f i LocalizerTxt.obj
 0001:00004236       ??$_Ptr_cat@U?$pair@HULine@LocalizerResourceTxt@@@std@@U12@@std@@YG?AU_Nonscalar_ptr_iterator_tag@0@PAU?$pair@HULine@LocalizerResourceTxt@@@0@0@Z 10005236 f i LocalizerTxt.obj
 0001:0000423f       ??$_Ptr_cat@URange@LocalizerResourceTxt@@U12@@std@@YG?AU_Nonscalar_ptr_iterator_tag@0@PAURange@LocalizerResourceTxt@@0@Z 1000523f f i LocalizerTxt.obj
 0001:00004248       ??$_Push_heap@PAURange@LocalizerResourceTxt@@HU12@VRangeArrayLess@?A0x10e53216@@@std@@YGXPAURange@LocalizerResourceTxt@@HH$$QAU12@VRangeArrayLess@?A0x10e53216@@@Z 10005248 f i LocalizerTxt.obj
 0001:00004297       ??$_Rechecked@PAU?$pair@HULine@LocalizerResourceTxt@@@std@@PAU12@@std@@YGAAPAU?$pair@HULine@LocalizerResourceTxt@@@0@AAPAU10@PAU10@@Z 10005297 f i LocalizerTxt.obj
 0001:000042a4       ??$_Rechecked@PBU?$pair@HULine@LocalizerResourceTxt@@@std@@PBU12@@std@@YGAAPBU?$pair@HULine@LocalizerResourceTxt@@@0@AAPBU10@PBU10@@Z 100052a4 f i LocalizerTxt.obj
 0001:000042b1       ??$_Rechecked@V?$_Vector_val@U?$_Simple_types@U?$pair@HULine@LocalizerResourceTxt@@@std@@@std@@@std@@@std@@YGAAV?$_Vector_const_iterator@V?$_Vector_val@U?$_Simple_types@U?$pair@HULine@LocalizerResourceTxt@@@std@@@std@@@std@@@0@AAV10@PBU?$pair@HULine@LocalizerResourceTxt@@@0@@Z 100052b1 f i LocalizerTxt.obj
 0001:000042be       ??$_Rechecked@V?$_Vector_val@U?$_Simple_types@U?$pair@HULine@LocalizerResourceTxt@@@std@@@std@@@std@@@std@@YGAAV?$_Vector_iterator@V?$_Vector_val@U?$_Simple_types@U?$pair@HULine@LocalizerResourceTxt@@@std@@@std@@@std@@@0@AAV10@PAU?$pair@HULine@LocalizerResourceTxt@@@0@@Z 100052be f i LocalizerTxt.obj
 0001:000042cb       ??$_Rotate@PAU?$pair@HULine@LocalizerResourceTxt@@@std@@@std@@YGXPAU?$pair@HULine@LocalizerResourceTxt@@@0@00Urandom_access_iterator_tag@0@@Z 100052cb f i LocalizerTxt.obj
 0001:000042e3       ??$_Rotate@PAU?$pair@HULine@LocalizerResourceTxt@@@std@@HU12@@std@@YGXPAU?$pair@HULine@LocalizerResourceTxt@@@0@00PAH0@Z 100052e3 f i LocalizerTxt.obj
 0001:0000438d       ??$_Sort@PAURange@LocalizerResourceTxt@@HVRangeArrayLess@?A0x10e53216@@@std@@YGXPAURange@LocalizerResourceTxt@@0HVRangeArrayLess@?A0x10e53216@@@Z 1000538d f i LocalizerTxt.obj
 0001:00004463       ??$_Sort_heap@PAURange@LocalizerResourceTxt@@VRangeArrayLess@?A0x10e53216@@@std@@YGXPAURange@LocalizerResourceTxt@@0VRangeArrayLess@?A0x10e53216@@@Z 10005463 f i LocalizerTxt.obj
 0001:00004499       ??$_Swap_adl@H@std@@YGXAAH0@Z 10005499 f i LocalizerTxt.obj
 0001:000044ae       ??$_Swap_adl@ULine@LocalizerResourceTxt@@@std@@YGXAAULine@LocalizerResourceTxt@@0@Z 100054ae f i LocalizerTxt.obj
 0001:000044d7       ??$_Umove@PAU?$pair@HULine@LocalizerResourceTxt@@@std@@@?$vector@U?$pair@HULine@LocalizerResourceTxt@@@std@@V?$mempool_alloc@U?$pair@HULine@LocalizerResourceTxt@@@std@@@@@std@@IAEPAU?$pair@HULine@LocalizerResourceTxt@@@1@PAU21@00@Z 100054d7 f i LocalizerTxt.obj
 0001:000044f6       ??$_Umove@PAURange@LocalizerResourceTxt@@@?$vector@URange@LocalizerResourceTxt@@V?$mempool_alloc@URange@LocalizerResourceTxt@@@@@std@@IAEPAURange@LocalizerResourceTxt@@PAU23@00@Z 100054f6 f i LocalizerTxt.obj
 0001:00004515       ??$_Unchecked@PAU?$pair@HULine@LocalizerResourceTxt@@@std@@@std@@YGPAU?$pair@HULine@LocalizerResourceTxt@@@0@PAU10@@Z 10005515 f i LocalizerTxt.obj
 0001:0000451c       ??$_Unchecked@PAURange@LocalizerResourceTxt@@@std@@YGPAURange@LocalizerResourceTxt@@PAU12@@Z 1000551c f i LocalizerTxt.obj
 0001:00004523       ??$_Unchecked@PBU?$pair@HULine@LocalizerResourceTxt@@@std@@@std@@YGPBU?$pair@HULine@LocalizerResourceTxt@@@0@PBU10@@Z 10005523 f i LocalizerTxt.obj
 0001:0000452a       ??$_Unchecked@V?$_Vector_val@U?$_Simple_types@U?$pair@HULine@LocalizerResourceTxt@@@std@@@std@@@std@@@std@@YGPAU?$pair@HULine@LocalizerResourceTxt@@@0@V?$_Vector_iterator@V?$_Vector_val@U?$_Simple_types@U?$pair@HULine@LocalizerResourceTxt@@@std@@@std@@@std@@@0@@Z 1000552a f i LocalizerTxt.obj
 0001:00004531       ??$_Unchecked@V?$_Vector_val@U?$_Simple_types@U?$pair@HULine@LocalizerResourceTxt@@@std@@@std@@@std@@@std@@YGPBU?$pair@HULine@LocalizerResourceTxt@@@0@V?$_Vector_const_iterator@V?$_Vector_val@U?$_Simple_types@U?$pair@HULine@LocalizerResourceTxt@@@std@@@std@@@std@@@0@@Z 10005531 f i LocalizerTxt.obj
 0001:00004538       ??$_Unchecked@V?$_Vector_val@U?$_Simple_types@URange@LocalizerResourceTxt@@@std@@@std@@@std@@YGPAURange@LocalizerResourceTxt@@V?$_Vector_iterator@V?$_Vector_val@U?$_Simple_types@URange@LocalizerResourceTxt@@@std@@@std@@@0@@Z 10005538 f i LocalizerTxt.obj
 0001:0000453f       ??$_Unguarded_partition@PAURange@LocalizerResourceTxt@@VRangeArrayLess@?A0x10e53216@@@std@@YG?AU?$pair@PAURange@LocalizerResourceTxt@@PAU12@@0@PAURange@LocalizerResourceTxt@@0VRangeArrayLess@?A0x10e53216@@@Z 1000553f f i LocalizerTxt.obj
 0001:0000473d       ??$_Uninit_move@PAU?$pair@HULine@LocalizerResourceTxt@@@std@@PAU12@V?$mempool_alloc@U?$pair@HULine@LocalizerResourceTxt@@@std@@@@U12@@std@@YGPAU?$pair@HULine@LocalizerResourceTxt@@@0@PAU10@00AAU?$_Wrap_alloc@V?$mempool_alloc@U?$pair@HULine@LocalizerResourceTxt@@@std@@@@@0@0U_Nonscalar_ptr_iterator_tag@0@@Z 1000573d f i LocalizerTxt.obj
 0001:0000476a       ??$_Uninit_move@PAURange@LocalizerResourceTxt@@PAU12@V?$mempool_alloc@URange@LocalizerResourceTxt@@@@U12@@std@@YGPAURange@LocalizerResourceTxt@@PAU12@00AAU?$_Wrap_alloc@V?$mempool_alloc@URange@LocalizerResourceTxt@@@@@0@0U_Nonscalar_ptr_iterator_tag@0@@Z 1000576a f i LocalizerTxt.obj
 0001:00004796       ??$_Uninitialized_move@PAU?$pair@HULine@LocalizerResourceTxt@@@std@@PAU12@U?$_Wrap_alloc@V?$mempool_alloc@U?$pair@HULine@LocalizerResourceTxt@@@std@@@@@2@@std@@YGPAU?$pair@HULine@LocalizerResourceTxt@@@0@PAU10@00AAU?$_Wrap_alloc@V?$mempool_alloc@U?$pair@HULine@LocalizerResourceTxt@@@std@@@@@0@@Z 10005796 f i LocalizerTxt.obj
 0001:000047b3       ??$_Uninitialized_move@PAURange@LocalizerResourceTxt@@PAU12@U?$_Wrap_alloc@V?$mempool_alloc@URange@LocalizerResourceTxt@@@@@std@@@std@@YGPAURange@LocalizerResourceTxt@@PAU12@00AAU?$_Wrap_alloc@V?$mempool_alloc@URange@LocalizerResourceTxt@@@@@0@@Z 100057b3 f i LocalizerTxt.obj
 0001:000047d0       ??$_Upper_bound@PAU?$pair@HULine@LocalizerResourceTxt@@@std@@HHVLineArrayLess@?A0x10e53216@@@std@@YGPAU?$pair@HULine@LocalizerResourceTxt@@@0@PAU10@0ABHVLineArrayLess@?A0x10e53216@@PAH@Z 100057d0 f i LocalizerTxt.obj
 0001:00004817       ??$_Upper_bound@PBU?$pair@HULine@LocalizerResourceTxt@@@std@@HHVLineArrayLess@?A0x10e53216@@@std@@YGPBU?$pair@HULine@LocalizerResourceTxt@@@0@PBU10@0ABHVLineArrayLess@?A0x10e53216@@PAH@Z 10005817 f i LocalizerTxt.obj
 0001:0000485e       ??$_Val_type@PAU?$pair@HULine@LocalizerResourceTxt@@@std@@@std@@YGPAU?$pair@HULine@LocalizerResourceTxt@@@0@PAU10@@Z 1000585e f i LocalizerTxt.obj
 0001:00004863       ??$_Val_type@PAURange@LocalizerResourceTxt@@@std@@YGPAURange@LocalizerResourceTxt@@PAU12@@Z 10005863 f i LocalizerTxt.obj
 0001:00004868       ??$addressof@$$CBU?$pair@HULine@LocalizerResourceTxt@@@std@@@std@@YGPBU?$pair@HULine@LocalizerResourceTxt@@@0@ABU10@@Z 10005868 f i LocalizerTxt.obj
 0001:0000486f       ??$addressof@$$CBURange@LocalizerResourceTxt@@@std@@YGPBURange@LocalizerResourceTxt@@ABU12@@Z 1000586f f i LocalizerTxt.obj
 0001:00004876       ??$addressof@U?$pair@HULine@LocalizerResourceTxt@@@std@@@std@@YGPAU?$pair@HULine@LocalizerResourceTxt@@@0@AAU10@@Z 10005876 f i LocalizerTxt.obj
 0001:0000487d       ??$addressof@URange@LocalizerResourceTxt@@@std@@YGPAURange@LocalizerResourceTxt@@AAU12@@Z 1000587d f i LocalizerTxt.obj
 0001:00004884       ??$advance@PAU?$pair@HULine@LocalizerResourceTxt@@@std@@H@std@@YGXAAPAU?$pair@HULine@LocalizerResourceTxt@@@0@H@Z 10005884 f i LocalizerTxt.obj
 0001:00004894       ??$advance@PBU?$pair@HULine@LocalizerResourceTxt@@@std@@H@std@@YGXAAPBU?$pair@HULine@LocalizerResourceTxt@@@0@H@Z 10005894 f i LocalizerTxt.obj
 0001:000048a4       ??$advance@V?$_Vector_iterator@V?$_Vector_val@U?$_Simple_types@U?$pair@HULine@LocalizerResourceTxt@@@std@@@std@@@std@@@std@@H@std@@YGXAAV?$_Vector_iterator@V?$_Vector_val@U?$_Simple_types@U?$pair@HULine@LocalizerResourceTxt@@@std@@@std@@@std@@@0@H@Z 100058a4 f i LocalizerTxt.obj
 0001:000048b4       ??$construct@U?$pair@HULine@LocalizerResourceTxt@@@std@@U12@@?$_Wrap_alloc@V?$mempool_alloc@U?$pair@HULine@LocalizerResourceTxt@@@std@@@@@std@@QAEXPAU?$pair@HULine@LocalizerResourceTxt@@@1@$$QAU21@@Z 100058b4 f i LocalizerTxt.obj
 0001:000048cb       ??$construct@U?$pair@HULine@LocalizerResourceTxt@@@std@@U12@@?$allocator_traits@V?$mempool_alloc@U?$pair@HULine@LocalizerResourceTxt@@@std@@@@@std@@SGXAAV?$mempool_alloc@U?$pair@HULine@LocalizerResourceTxt@@@std@@@@PAU?$pair@HULine@LocalizerResourceTxt@@@1@$$QAU31@@Z 100058cb f i LocalizerTxt.obj
 0001:000048e2       ??$construct@URange@LocalizerResourceTxt@@AAU12@@?$_Wrap_alloc@V?$mempool_alloc@URange@LocalizerResourceTxt@@@@@std@@QAEXPAURange@LocalizerResourceTxt@@AAU23@@Z 100058e2 f i LocalizerTxt.obj
 0001:000048f8       ??$construct@URange@LocalizerResourceTxt@@AAU12@@?$allocator_traits@V?$mempool_alloc@URange@LocalizerResourceTxt@@@@@std@@SGXAAV?$mempool_alloc@URange@LocalizerResourceTxt@@@@PAURange@LocalizerResourceTxt@@AAU34@@Z 100058f8 f i LocalizerTxt.obj
 0001:0000490e       ??$construct@URange@LocalizerResourceTxt@@ABU12@@?$_Wrap_alloc@V?$mempool_alloc@URange@LocalizerResourceTxt@@@@@std@@QAEXPAURange@LocalizerResourceTxt@@ABU23@@Z 1000590e f i LocalizerTxt.obj
 0001:00004924       ??$construct@URange@LocalizerResourceTxt@@ABU12@@?$allocator_traits@V?$mempool_alloc@URange@LocalizerResourceTxt@@@@@std@@SGXAAV?$mempool_alloc@URange@LocalizerResourceTxt@@@@PAURange@LocalizerResourceTxt@@ABU34@@Z 10005924 f i LocalizerTxt.obj
 0001:0000493a       ??$construct@URange@LocalizerResourceTxt@@U12@@?$_Wrap_alloc@V?$mempool_alloc@URange@LocalizerResourceTxt@@@@@std@@QAEXPAURange@LocalizerResourceTxt@@$$QAU23@@Z 1000593a f i LocalizerTxt.obj
 0001:00004950       ??$construct@URange@LocalizerResourceTxt@@U12@@?$allocator_traits@V?$mempool_alloc@URange@LocalizerResourceTxt@@@@@std@@SGXAAV?$mempool_alloc@URange@LocalizerResourceTxt@@@@PAURange@LocalizerResourceTxt@@$$QAU34@@Z 10005950 f i LocalizerTxt.obj
 0001:00004966       ??$destroy@U?$pair@HULine@LocalizerResourceTxt@@@std@@@?$_Wrap_alloc@V?$mempool_alloc@U?$pair@HULine@LocalizerResourceTxt@@@std@@@@@std@@QAEXPAU?$pair@HULine@LocalizerResourceTxt@@@1@@Z 10005966 f i LocalizerTxt.obj
 0001:00004969       ??$destroy@U?$pair@HULine@LocalizerResourceTxt@@@std@@@?$allocator_traits@V?$mempool_alloc@U?$pair@HULine@LocalizerResourceTxt@@@std@@@@@std@@SGXAAV?$mempool_alloc@U?$pair@HULine@LocalizerResourceTxt@@@std@@@@PAU?$pair@HULine@LocalizerResourceTxt@@@1@@Z 10005969 f i LocalizerTxt.obj
 0001:0000496c       ??$destroy@URange@LocalizerResourceTxt@@@?$_Wrap_alloc@V?$mempool_alloc@URange@LocalizerResourceTxt@@@@@std@@QAEXPAURange@LocalizerResourceTxt@@@Z 1000596c f i LocalizerTxt.obj
 0001:0000496f       ??$destroy@URange@LocalizerResourceTxt@@@?$allocator_traits@V?$mempool_alloc@URange@LocalizerResourceTxt@@@@@std@@SGXAAV?$mempool_alloc@URange@LocalizerResourceTxt@@@@PAURange@LocalizerResourceTxt@@@Z 1000596f f i LocalizerTxt.obj
 0001:00004972       ??$distance@V?$_Vector_iterator@V?$_Vector_val@U?$_Simple_types@U?$pair@HULine@LocalizerResourceTxt@@@std@@@std@@@std@@@std@@@std@@YGHV?$_Vector_iterator@V?$_Vector_val@U?$_Simple_types@U?$pair@HULine@LocalizerResourceTxt@@@std@@@std@@@std@@@0@0@Z 10005972 f i LocalizerTxt.obj
 0001:00004980       ??$emplace@U?$pair@HULine@LocalizerResourceTxt@@@std@@@?$vector@U?$pair@HULine@LocalizerResourceTxt@@@std@@V?$mempool_alloc@U?$pair@HULine@LocalizerResourceTxt@@@std@@@@@std@@QAE?AV?$_Vector_iterator@V?$_Vector_val@U?$_Simple_types@U?$pair@HULine@LocalizerResourceTxt@@@std@@@std@@@std@@@1@V?$_Vector_const_iterator@V?$_Vector_val@U?$_Simple_types@U?$pair@HULine@LocalizerResourceTxt@@@std@@@std@@@std@@@1@$$QAU?$pair@HULine@LocalizerResourceTxt@@@1@@Z 10005980 f i LocalizerTxt.obj
 0001:000049bc       ??$emplace_back@U?$pair@HULine@LocalizerResourceTxt@@@std@@@?$vector@U?$pair@HULine@LocalizerResourceTxt@@@std@@V?$mempool_alloc@U?$pair@HULine@LocalizerResourceTxt@@@std@@@@@std@@QAEX$$QAU?$pair@HULine@LocalizerResourceTxt@@@1@@Z 100059bc f i LocalizerTxt.obj
 0001:000049e9       ??$equal_range@V?$_Vector_const_iterator@V?$_Vector_val@U?$_Simple_types@U?$pair@HULine@LocalizerResourceTxt@@@std@@@std@@@std@@@std@@HVLineArrayLess@?A0x10e53216@@@std@@YG?AU?$pair@V?$_Vector_const_iterator@V?$_Vector_val@U?$_Simple_types@U?$pair@HULine@LocalizerResourceTxt@@@std@@@std@@@std@@@std@@V12@@0@V?$_Vector_const_iterator@V?$_Vector_val@U?$_Simple_types@U?$pair@HULine@LocalizerResourceTxt@@@std@@@std@@@std@@@0@0ABHVLineArrayLess@?A0x10e53216@@@Z 100059e9 f i LocalizerTxt.obj
 0001:00004a16       ??$equal_range@V?$_Vector_iterator@V?$_Vector_val@U?$_Simple_types@U?$pair@HULine@LocalizerResourceTxt@@@std@@@std@@@std@@@std@@HVLineArrayLess@?A0x10e53216@@@std@@YG?AU?$pair@V?$_Vector_iterator@V?$_Vector_val@U?$_Simple_types@U?$pair@HULine@LocalizerResourceTxt@@@std@@@std@@@std@@@std@@V12@@0@V?$_Vector_iterator@V?$_Vector_val@U?$_Simple_types@U?$pair@HULine@LocalizerResourceTxt@@@std@@@std@@@std@@@0@0ABHVLineArrayLess@?A0x10e53216@@@Z 10005a16 f i LocalizerTxt.obj
 0001:00004a43       ??$for_each@V?$_Vector_iterator@V?$_Vector_val@U?$_Simple_types@U?$pair@HULine@LocalizerResourceTxt@@@std@@@std@@@std@@@std@@P6GXAAU?$pair@HULine@LocalizerResourceTxt@@@2@@Z@std@@YGP6GXAAU?$pair@HULine@LocalizerResourceTxt@@@0@@ZV?$_Vector_iterator@V?$_Vector_val@U?$_Simple_types@U?$pair@HULine@LocalizerResourceTxt@@@std@@@std@@@std@@@0@1P6GX0@Z@Z 10005a43 f i LocalizerTxt.obj
 0001:00004a5c       ??$for_each@V?$_Vector_iterator@V?$_Vector_val@U?$_Simple_types@URange@LocalizerResourceTxt@@@std@@@std@@@std@@P6GXAAURange@LocalizerResourceTxt@@@Z@std@@YGP6GXAAURange@LocalizerResourceTxt@@@ZV?$_Vector_iterator@V?$_Vector_val@U?$_Simple_types@URange@LocalizerResourceTxt@@@std@@@std@@@0@1P6GX0@Z@Z 10005a5c f i LocalizerTxt.obj
 0001:00004a75       ??$forward@AAH@std@@YGAAHAAH@Z 10005a75 f i LocalizerTxt.obj
 0001:00004a7c       ??$forward@AAPAU?$pair@HULine@LocalizerResourceTxt@@@std@@@std@@YGAAPAU?$pair@HULine@LocalizerResourceTxt@@@0@AAPAU10@@Z 10005a7c f i LocalizerTxt.obj
 0001:00004a83       ??$forward@AAPAURange@LocalizerResourceTxt@@@std@@YGAAPAURange@LocalizerResourceTxt@@AAPAU12@@Z 10005a83 f i LocalizerTxt.obj
 0001:00004a8a       ??$forward@AAPBU?$pair@HULine@LocalizerResourceTxt@@@std@@@std@@YGAAPBU?$pair@HULine@LocalizerResourceTxt@@@0@AAPBU10@@Z 10005a8a f i LocalizerTxt.obj
 0001:00004a91       ??$forward@AAULine@LocalizerResourceTxt@@@std@@YGAAULine@LocalizerResourceTxt@@AAU12@@Z 10005a91 f i LocalizerTxt.obj
 0001:00004a98       ??$forward@AAURange@LocalizerResourceTxt@@@std@@YGAAURange@LocalizerResourceTxt@@AAU12@@Z 10005a98 f i LocalizerTxt.obj
 0001:00004a9f       ??$forward@AAV?$_Vector_const_iterator@V?$_Vector_val@U?$_Simple_types@U?$pair@HULine@LocalizerResourceTxt@@@std@@@std@@@std@@@std@@@std@@YGAAV?$_Vector_const_iterator@V?$_Vector_val@U?$_Simple_types@U?$pair@HULine@LocalizerResourceTxt@@@std@@@std@@@std@@@0@AAV10@@Z 10005a9f f i LocalizerTxt.obj
 0001:00004aa6       ??$forward@AAV?$_Vector_iterator@V?$_Vector_val@U?$_Simple_types@U?$pair@HULine@LocalizerResourceTxt@@@std@@@std@@@std@@@std@@@std@@YGAAV?$_Vector_iterator@V?$_Vector_val@U?$_Simple_types@U?$pair@HULine@LocalizerResourceTxt@@@std@@@std@@@std@@@0@AAV10@@Z 10005aa6 f i LocalizerTxt.obj
 0001:00004aad       ??$forward@ABURange@LocalizerResourceTxt@@@std@@YGABURange@LocalizerResourceTxt@@ABU12@@Z 10005aad f i LocalizerTxt.obj
 0001:00004ab4       ??$forward@H@std@@YG$$QAHAAH@Z 10005ab4 f i LocalizerTxt.obj
 0001:00004abb       ??$forward@PAU?$pair@HULine@LocalizerResourceTxt@@@std@@@std@@YG$$QAPAU?$pair@HULine@LocalizerResourceTxt@@@0@AAPAU10@@Z 10005abb f i LocalizerTxt.obj
 0001:00004ac2       ??$forward@PAURange@LocalizerResourceTxt@@@std@@YG$$QAPAURange@LocalizerResourceTxt@@AAPAU12@@Z 10005ac2 f i LocalizerTxt.obj
 0001:00004ac9       ??$forward@PBU?$pair@HULine@LocalizerResourceTxt@@@std@@@std@@YG$$QAPBU?$pair@HULine@LocalizerResourceTxt@@@0@AAPBU10@@Z 10005ac9 f i LocalizerTxt.obj
 0001:00004ad0       ??$forward@U?$pair@HULine@LocalizerResourceTxt@@@std@@@std@@YG$$QAU?$pair@HULine@LocalizerResourceTxt@@@0@AAU10@@Z 10005ad0 f i LocalizerTxt.obj
 0001:00004ad7       ??$forward@ULine@LocalizerResourceTxt@@@std@@YG$$QAULine@LocalizerResourceTxt@@AAU12@@Z 10005ad7 f i LocalizerTxt.obj
 0001:00004ade       ??$forward@URange@LocalizerResourceTxt@@@std@@YG$$QAURange@LocalizerResourceTxt@@AAU12@@Z 10005ade f i LocalizerTxt.obj
 0001:00004ae5       ??$forward@V?$_Vector_const_iterator@V?$_Vector_val@U?$_Simple_types@U?$pair@HULine@LocalizerResourceTxt@@@std@@@std@@@std@@@std@@@std@@YG$$QAV?$_Vector_const_iterator@V?$_Vector_val@U?$_Simple_types@U?$pair@HULine@LocalizerResourceTxt@@@std@@@std@@@std@@@0@AAV10@@Z 10005ae5 f i LocalizerTxt.obj
 0001:00004aec       ??$forward@V?$_Vector_iterator@V?$_Vector_val@U?$_Simple_types@U?$pair@HULine@LocalizerResourceTxt@@@std@@@std@@@std@@@std@@@std@@YG$$QAV?$_Vector_iterator@V?$_Vector_val@U?$_Simple_types@U?$pair@HULine@LocalizerResourceTxt@@@std@@@std@@@std@@@0@AAV10@@Z 10005aec f i LocalizerTxt.obj
 0001:00004af3       ??$iter_swap@PAU?$pair@HULine@LocalizerResourceTxt@@@std@@PAU12@@std@@YGXPAU?$pair@HULine@LocalizerResourceTxt@@@0@0@Z 10005af3 f i LocalizerTxt.obj
 0001:00004b03       ??$iter_swap@PAURange@LocalizerResourceTxt@@PAU12@@std@@YGXPAURange@LocalizerResourceTxt@@0@Z 10005b03 f i LocalizerTxt.obj
 0001:00004b2c       ??$lower_bound@PAU?$pair@HULine@LocalizerResourceTxt@@@std@@HVLineArrayLess@?A0x10e53216@@@std@@YGPAU?$pair@HULine@LocalizerResourceTxt@@@0@PAU10@0ABHVLineArrayLess@?A0x10e53216@@@Z 10005b2c f i LocalizerTxt.obj
 0001:00004b46       ??$lower_bound@PBU?$pair@HULine@LocalizerResourceTxt@@@std@@HVLineArrayLess@?A0x10e53216@@@std@@YGPBU?$pair@HULine@LocalizerResourceTxt@@@0@PBU10@0ABHVLineArrayLess@?A0x10e53216@@@Z 10005b46 f i LocalizerTxt.obj
 0001:00004b60       ??$make_heap@PAURange@LocalizerResourceTxt@@VRangeArrayLess@?A0x10e53216@@@std@@YGXPAURange@LocalizerResourceTxt@@0VRangeArrayLess@?A0x10e53216@@@Z 10005b60 f i LocalizerTxt.obj
 0001:00004b8a       ??$move@AAP6GXAAU?$pair@HULine@LocalizerResourceTxt@@@std@@@Z@std@@YG$$QAP6GXAAU?$pair@HULine@LocalizerResourceTxt@@@0@@ZAAP6GX0@Z@Z 10005b8a f i LocalizerTxt.obj
 0001:00004b91       ??$move@AAP6GXAAURange@LocalizerResourceTxt@@@Z@std@@YG$$QAP6GXAAURange@LocalizerResourceTxt@@@ZAAP6GX0@Z@Z 10005b91 f i LocalizerTxt.obj
 0001:00004b98       ??$move@AAU?$pair@HULine@LocalizerResourceTxt@@@std@@@std@@YG$$QAU?$pair@HULine@LocalizerResourceTxt@@@0@AAU10@@Z 10005b98 f i LocalizerTxt.obj
 0001:00004b9f       ??$move@AAURange@LocalizerResourceTxt@@@std@@YG$$QAURange@LocalizerResourceTxt@@AAU12@@Z 10005b9f f i LocalizerTxt.obj
 0001:00004ba6       ??$rotate@V?$_Vector_iterator@V?$_Vector_val@U?$_Simple_types@U?$pair@HULine@LocalizerResourceTxt@@@std@@@std@@@std@@@std@@@std@@YG?AV?$_Vector_iterator@V?$_Vector_val@U?$_Simple_types@U?$pair@HULine@LocalizerResourceTxt@@@std@@@std@@@std@@@0@V10@00@Z 10005ba6 f i LocalizerTxt.obj
 0001:00004be1       ??$sort@V?$_Vector_iterator@V?$_Vector_val@U?$_Simple_types@URange@LocalizerResourceTxt@@@std@@@std@@@std@@VRangeArrayLess@?A0x10e53216@@@std@@YGXV?$_Vector_iterator@V?$_Vector_val@U?$_Simple_types@URange@LocalizerResourceTxt@@@std@@@std@@@0@0VRangeArrayLess@?A0x10e53216@@@Z 10005be1 f i LocalizerTxt.obj
 0001:00004c03       ??$sort_heap@PAURange@LocalizerResourceTxt@@VRangeArrayLess@?A0x10e53216@@@std@@YGXPAURange@LocalizerResourceTxt@@0VRangeArrayLess@?A0x10e53216@@@Z 10005c03 f i LocalizerTxt.obj
 0001:00004c17       ??$swap@H@std@@YGXAAH0@Z   10005c17 f i LocalizerTxt.obj
 0001:00004c2c       ??$swap@HULine@LocalizerResourceTxt@@@std@@YGXAAU?$pair@HULine@LocalizerResourceTxt@@@0@0@Z 10005c2c f i LocalizerTxt.obj
 0001:00004c3c       ??$swap@ULine@LocalizerResourceTxt@@@std@@YGXAAULine@LocalizerResourceTxt@@0@Z 10005c3c f i LocalizerTxt.obj
 0001:00004c65       ??$swap@URange@LocalizerResourceTxt@@@std@@YGXAAURange@LocalizerResourceTxt@@0@Z 10005c65 f i LocalizerTxt.obj
 0001:00004c8e       ??$upper_bound@PAU?$pair@HULine@LocalizerResourceTxt@@@std@@HVLineArrayLess@?A0x10e53216@@@std@@YGPAU?$pair@HULine@LocalizerResourceTxt@@@0@PAU10@0ABHVLineArrayLess@?A0x10e53216@@@Z 10005c8e f i LocalizerTxt.obj
 0001:00004ca8       ??$upper_bound@PBU?$pair@HULine@LocalizerResourceTxt@@@std@@HVLineArrayLess@?A0x10e53216@@@std@@YGPBU?$pair@HULine@LocalizerResourceTxt@@@0@PBU10@0ABHVLineArrayLess@?A0x10e53216@@@Z 10005ca8 f i LocalizerTxt.obj
 0001:00004cc2       ??0?$_Vector_alloc@$00U?$_Vec_base_types@U?$pair@HULine@LocalizerResourceTxt@@@std@@V?$mempool_alloc@U?$pair@HULine@LocalizerResourceTxt@@@std@@@@@std@@@std@@QAE@ABV?$mempool_alloc@U?$pair@HULine@LocalizerResourceTxt@@@std@@@@@Z 10005cc2 f i LocalizerTxt.obj
 0001:00004cda       ??0?$_Vector_alloc@$00U?$_Vec_base_types@URange@LocalizerResourceTxt@@V?$mempool_alloc@URange@LocalizerResourceTxt@@@@@std@@@std@@QAE@ABV?$mempool_alloc@URange@LocalizerResourceTxt@@@@@Z 10005cda f i LocalizerTxt.obj
 0001:00004cf2       ??0?$_Vector_const_iterator@V?$_Vector_val@U?$_Simple_types@U?$pair@HULine@LocalizerResourceTxt@@@std@@@std@@@std@@@std@@QAE@PAU?$pair@HULine@LocalizerResourceTxt@@@1@PBU_Container_base0@1@@Z 10005cf2 f i LocalizerTxt.obj
 0001:00004cfd       ??0?$_Vector_const_iterator@V?$_Vector_val@U?$_Simple_types@URange@LocalizerResourceTxt@@@std@@@std@@@std@@QAE@PAURange@LocalizerResourceTxt@@PBU_Container_base0@1@@Z 10005cfd f i LocalizerTxt.obj
 0001:00004d08       ??0?$_Vector_iterator@V?$_Vector_val@U?$_Simple_types@U?$pair@HULine@LocalizerResourceTxt@@@std@@@std@@@std@@@std@@QAE@PAU?$pair@HULine@LocalizerResourceTxt@@@1@PBU_Container_base0@1@@Z 10005d08 f i LocalizerTxt.obj
 0001:00004d13       ??0?$_Vector_iterator@V?$_Vector_val@U?$_Simple_types@URange@LocalizerResourceTxt@@@std@@@std@@@std@@QAE@PAURange@LocalizerResourceTxt@@PBU_Container_base0@1@@Z 10005d13 f i LocalizerTxt.obj
 0001:00004d1e       ??0?$_Vector_val@U?$_Simple_types@U?$pair@HULine@LocalizerResourceTxt@@@std@@@std@@@std@@QAE@XZ 10005d1e f i LocalizerTxt.obj
 0001:00004d2b       ??0?$_Vector_val@U?$_Simple_types@URange@LocalizerResourceTxt@@@std@@@std@@QAE@XZ 10005d2b f i LocalizerTxt.obj
 0001:00004d38       ??0?$_Wrap_alloc@V?$mempool_alloc@U?$pair@HULine@LocalizerResourceTxt@@@std@@@@@std@@QAE@ABV?$mempool_alloc@U?$pair@HULine@LocalizerResourceTxt@@@std@@@@@Z 10005d38 f i LocalizerTxt.obj
 0001:00004d45       ??0?$_Wrap_alloc@V?$mempool_alloc@URange@LocalizerResourceTxt@@@@@std@@QAE@ABV?$mempool_alloc@URange@LocalizerResourceTxt@@@@@Z 10005d45 f i LocalizerTxt.obj
 0001:00004d52       ??0?$auto_ptr@VLocalizerResourceTxt@@@std@@QAE@PAVLocalizerResourceTxt@@@Z 10005d52 f i LocalizerTxt.obj
 0001:00004d5d       ??0?$mempool_alloc@U?$pair@HULine@LocalizerResourceTxt@@@std@@@@QAE@PAU_HMEMPOOL@@@Z 10005d5d f i LocalizerTxt.obj
 0001:00004d68       ??0?$mempool_alloc@URange@LocalizerResourceTxt@@@@QAE@PAU_HMEMPOOL@@@Z 10005d68 f i LocalizerTxt.obj
 0001:00004d73       ??0?$vector@U?$pair@HULine@LocalizerResourceTxt@@@std@@V?$mempool_alloc@U?$pair@HULine@LocalizerResourceTxt@@@std@@@@@std@@QAE@ABV?$mempool_alloc@U?$pair@HULine@LocalizerResourceTxt@@@std@@@@@Z 10005d73 f i LocalizerTxt.obj
 0001:00004d8b       ??0?$vector@URange@LocalizerResourceTxt@@V?$mempool_alloc@URange@LocalizerResourceTxt@@@@@std@@QAE@ABV?$mempool_alloc@URange@LocalizerResourceTxt@@@@@Z 10005d8b f i LocalizerTxt.obj
 0001:00004da3       ??0LocalizerResourceTxt@@AAE@PBD@Z 10005da3 f   LocalizerTxt.obj
 0001:00004e10       ??0ParseOut@?A0x10e53216@@QAE@XZ 10005e10 f i LocalizerTxt.obj
 0001:00004e2a       ??0_Wrap_int@std@@QAE@H@Z  10005e2a f i LocalizerTxt.obj
 0001:00004e2f       ??1?$_Vector_alloc@$00U?$_Vec_base_types@U?$pair@HULine@LocalizerResourceTxt@@@std@@V?$mempool_alloc@U?$pair@HULine@LocalizerResourceTxt@@@std@@@@@std@@@std@@QAE@XZ 10005e2f f i LocalizerTxt.obj
 0001:00004e30       ??1?$_Vector_alloc@$00U?$_Vec_base_types@URange@LocalizerResourceTxt@@V?$mempool_alloc@URange@LocalizerResourceTxt@@@@@std@@@std@@QAE@XZ 10005e30 f i LocalizerTxt.obj
 0001:00004e31       ??1?$_Wrap_alloc@V?$mempool_alloc@U?$pair@HULine@LocalizerResourceTxt@@@std@@@@@std@@QAE@XZ 10005e31 f i LocalizerTxt.obj
 0001:00004e32       ??1?$_Wrap_alloc@V?$mempool_alloc@URange@LocalizerResourceTxt@@@@@std@@QAE@XZ 10005e32 f i LocalizerTxt.obj
 0001:00004e33       ??1?$auto_ptr@VLocalizerResourceTxt@@@std@@QAE@XZ 10005e33 f i LocalizerTxt.obj
 0001:00004e40       ??1?$mempool_alloc@U?$pair@HULine@LocalizerResourceTxt@@@std@@@@QAE@XZ 10005e40 f i LocalizerTxt.obj
 0001:00004e41       ??1?$mempool_alloc@URange@LocalizerResourceTxt@@@@QAE@XZ 10005e41 f i LocalizerTxt.obj
 0001:00004e42       ??1?$vector@U?$pair@HULine@LocalizerResourceTxt@@@std@@V?$mempool_alloc@U?$pair@HULine@LocalizerResourceTxt@@@std@@@@@std@@QAE@XZ 10005e42 f i LocalizerTxt.obj
 0001:00004e47       ??1?$vector@URange@LocalizerResourceTxt@@V?$mempool_alloc@URange@LocalizerResourceTxt@@@@@std@@QAE@XZ 10005e47 f i LocalizerTxt.obj
 0001:00004e4c       ??1LocalizerResourceTxt@@UAE@XZ 10005e4c f   LocalizerTxt.obj
 0001:00004ef8       ??1ParseOut@?A0x10e53216@@QAE@XZ 10005ef8 f i LocalizerTxt.obj
 0001:00004f0c       ??4?$basic_string@DU?$char_traits@D@std@@V?$allocator@D@2@@std@@QAEAAV01@PBD@Z 10005f0c f i LocalizerTxt.obj
 0001:00004f29       ??4?$pair@HULine@LocalizerResourceTxt@@@std@@QAEAAU01@$$QAU01@@Z 10005f29 f i LocalizerTxt.obj
 0001:00004f43       ??8?$_Vector_const_iterator@V?$_Vector_val@U?$_Simple_types@U?$pair@HULine@LocalizerResourceTxt@@@std@@@std@@@std@@@std@@QBE_NABV01@@Z 10005f43 f i LocalizerTxt.obj
 0001:00004f53       ??8?$_Vector_const_iterator@V?$_Vector_val@U?$_Simple_types@URange@LocalizerResourceTxt@@@std@@@std@@@std@@QBE_NABV01@@Z 10005f53 f i LocalizerTxt.obj
 0001:00004f63       ??9?$_Vector_const_iterator@V?$_Vector_val@U?$_Simple_types@U?$pair@HULine@LocalizerResourceTxt@@@std@@@std@@@std@@@std@@QBE_NABV01@@Z 10005f63 f i LocalizerTxt.obj
 0001:00004f73       ??9?$_Vector_const_iterator@V?$_Vector_val@U?$_Simple_types@URange@LocalizerResourceTxt@@@std@@@std@@@std@@QBE_NABV01@@Z 10005f73 f i LocalizerTxt.obj
 0001:00004f83       ??C?$_Vector_const_iterator@V?$_Vector_val@U?$_Simple_types@U?$pair@HULine@LocalizerResourceTxt@@@std@@@std@@@std@@@std@@QBEPBU?$pair@HULine@LocalizerResourceTxt@@@1@XZ 10005f83 f i LocalizerTxt.obj
 0001:00004f86       ??C?$_Vector_const_iterator@V?$_Vector_val@U?$_Simple_types@URange@LocalizerResourceTxt@@@std@@@std@@@std@@QBEPBURange@LocalizerResourceTxt@@XZ 10005f86 f i LocalizerTxt.obj
 0001:00004f89       ??C?$_Vector_iterator@V?$_Vector_val@U?$_Simple_types@U?$pair@HULine@LocalizerResourceTxt@@@std@@@std@@@std@@@std@@QBEPAU?$pair@HULine@LocalizerResourceTxt@@@1@XZ 10005f89 f i LocalizerTxt.obj
 0001:00004f8c       ??C?$_Vector_iterator@V?$_Vector_val@U?$_Simple_types@URange@LocalizerResourceTxt@@@std@@@std@@@std@@QBEPAURange@LocalizerResourceTxt@@XZ 10005f8c f i LocalizerTxt.obj
 0001:00004f8f       ??C?$auto_ptr@VLocalizerResourceTxt@@@std@@QBEPAVLocalizerResourceTxt@@XZ 10005f8f f i LocalizerTxt.obj
 0001:00004f92       ??D?$_Vector_const_iterator@V?$_Vector_val@U?$_Simple_types@U?$pair@HULine@LocalizerResourceTxt@@@std@@@std@@@std@@@std@@QBEABU?$pair@HULine@LocalizerResourceTxt@@@1@XZ 10005f92 f i LocalizerTxt.obj
 0001:00004f95       ??D?$_Vector_const_iterator@V?$_Vector_val@U?$_Simple_types@URange@LocalizerResourceTxt@@@std@@@std@@@std@@QBEABURange@LocalizerResourceTxt@@XZ 10005f95 f i LocalizerTxt.obj
 0001:00004f98       ??D?$_Vector_iterator@V?$_Vector_val@U?$_Simple_types@U?$pair@HULine@LocalizerResourceTxt@@@std@@@std@@@std@@@std@@QBEAAU?$pair@HULine@LocalizerResourceTxt@@@1@XZ 10005f98 f i LocalizerTxt.obj
 0001:00004f9b       ??D?$_Vector_iterator@V?$_Vector_val@U?$_Simple_types@URange@LocalizerResourceTxt@@@std@@@std@@@std@@QBEAAURange@LocalizerResourceTxt@@XZ 10005f9b f i LocalizerTxt.obj
 0001:00004f9e       ??E?$_Vector_const_iterator@V?$_Vector_val@U?$_Simple_types@URange@LocalizerResourceTxt@@@std@@@std@@@std@@QAEAAV01@XZ 10005f9e f i LocalizerTxt.obj
 0001:00004fa4       ??E?$_Vector_iterator@V?$_Vector_val@U?$_Simple_types@URange@LocalizerResourceTxt@@@std@@@std@@@std@@QAEAAV01@XZ 10005fa4 f i LocalizerTxt.obj
 0001:00004faa       ??G?$_Vector_const_iterator@V?$_Vector_val@U?$_Simple_types@U?$pair@HULine@LocalizerResourceTxt@@@std@@@std@@@std@@@std@@QBEHABV01@@Z 10005faa f i LocalizerTxt.obj
 0001:00004fb8       ??G?$_Vector_const_iterator@V?$_Vector_val@U?$_Simple_types@URange@LocalizerResourceTxt@@@std@@@std@@@std@@QBEHABV01@@Z 10005fb8 f i LocalizerTxt.obj
 0001:00004fc9       ??G?$_Vector_iterator@V?$_Vector_val@U?$_Simple_types@U?$pair@HULine@LocalizerResourceTxt@@@std@@@std@@@std@@@std@@QBE?AV01@H@Z 10005fc9 f i LocalizerTxt.obj
 0001:00004fdd       ??G?$_Vector_iterator@V?$_Vector_val@U?$_Simple_types@U?$pair@HULine@LocalizerResourceTxt@@@std@@@std@@@std@@@std@@QBEHABV?$_Vector_const_iterator@V?$_Vector_val@U?$_Simple_types@U?$pair@HULine@LocalizerResourceTxt@@@std@@@std@@@std@@@1@@Z 10005fdd f i LocalizerTxt.obj
 0001:00004feb       ??G?$_Vector_iterator@V?$_Vector_val@U?$_Simple_types@URange@LocalizerResourceTxt@@@std@@@std@@@std@@QBE?AV01@H@Z 10005feb f i LocalizerTxt.obj
 0001:00004fff       ??G?$_Vector_iterator@V?$_Vector_val@U?$_Simple_types@URange@LocalizerResourceTxt@@@std@@@std@@@std@@QBEHABV?$_Vector_const_iterator@V?$_Vector_val@U?$_Simple_types@URange@LocalizerResourceTxt@@@std@@@std@@@1@@Z 10005fff f i LocalizerTxt.obj
 0001:00005010       ??H?$_Vector_iterator@V?$_Vector_val@U?$_Simple_types@U?$pair@HULine@LocalizerResourceTxt@@@std@@@std@@@std@@@std@@QBE?AV01@H@Z 10006010 f i LocalizerTxt.obj
 0001:00005022       ??RLineArrayLess@?A0x10e53216@@QBE_NABU?$pair@HULine@LocalizerResourceTxt@@@std@@H@Z 10006022 f i LocalizerTxt.obj
 0001:00005034       ??RLineArrayLess@?A0x10e53216@@QBE_NHABU?$pair@HULine@LocalizerResourceTxt@@@std@@@Z 10006034 f i LocalizerTxt.obj
 0001:00005046       ??RRangeArrayLess@?A0x10e53216@@QBE_NABURange@LocalizerResourceTxt@@0@Z 10006046 f i LocalizerTxt.obj
 0001:0000505b       ??Y?$_Vector_const_iterator@V?$_Vector_val@U?$_Simple_types@U?$pair@HULine@LocalizerResourceTxt@@@std@@@std@@@std@@@std@@QAEAAV01@H@Z 1000605b f i LocalizerTxt.obj
 0001:00005069       ??Y?$_Vector_const_iterator@V?$_Vector_val@U?$_Simple_types@URange@LocalizerResourceTxt@@@std@@@std@@@std@@QAEAAV01@H@Z 10006069 f i LocalizerTxt.obj
 0001:00005077       ??Y?$_Vector_iterator@V?$_Vector_val@U?$_Simple_types@U?$pair@HULine@LocalizerResourceTxt@@@std@@@std@@@std@@@std@@QAEAAV01@H@Z 10006077 f i LocalizerTxt.obj
 0001:00005085       ??Y?$_Vector_iterator@V?$_Vector_val@U?$_Simple_types@URange@LocalizerResourceTxt@@@std@@@std@@@std@@QAEAAV01@H@Z 10006085 f i LocalizerTxt.obj
 0001:00005093       ??Y?$basic_string@DU?$char_traits@D@std@@V?$allocator@D@2@@std@@QAEAAV01@ABV01@@Z 10006093 f i LocalizerTxt.obj
 0001:000050a3       ??Z?$_Vector_iterator@V?$_Vector_val@U?$_Simple_types@U?$pair@HULine@LocalizerResourceTxt@@@std@@@std@@@std@@@std@@QAEAAV01@H@Z 100060a3 f i LocalizerTxt.obj
 0001:000050b1       ??Z?$_Vector_iterator@V?$_Vector_val@U?$_Simple_types@URange@LocalizerResourceTxt@@@std@@@std@@@std@@QAEAAV01@H@Z 100060b1 f i LocalizerTxt.obj
 0001:000050bf       ??_GLocalizerResourceTxt@@UAEPAXI@Z 100060bf f i LocalizerTxt.obj
 0001:000050bf       ??_ELocalizerResourceTxt@@UAEPAXI@Z 100060bf f i LocalizerTxt.obj
 0001:000050db       ?AddRange@LocalizerResourceTxt@@QAE_NAAH0IPBD@Z 100060db f   LocalizerTxt.obj
 0001:000051aa       ?AddText@LocalizerResourceTxt@@QAEHPB_WHHH@Z 100061aa f   LocalizerTxt.obj
 0001:000052d1       ?Begin@LocalizerResourceTxt@@QBE?AV?$_Vector_const_iterator@V?$_Vector_val@U?$_Simple_types@U?$pair@HULine@LocalizerResourceTxt@@@std@@@std@@@std@@@std@@XZ 100062d1 f   LocalizerTxt.obj
 0001:000052dd       ?End@LocalizerResourceTxt@@QBE?AV?$_Vector_const_iterator@V?$_Vector_val@U?$_Simple_types@U?$pair@HULine@LocalizerResourceTxt@@@std@@@std@@@std@@@std@@XZ 100062dd f   LocalizerTxt.obj
 0001:000052e9       ?GetName@LocalizerResourceTxt@@UBEPBDXZ 100062e9 f   LocalizerTxt.obj
 0001:000052f5       ?GetString@LocalizerResourceTxt@@UBE_NPA_WIH@Z 100062f5 f   LocalizerTxt.obj
 0001:000055e5       ?Load@LocalizerResourceTxt@@SGPAVResource@LocalizerImp@@PBD@Z 100065e5 f   LocalizerTxt.obj
 0001:00005b40       ?RangeGetNextId@@YGHABURange@LocalizerResourceTxt@@ABV?$vector@U?$pair@HULine@LocalizerResourceTxt@@@std@@V?$mempool_alloc@U?$pair@HULine@LocalizerResourceTxt@@@std@@@@@std@@@Z 10006b40 f   LocalizerTxt.obj
 0001:00005b71       ?RangeMax@LocalizerResourceTxt@@UBEHXZ 10006b71 f   LocalizerTxt.obj
 0001:00005b75       ?RangeMin@LocalizerResourceTxt@@UBEHXZ 10006b75 f   LocalizerTxt.obj
 0001:00005bdd       ?ResetRange@LocalizerResourceTxt@@QAE_NHH@Z 10006bdd f   LocalizerTxt.obj
 0001:00005c53       ?Save@LocalizerResourceTxt@@QAE_NPBD@Z 10006c53 f   LocalizerTxt.obj
 0001:00006053       ?_Compat@?$_Vector_const_iterator@V?$_Vector_val@U?$_Simple_types@U?$pair@HULine@LocalizerResourceTxt@@@std@@@std@@@std@@@std@@QBEXABV12@@Z 10007053 f i LocalizerTxt.obj
 0001:00006056       ?_Compat@?$_Vector_const_iterator@V?$_Vector_val@U?$_Simple_types@URange@LocalizerResourceTxt@@@std@@@std@@@std@@QBEXABV12@@Z 10007056 f i LocalizerTxt.obj
 0001:00006059       ?_Destroy@?$vector@U?$pair@HULine@LocalizerResourceTxt@@@std@@V?$mempool_alloc@U?$pair@HULine@LocalizerResourceTxt@@@std@@@@@std@@IAEXPAU?$pair@HULine@LocalizerResourceTxt@@@2@0@Z 10007059 f i LocalizerTxt.obj
 0001:0000605c       ?_Destroy@?$vector@URange@LocalizerResourceTxt@@V?$mempool_alloc@URange@LocalizerResourceTxt@@@@@std@@IAEXPAURange@LocalizerResourceTxt@@0@Z 1000705c f i LocalizerTxt.obj
 0001:0000605f       ?_Getal@?$_Vector_alloc@$00U?$_Vec_base_types@U?$pair@HULine@LocalizerResourceTxt@@@std@@V?$mempool_alloc@U?$pair@HULine@LocalizerResourceTxt@@@std@@@@@std@@@std@@QAEAAU?$_Wrap_alloc@V?$mempool_alloc@U?$pair@HULine@LocalizerResourceTxt@@@std@@@@@2@XZ 1000705f f i LocalizerTxt.obj
 0001:00006063       ?_Getal@?$_Vector_alloc@$00U?$_Vec_base_types@U?$pair@HULine@LocalizerResourceTxt@@@std@@V?$mempool_alloc@U?$pair@HULine@LocalizerResourceTxt@@@std@@@@@std@@@std@@QBEABU?$_Wrap_alloc@V?$mempool_alloc@U?$pair@HULine@LocalizerResourceTxt@@@std@@@@@2@XZ 10007063 f i LocalizerTxt.obj
 0001:00006067       ?_Getal@?$_Vector_alloc@$00U?$_Vec_base_types@URange@LocalizerResourceTxt@@V?$mempool_alloc@URange@LocalizerResourceTxt@@@@@std@@@std@@QAEAAU?$_Wrap_alloc@V?$mempool_alloc@URange@LocalizerResourceTxt@@@@@2@XZ 10007067 f i LocalizerTxt.obj
 0001:0000606b       ?_Getal@?$_Vector_alloc@$00U?$_Vec_base_types@URange@LocalizerResourceTxt@@V?$mempool_alloc@URange@LocalizerResourceTxt@@@@@std@@@std@@QBEABU?$_Wrap_alloc@V?$mempool_alloc@URange@LocalizerResourceTxt@@@@@2@XZ 1000706b f i LocalizerTxt.obj
 0001:0000606f       ?_Grow_to@?$vector@U?$pair@HULine@LocalizerResourceTxt@@@std@@V?$mempool_alloc@U?$pair@HULine@LocalizerResourceTxt@@@std@@@@@std@@IBEII@Z 1000706f f i LocalizerTxt.obj
 0001:00006098       ?_Grow_to@?$vector@URange@LocalizerResourceTxt@@V?$mempool_alloc@URange@LocalizerResourceTxt@@@@@std@@IBEII@Z 10007098 f i LocalizerTxt.obj
 0001:000060c6       ?_Inside@?$vector@URange@LocalizerResourceTxt@@V?$mempool_alloc@URange@LocalizerResourceTxt@@@@@std@@IBE_NPBURange@LocalizerResourceTxt@@@Z 100070c6 f i LocalizerTxt.obj
 0001:000060dd       ?_Make_iter@?$vector@U?$pair@HULine@LocalizerResourceTxt@@@std@@V?$mempool_alloc@U?$pair@HULine@LocalizerResourceTxt@@@std@@@@@std@@QBE?AV?$_Vector_iterator@V?$_Vector_val@U?$_Simple_types@U?$pair@HULine@LocalizerResourceTxt@@@std@@@std@@@std@@@2@V?$_Vector_const_iterator@V?$_Vector_val@U?$_Simple_types@U?$pair@HULine@LocalizerResourceTxt@@@std@@@std@@@std@@@2@@Z 100070dd f i LocalizerTxt.obj
 0001:000060ea       ?_Orphan_range@?$vector@U?$pair@HULine@LocalizerResourceTxt@@@std@@V?$mempool_alloc@U?$pair@HULine@LocalizerResourceTxt@@@std@@@@@std@@IBEXPAU?$pair@HULine@LocalizerResourceTxt@@@2@0@Z 100070ea f i LocalizerTxt.obj
 0001:000060ed       ?_Orphan_range@?$vector@URange@LocalizerResourceTxt@@V?$mempool_alloc@URange@LocalizerResourceTxt@@@@@std@@IBEXPAURange@LocalizerResourceTxt@@0@Z 100070ed f i LocalizerTxt.obj
 0001:000060f0       ?_Reallocate@?$vector@U?$pair@HULine@LocalizerResourceTxt@@@std@@V?$mempool_alloc@U?$pair@HULine@LocalizerResourceTxt@@@std@@@@@std@@IAEXI@Z 100070f0 f i LocalizerTxt.obj
 0001:00006195       ?_Reallocate@?$vector@URange@LocalizerResourceTxt@@V?$mempool_alloc@URange@LocalizerResourceTxt@@@@@std@@IAEXI@Z 10007195 f i LocalizerTxt.obj
 0001:00006245       ?_Rechecked@?$_Vector_const_iterator@V?$_Vector_val@U?$_Simple_types@U?$pair@HULine@LocalizerResourceTxt@@@std@@@std@@@std@@@std@@QAEAAV12@PBU?$pair@HULine@LocalizerResourceTxt@@@2@@Z 10007245 f i LocalizerTxt.obj
 0001:00006250       ?_Rechecked@?$_Vector_iterator@V?$_Vector_val@U?$_Simple_types@U?$pair@HULine@LocalizerResourceTxt@@@std@@@std@@@std@@@std@@QAEAAV12@PAU?$pair@HULine@LocalizerResourceTxt@@@2@@Z 10007250 f i LocalizerTxt.obj
 0001:0000625b       ?_Reserve@?$vector@U?$pair@HULine@LocalizerResourceTxt@@@std@@V?$mempool_alloc@U?$pair@HULine@LocalizerResourceTxt@@@std@@@@@std@@IAEXI@Z 1000725b f i LocalizerTxt.obj
 0001:000062a1       ?_Reserve@?$vector@URange@LocalizerResourceTxt@@V?$mempool_alloc@URange@LocalizerResourceTxt@@@@@std@@IAEXI@Z 100072a1 f i LocalizerTxt.obj
 0001:000062ef       ?_Tidy@?$vector@U?$pair@HULine@LocalizerResourceTxt@@@std@@V?$mempool_alloc@U?$pair@HULine@LocalizerResourceTxt@@@std@@@@@std@@IAEXXZ 100072ef f i LocalizerTxt.obj
 0001:00006319       ?_Tidy@?$vector@URange@LocalizerResourceTxt@@V?$mempool_alloc@URange@LocalizerResourceTxt@@@@@std@@IAEXXZ 10007319 f i LocalizerTxt.obj
 0001:00006343       ?_Unchecked@?$_Vector_const_iterator@V?$_Vector_val@U?$_Simple_types@U?$pair@HULine@LocalizerResourceTxt@@@std@@@std@@@std@@@std@@QBEPBU?$pair@HULine@LocalizerResourceTxt@@@2@XZ 10007343 f i LocalizerTxt.obj
 0001:00006346       ?_Unchecked@?$_Vector_iterator@V?$_Vector_val@U?$_Simple_types@U?$pair@HULine@LocalizerResourceTxt@@@std@@@std@@@std@@@std@@QBEPAU?$pair@HULine@LocalizerResourceTxt@@@2@XZ 10007346 f i LocalizerTxt.obj
 0001:00006349       ?_Unchecked@?$_Vector_iterator@V?$_Vector_val@U?$_Simple_types@URange@LocalizerResourceTxt@@@std@@@std@@@std@@QBEPAURange@LocalizerResourceTxt@@XZ 10007349 f i LocalizerTxt.obj
 0001:0000634c       ?_Unused_capacity@?$vector@U?$pair@HULine@LocalizerResourceTxt@@@std@@V?$mempool_alloc@U?$pair@HULine@LocalizerResourceTxt@@@std@@@@@std@@QBEIXZ 1000734c f i LocalizerTxt.obj
 0001:00006356       ?_Unused_capacity@?$vector@URange@LocalizerResourceTxt@@V?$mempool_alloc@URange@LocalizerResourceTxt@@@@@std@@QBEIXZ 10007356 f i LocalizerTxt.obj
 0001:00006363       ?_Xlen@?$vector@U?$pair@HULine@LocalizerResourceTxt@@@std@@V?$mempool_alloc@U?$pair@HULine@LocalizerResourceTxt@@@std@@@@@std@@IBEXXZ 10007363 f i LocalizerTxt.obj
 0001:0000636f       ?_Xlen@?$vector@URange@LocalizerResourceTxt@@V?$mempool_alloc@URange@LocalizerResourceTxt@@@@@std@@IBEXXZ 1000736f f i LocalizerTxt.obj
 0001:0000637b       ?allocate@?$_Wrap_alloc@V?$mempool_alloc@U?$pair@HULine@LocalizerResourceTxt@@@std@@@@@std@@QAEPAU?$pair@HULine@LocalizerResourceTxt@@@2@I@Z 1000737b f i LocalizerTxt.obj
 0001:00006396       ?allocate@?$_Wrap_alloc@V?$mempool_alloc@URange@LocalizerResourceTxt@@@@@std@@QAEPAURange@LocalizerResourceTxt@@I@Z 10007396 f i LocalizerTxt.obj
 0001:000063b1       ?allocate@?$mempool_alloc@U?$pair@HULine@LocalizerResourceTxt@@@std@@@@QAEPAU?$pair@HULine@LocalizerResourceTxt@@@std@@IPBX@Z 100073b1 f i LocalizerTxt.obj
 0001:000063cc       ?allocate@?$mempool_alloc@URange@LocalizerResourceTxt@@@@QAEPAURange@LocalizerResourceTxt@@IPBX@Z 100073cc f i LocalizerTxt.obj
 0001:000063e7       ?append@?$basic_string@DU?$char_traits@D@std@@V?$allocator@D@2@@std@@QAEAAV12@ABV12@@Z 100073e7 f i LocalizerTxt.obj
 0001:000063f7       ?back@?$vector@URange@LocalizerResourceTxt@@V?$mempool_alloc@URange@LocalizerResourceTxt@@@@@std@@QAEAAURange@LocalizerResourceTxt@@XZ 100073f7 f i LocalizerTxt.obj
 0001:000063fe       ?begin@?$vector@U?$pair@HULine@LocalizerResourceTxt@@@std@@V?$mempool_alloc@U?$pair@HULine@LocalizerResourceTxt@@@std@@@@@std@@QAE?AV?$_Vector_iterator@V?$_Vector_val@U?$_Simple_types@U?$pair@HULine@LocalizerResourceTxt@@@std@@@std@@@std@@@2@XZ 100073fe f i LocalizerTxt.obj
 0001:00006409       ?begin@?$vector@U?$pair@HULine@LocalizerResourceTxt@@@std@@V?$mempool_alloc@U?$pair@HULine@LocalizerResourceTxt@@@std@@@@@std@@QBE?AV?$_Vector_const_iterator@V?$_Vector_val@U?$_Simple_types@U?$pair@HULine@LocalizerResourceTxt@@@std@@@std@@@std@@@2@XZ 10007409 f i LocalizerTxt.obj
 0001:00006414       ?begin@?$vector@URange@LocalizerResourceTxt@@V?$mempool_alloc@URange@LocalizerResourceTxt@@@@@std@@QAE?AV?$_Vector_iterator@V?$_Vector_val@U?$_Simple_types@URange@LocalizerResourceTxt@@@std@@@std@@@2@XZ 10007414 f i LocalizerTxt.obj
 0001:0000641f       ?begin@?$vector@URange@LocalizerResourceTxt@@V?$mempool_alloc@URange@LocalizerResourceTxt@@@@@std@@QBE?AV?$_Vector_const_iterator@V?$_Vector_val@U?$_Simple_types@URange@LocalizerResourceTxt@@@std@@@std@@@2@XZ 1000741f f i LocalizerTxt.obj
 0001:0000642a       ?capacity@?$vector@U?$pair@HULine@LocalizerResourceTxt@@@std@@V?$mempool_alloc@U?$pair@HULine@LocalizerResourceTxt@@@std@@@@@std@@QBEIXZ 1000742a f i LocalizerTxt.obj
 0001:00006433       ?capacity@?$vector@URange@LocalizerResourceTxt@@V?$mempool_alloc@URange@LocalizerResourceTxt@@@@@std@@QBEIXZ 10007433 f i LocalizerTxt.obj
 0001:0000643f       ?clear@?$vector@U?$pair@HULine@LocalizerResourceTxt@@@std@@V?$mempool_alloc@U?$pair@HULine@LocalizerResourceTxt@@@std@@@@@std@@QAEXXZ 1000743f f i LocalizerTxt.obj
 0001:0000644f       ?clear@?$vector@URange@LocalizerResourceTxt@@V?$mempool_alloc@URange@LocalizerResourceTxt@@@@@std@@QAEXXZ 1000744f f i LocalizerTxt.obj
 0001:0000645f       ?construct@?$mempool_alloc@U?$pair@HULine@LocalizerResourceTxt@@@std@@@@QAEXPAU?$pair@HULine@LocalizerResourceTxt@@@std@@ABU23@@Z 1000745f f i LocalizerTxt.obj
 0001:00006476       ?construct@?$mempool_alloc@URange@LocalizerResourceTxt@@@@QAEXPAURange@LocalizerResourceTxt@@ABU23@@Z 10007476 f i LocalizerTxt.obj
 0001:0000648c       ?deallocate@?$_Wrap_alloc@V?$mempool_alloc@U?$pair@HULine@LocalizerResourceTxt@@@std@@@@@std@@QAEXPAU?$pair@HULine@LocalizerResourceTxt@@@2@I@Z 1000748c f i LocalizerTxt.obj
 0001:000064a2       ?deallocate@?$_Wrap_alloc@V?$mempool_alloc@URange@LocalizerResourceTxt@@@@@std@@QAEXPAURange@LocalizerResourceTxt@@I@Z 100074a2 f i LocalizerTxt.obj
 0001:000064b8       ?deallocate@?$mempool_alloc@U?$pair@HULine@LocalizerResourceTxt@@@std@@@@QAEXPAU?$pair@HULine@LocalizerResourceTxt@@@std@@I@Z 100074b8 f i LocalizerTxt.obj
 0001:000064ce       ?deallocate@?$mempool_alloc@URange@LocalizerResourceTxt@@@@QAEXPAURange@LocalizerResourceTxt@@I@Z 100074ce f i LocalizerTxt.obj
 0001:000064e4       ?destroy@?$mempool_alloc@U?$pair@HULine@LocalizerResourceTxt@@@std@@@@QAEXPAU?$pair@HULine@LocalizerResourceTxt@@@std@@@Z 100074e4 f i LocalizerTxt.obj
 0001:000064e7       ?destroy@?$mempool_alloc@URange@LocalizerResourceTxt@@@@QAEXPAURange@LocalizerResourceTxt@@@Z 100074e7 f i LocalizerTxt.obj
 0001:000064fa       ?end@?$vector@U?$pair@HULine@LocalizerResourceTxt@@@std@@V?$mempool_alloc@U?$pair@HULine@LocalizerResourceTxt@@@std@@@@@std@@QAE?AV?$_Vector_iterator@V?$_Vector_val@U?$_Simple_types@U?$pair@HULine@LocalizerResourceTxt@@@std@@@std@@@std@@@2@XZ 100074fa f i LocalizerTxt.obj
 0001:00006506       ?end@?$vector@U?$pair@HULine@LocalizerResourceTxt@@@std@@V?$mempool_alloc@U?$pair@HULine@LocalizerResourceTxt@@@std@@@@@std@@QBE?AV?$_Vector_const_iterator@V?$_Vector_val@U?$_Simple_types@U?$pair@HULine@LocalizerResourceTxt@@@std@@@std@@@std@@@2@XZ 10007506 f i LocalizerTxt.obj
 0001:00006512       ?end@?$vector@URange@LocalizerResourceTxt@@V?$mempool_alloc@URange@LocalizerResourceTxt@@@@@std@@QAE?AV?$_Vector_iterator@V?$_Vector_val@U?$_Simple_types@URange@LocalizerResourceTxt@@@std@@@std@@@2@XZ 10007512 f i LocalizerTxt.obj
 0001:0000651e       ?end@?$vector@URange@LocalizerResourceTxt@@V?$mempool_alloc@URange@LocalizerResourceTxt@@@@@std@@QBE?AV?$_Vector_const_iterator@V?$_Vector_val@U?$_Simple_types@URange@LocalizerResourceTxt@@@std@@@std@@@2@XZ 1000751e f i LocalizerTxt.obj
 0001:0000652a       ?erase@?$vector@U?$pair@HULine@LocalizerResourceTxt@@@std@@V?$mempool_alloc@U?$pair@HULine@LocalizerResourceTxt@@@std@@@@@std@@QAE?AV?$_Vector_iterator@V?$_Vector_val@U?$_Simple_types@U?$pair@HULine@LocalizerResourceTxt@@@std@@@std@@@std@@@2@V?$_Vector_const_iterator@V?$_Vector_val@U?$_Simple_types@U?$pair@HULine@LocalizerResourceTxt@@@std@@@std@@@std@@@2@@Z 1000752a f i LocalizerTxt.obj
 0001:00006554       ?get@?$auto_ptr@VLocalizerResourceTxt@@@std@@QBEPAVLocalizerResourceTxt@@XZ 10007554 f i LocalizerTxt.obj
 0001:00006557       ?insert@?$vector@U?$pair@HULine@LocalizerResourceTxt@@@std@@V?$mempool_alloc@U?$pair@HULine@LocalizerResourceTxt@@@std@@@@@std@@QAE?AV?$_Vector_iterator@V?$_Vector_val@U?$_Simple_types@U?$pair@HULine@LocalizerResourceTxt@@@std@@@std@@@std@@@2@V?$_Vector_const_iterator@V?$_Vector_val@U?$_Simple_types@U?$pair@HULine@LocalizerResourceTxt@@@std@@@std@@@std@@@2@$$QAU?$pair@HULine@LocalizerResourceTxt@@@2@@Z 10007557 f i LocalizerTxt.obj
 0001:0000656f       ?max@?$numeric_limits@I@std@@SGIXZ 1000756f f i LocalizerTxt.obj
 0001:00006573       ?max_size@?$_Wrap_alloc@V?$mempool_alloc@U?$pair@HULine@LocalizerResourceTxt@@@std@@@@@std@@QBEIXZ 10007573 f i LocalizerTxt.obj
 0001:00006577       ?max_size@?$_Wrap_alloc@V?$mempool_alloc@URange@LocalizerResourceTxt@@@@@std@@QBEIXZ 10007577 f i LocalizerTxt.obj
 0001:0000657b       ?max_size@?$allocator_traits@V?$mempool_alloc@U?$pair@HULine@LocalizerResourceTxt@@@std@@@@@std@@SGIABV?$mempool_alloc@U?$pair@HULine@LocalizerResourceTxt@@@std@@@@@Z 1000757b f i LocalizerTxt.obj
 0001:00006581       ?max_size@?$allocator_traits@V?$mempool_alloc@URange@LocalizerResourceTxt@@@@@std@@SGIABV?$mempool_alloc@URange@LocalizerResourceTxt@@@@@Z 10007581 f i LocalizerTxt.obj
 0001:00006587       ?max_size@?$vector@U?$pair@HULine@LocalizerResourceTxt@@@std@@V?$mempool_alloc@U?$pair@HULine@LocalizerResourceTxt@@@std@@@@@std@@QBEIXZ 10007587 f i LocalizerTxt.obj
 0001:0000658b       ?max_size@?$vector@URange@LocalizerResourceTxt@@V?$mempool_alloc@URange@LocalizerResourceTxt@@@@@std@@QBEIXZ 1000758b f i LocalizerTxt.obj
 0001:0000658f       ?pointer_to@?$pointer_traits@PAU?$pair@HULine@LocalizerResourceTxt@@@std@@@std@@SGPAU?$pair@HULine@LocalizerResourceTxt@@@2@AAU32@@Z 1000758f f i LocalizerTxt.obj
 0001:00006596       ?pointer_to@?$pointer_traits@PAURange@LocalizerResourceTxt@@@std@@SGPAURange@LocalizerResourceTxt@@AAU34@@Z 10007596 f i LocalizerTxt.obj
 0001:0000659d       ?pointer_to@?$pointer_traits@PBU?$pair@HULine@LocalizerResourceTxt@@@std@@@std@@SGPBU?$pair@HULine@LocalizerResourceTxt@@@2@ABU32@@Z 1000759d f i LocalizerTxt.obj
 0001:000065a4       ?pointer_to@?$pointer_traits@PBURange@LocalizerResourceTxt@@@std@@SGPBURange@LocalizerResourceTxt@@ABU34@@Z 100075a4 f i LocalizerTxt.obj
 0001:000065ab       ?push_back@?$vector@URange@LocalizerResourceTxt@@V?$mempool_alloc@URange@LocalizerResourceTxt@@@@@std@@QAEXABURange@LocalizerResourceTxt@@@Z 100075ab f i LocalizerTxt.obj
 0001:00006611       ?release@?$auto_ptr@VLocalizerResourceTxt@@@std@@QAEPAVLocalizerResourceTxt@@XZ 10007611 f i LocalizerTxt.obj
 0001:00006617       ?reserve@?$basic_string@DU?$char_traits@D@std@@V?$allocator@D@2@@std@@QAEXI@Z 10007617 f i LocalizerTxt.obj
 0001:0000664b       ?size@?$vector@U?$pair@HULine@LocalizerResourceTxt@@@std@@V?$mempool_alloc@U?$pair@HULine@LocalizerResourceTxt@@@std@@@@@std@@QBEIXZ 1000764b f i LocalizerTxt.obj
 0001:00006654       ?size@?$vector@URange@LocalizerResourceTxt@@V?$mempool_alloc@URange@LocalizerResourceTxt@@@@@std@@QBEIXZ 10007654 f i LocalizerTxt.obj
 0001:00006660       ?swap@?$pair@HULine@LocalizerResourceTxt@@@std@@QAEXAAU12@@Z 10007660 f i LocalizerTxt.obj
 0001:0000669b       ??$?0AAPAULine@LocalizerResourceUCS@@AAPAU01@@?$pair@PAULine@LocalizerResourceUCS@@PAU12@@std@@QAE@AAPAULine@LocalizerResourceUCS@@0PAPAX@Z 1000769b f i LocalizerUCS.obj
 0001:000066b1       ??$?0PAULine@LocalizerResourceUCS@@PAU01@@?$pair@PAULine@LocalizerResourceUCS@@PAU12@@std@@QAE@$$QAU01@PAPAX@Z 100076b1 f i LocalizerUCS.obj
 0001:000066c4       ??$?0PAULine@LocalizerResourceUCS@@PAU01@@?$pair@PBULine@LocalizerResourceUCS@@PBU12@@std@@QAE@$$QAU?$pair@PAULine@LocalizerResourceUCS@@PAU12@@1@PAPAX@Z 100076c4 f i LocalizerUCS.obj
 0001:000066d7       ??$?APAI@?$list4@AAPB_WAAPB_WAAPB_WAAPB_W@_bi@boost@@QBEABQAIABV?$value@PAI@12@@Z 100076d7 f i LocalizerUCS.obj
 0001:000066de       ??$?APAPA_W@?$list4@AAPB_WAAPB_WAAPB_WAAPB_W@_bi@boost@@QBEABQAPA_WABV?$value@PAPA_W@12@@Z 100076de f i LocalizerUCS.obj
 0001:000066e5       ??$?APAULine@LocalizerResourceUCS@@@?$list4@AAPB_WAAPB_WAAPB_WAAPB_W@_bi@boost@@QBEABQAULine@LocalizerResourceUCS@@ABV?$value@PAULine@LocalizerResourceUCS@@@12@@Z 100076e5 f i LocalizerUCS.obj
 0001:000066ec       ??$?RPB_WPB_WPB_WPB_W@?$bind_t@_NP6G_NPB_W000PAI1@ZV?$list6@V?$arg@$00@boost@@V?$arg@$01@2@V?$arg@$02@2@V?$arg@$03@2@V?$value@PAI@_bi@2@V672@@_bi@boost@@@_bi@boost@@QAE_NAAPB_W000@Z 100076ec f i LocalizerUCS.obj
 0001:00006711       ??$?RPB_WPB_WPB_WPB_W@?$bind_t@_NP6G_NPB_W000PAULine@LocalizerResourceUCS@@PAIPAPA_W@ZV?$list7@V?$arg@$00@boost@@V?$arg@$01@2@V?$arg@$02@2@V?$arg@$03@2@V?$value@PAULine@LocalizerResourceUCS@@@_bi@2@V?$value@PAI@72@V?$value@PAPA_W@72@@_bi@boost@@@_bi@boost@@QAE_NAAPB_W000@Z 10007711 f i LocalizerUCS.obj
 0001:00006748       ??$?R_NP6G_NPB_W000PAI1@ZV?$list4@AAPB_WAAPB_WAAPB_WAAPB_W@_bi@boost@@@?$list6@V?$arg@$00@boost@@V?$arg@$01@2@V?$arg@$02@2@V?$arg@$03@2@V?$value@PAI@_bi@2@V672@@_bi@boost@@QBE_NV?$type@_N@12@P6G_NPB_W111PAI2@ZAAV?$list4@AAPB_WAAPB_WAAPB_WAAPB_W@12@@Z 10007748 f i LocalizerUCS.obj
 0001:00006770       ??$?R_NP6G_NPB_W000PAULine@LocalizerResourceUCS@@PAIPAPA_W@ZV?$list4@AAPB_WAAPB_WAAPB_WAAPB_W@_bi@boost@@@?$list7@V?$arg@$00@boost@@V?$arg@$01@2@V?$arg@$02@2@V?$arg@$03@2@V?$value@PAULine@LocalizerResourceUCS@@@_bi@2@V?$value@PAI@72@V?$value@PAPA_W@72@@_bi@boost@@QBE_NV?$type@_N@12@P6G_NPB_W111PAULine@LocalizerResourceUCS@@PAIPAPA_W@ZAAV?$list4@AAPB_WAAPB_WAAPB_WAAPB_W@12@@Z 10007770 f i LocalizerUCS.obj
 0001:00006888       ??$_Adjacent_find@PAULine@LocalizerResourceUCS@@ULineEqual@?A0xa493ca04@@@std@@YGPAULine@LocalizerResourceUCS@@PAU12@0ULineEqual@?A0xa493ca04@@@Z 10007888 f i LocalizerUCS.obj
 0001:000068b0       ??$_Adjust_heap@PAULine@LocalizerResourceUCS@@HU12@ULineLess@?A0xa493ca04@@@std@@YGXPAULine@LocalizerResourceUCS@@HH$$QAU12@ULineLess@?A0xa493ca04@@@Z 100078b0 f i LocalizerUCS.obj
 0001:00006918       ??$_Advance@PAULine@LocalizerResourceUCS@@H@std@@YGXAAPAULine@LocalizerResourceUCS@@HUrandom_access_iterator_tag@0@@Z 10007918 f i LocalizerUCS.obj
 0001:00006928       ??$_Dist_type@PAULine@LocalizerResourceUCS@@@std@@YGPAHPAULine@LocalizerResourceUCS@@@Z 10007928 f i LocalizerUCS.obj
 0001:0000692d       ??$_Distance2@PAULine@LocalizerResourceUCS@@H@std@@YGXPAULine@LocalizerResourceUCS@@0AAHUrandom_access_iterator_tag@0@@Z 1000792d f i LocalizerUCS.obj
 0001:00006941       ??$_Distance@PAULine@LocalizerResourceUCS@@H@std@@YGXPAULine@LocalizerResourceUCS@@0AAH@Z 10007941 f i LocalizerUCS.obj
 0001:00006955       ??$_Equal_range@PAULine@LocalizerResourceUCS@@HHULineLess@?A0xa493ca04@@@std@@YG?AU?$pair@PAULine@LocalizerResourceUCS@@PAU12@@0@PAULine@LocalizerResourceUCS@@0ABHULineLess@?A0xa493ca04@@PAH@Z 10007955 f i LocalizerUCS.obj
 0001:000069de       ??$_Insertion_sort1@PAULine@LocalizerResourceUCS@@ULineLess@?A0xa493ca04@@U12@@std@@YGXPAULine@LocalizerResourceUCS@@0ULineLess@?A0xa493ca04@@0@Z 100079de f i LocalizerUCS.obj
 0001:00006a43       ??$_Insertion_sort@PAULine@LocalizerResourceUCS@@ULineLess@?A0xa493ca04@@@std@@YGXPAULine@LocalizerResourceUCS@@0ULineLess@?A0xa493ca04@@@Z 10007a43 f i LocalizerUCS.obj
 0001:00006a59       ??$_Iter_cat@PAULine@LocalizerResourceUCS@@@std@@YG?AUrandom_access_iterator_tag@0@ABQAULine@LocalizerResourceUCS@@@Z 10007a59 f i LocalizerUCS.obj
 0001:00006a60       ??$_Lower_bound@PAULine@LocalizerResourceUCS@@HHULineLess@?A0xa493ca04@@@std@@YGPAULine@LocalizerResourceUCS@@PAU12@0ABHULineLess@?A0xa493ca04@@PAH@Z 10007a60 f i LocalizerUCS.obj
 0001:00006aa2       ??$_Make_heap@PAULine@LocalizerResourceUCS@@HU12@ULineLess@?A0xa493ca04@@@std@@YGXPAULine@LocalizerResourceUCS@@0ULineLess@?A0xa493ca04@@PAH0@Z 10007aa2 f i LocalizerUCS.obj
 0001:00006afa       ??$_Med3@PAULine@LocalizerResourceUCS@@ULineLess@?A0xa493ca04@@@std@@YGXPAULine@LocalizerResourceUCS@@00ULineLess@?A0xa493ca04@@@Z 10007afa f i LocalizerUCS.obj
 0001:00006b56       ??$_Median@PAULine@LocalizerResourceUCS@@ULineLess@?A0xa493ca04@@@std@@YGXPAULine@LocalizerResourceUCS@@00ULineLess@?A0xa493ca04@@@Z 10007b56 f i LocalizerUCS.obj
 0001:00006beb       ??$_Move@AAULine@LocalizerResourceUCS@@@std@@YG$$QAULine@LocalizerResourceUCS@@AAU12@@Z 10007beb f i LocalizerUCS.obj
 0001:00006bf2       ??$_Move_backward@PAULine@LocalizerResourceUCS@@PAU12@@std@@YGPAULine@LocalizerResourceUCS@@PAU12@00@Z 10007bf2 f i LocalizerUCS.obj
 0001:00006c0a       ??$_Move_backward@PAULine@LocalizerResourceUCS@@PAU12@@std@@YGPAULine@LocalizerResourceUCS@@PAU12@00U_Nonscalar_ptr_iterator_tag@0@@Z 10007c0a f i LocalizerUCS.obj
 0001:00006c33       ??$_Pop_heap@PAULine@LocalizerResourceUCS@@HU12@ULineLess@?A0xa493ca04@@@std@@YGXPAULine@LocalizerResourceUCS@@00$$QAU12@ULineLess@?A0xa493ca04@@PAH@Z 10007c33 f i LocalizerUCS.obj
 0001:00006c61       ??$_Pop_heap@PAULine@LocalizerResourceUCS@@ULineLess@?A0xa493ca04@@@std@@YGXPAULine@LocalizerResourceUCS@@0ULineLess@?A0xa493ca04@@@Z 10007c61 f i LocalizerUCS.obj
 0001:00006c77       ??$_Pop_heap_0@PAULine@LocalizerResourceUCS@@U12@ULineLess@?A0xa493ca04@@@std@@YGXPAULine@LocalizerResourceUCS@@0ULineLess@?A0xa493ca04@@0@Z 10007c77 f i LocalizerUCS.obj
 0001:00006ca4       ??$_Ptr_cat@ULine@LocalizerResourceUCS@@U12@@std@@YG?AU_Nonscalar_ptr_iterator_tag@0@PAULine@LocalizerResourceUCS@@0@Z 10007ca4 f i LocalizerUCS.obj
 0001:00006cad       ??$_Push_heap@PAULine@LocalizerResourceUCS@@HU12@ULineLess@?A0xa493ca04@@@std@@YGXPAULine@LocalizerResourceUCS@@HH$$QAU12@ULineLess@?A0xa493ca04@@@Z 10007cad f i LocalizerUCS.obj
 0001:00006cf5       ??$_Rechecked@PAULine@LocalizerResourceUCS@@PAU12@@std@@YGAAPAULine@LocalizerResourceUCS@@AAPAU12@PAU12@@Z 10007cf5 f i LocalizerUCS.obj
 0001:00006d02       ??$_Sort@PAULine@LocalizerResourceUCS@@HULineLess@?A0xa493ca04@@@std@@YGXPAULine@LocalizerResourceUCS@@0HULineLess@?A0xa493ca04@@@Z 10007d02 f i LocalizerUCS.obj
 0001:00006dc8       ??$_Sort_heap@PAULine@LocalizerResourceUCS@@ULineLess@?A0xa493ca04@@@std@@YGXPAULine@LocalizerResourceUCS@@0ULineLess@?A0xa493ca04@@@Z 10007dc8 f i LocalizerUCS.obj
 0001:00006dfb       ??$_Unchecked@PAULine@LocalizerResourceUCS@@@std@@YGPAULine@LocalizerResourceUCS@@PAU12@@Z 10007dfb f i LocalizerUCS.obj
 0001:00006e02       ??$_Unguarded_partition@PAULine@LocalizerResourceUCS@@ULineLess@?A0xa493ca04@@@std@@YG?AU?$pair@PAULine@LocalizerResourceUCS@@PAU12@@0@PAULine@LocalizerResourceUCS@@0ULineLess@?A0xa493ca04@@@Z 10007e02 f i LocalizerUCS.obj
 0001:00006fb3       ??$_Upper_bound@PAULine@LocalizerResourceUCS@@HHULineLess@?A0xa493ca04@@@std@@YGPAULine@LocalizerResourceUCS@@PAU12@0ABHULineLess@?A0xa493ca04@@PAH@Z 10007fb3 f i LocalizerUCS.obj
 0001:00006ff5       ??$_Val_type@PAULine@LocalizerResourceUCS@@@std@@YGPAULine@LocalizerResourceUCS@@PAU12@@Z 10007ff5 f i LocalizerUCS.obj
 0001:00006ffa       ??$adjacent_find@PAULine@LocalizerResourceUCS@@ULineEqual@?A0xa493ca04@@@std@@YGPAULine@LocalizerResourceUCS@@PAU12@0ULineEqual@?A0xa493ca04@@@Z 10007ffa f i LocalizerUCS.obj
 0001:00006fff       ??$advance@PAULine@LocalizerResourceUCS@@H@std@@YGXAAPAULine@LocalizerResourceUCS@@H@Z 10007fff f i LocalizerUCS.obj
 0001:0000700f       ??$bind@_NPB_WPB_WPB_WPB_WPAIPAIV?$arg@$00@boost@@V?$arg@$01@2@V?$arg@$02@2@V?$arg@$03@2@PAIPAI@boost@@YG?AV?$bind_t@_NP6G_NPB_W000PAI1@ZV?$list6@V?$arg@$00@boost@@V?$arg@$01@2@V?$arg@$02@2@V?$arg@$03@2@V?$value@PAI@_bi@2@V672@@_bi@boost@@@_bi@0@P6G_NPB_W000PAI1@ZV?$arg@$00@0@V?$arg@$01@0@V?$arg@$02@0@V?$arg@$03@0@11@Z 1000800f f i LocalizerUCS.obj
 0001:0000703a       ??$bind@_NPB_WPB_WPB_WPB_WPAULine@LocalizerResourceUCS@@PAIPAPA_WV?$arg@$00@boost@@V?$arg@$01@4@V?$arg@$02@4@V?$arg@$03@4@PAU12@PAIPAPA_W@boost@@YG?AV?$bind_t@_NP6G_NPB_W000PAULine@LocalizerResourceUCS@@PAIPAPA_W@ZV?$list7@V?$arg@$00@boost@@V?$arg@$01@2@V?$arg@$02@2@V?$arg@$03@2@V?$value@PAULine@LocalizerResourceUCS@@@_bi@2@V?$value@PAI@72@V?$value@PAPA_W@72@@_bi@boost@@@_bi@0@P6G_NPB_W000PAULine@LocalizerResourceUCS@@PAIPAPA_W@ZV?$arg@$00@0@V?$arg@$01@0@V?$arg@$02@0@V?$arg@$03@0@123@Z 1000803a f i LocalizerUCS.obj
 0001:0000706c       ??$checked_delete@VFileBuffer@?A0xa493ca04@@@boost@@YGXPAVFileBuffer@?A0xa493ca04@@@Z 1000806c f i LocalizerUCS.obj
 0001:0000707e       ??$equal_range@PAULine@LocalizerResourceUCS@@HULineLess@?A0xa493ca04@@@std@@YG?AU?$pair@PAULine@LocalizerResourceUCS@@PAU12@@0@PAULine@LocalizerResourceUCS@@0ABHULineLess@?A0xa493ca04@@@Z 1000807e f i LocalizerUCS.obj
 0001:000070ab       ??$forward@AAPAULine@LocalizerResourceUCS@@@std@@YGAAPAULine@LocalizerResourceUCS@@AAPAU12@@Z 100080ab f i LocalizerUCS.obj
 0001:000070b2       ??$forward@PAULine@LocalizerResourceUCS@@@std@@YG$$QAPAULine@LocalizerResourceUCS@@AAPAU12@@Z 100080b2 f i LocalizerUCS.obj
 0001:000070b9       ??$iter_swap@PAULine@LocalizerResourceUCS@@PAU12@@std@@YGXPAULine@LocalizerResourceUCS@@0@Z 100080b9 f i LocalizerUCS.obj
 0001:000070dc       ??$lower_bound@PAULine@LocalizerResourceUCS@@HULineLess@?A0xa493ca04@@@std@@YGPAULine@LocalizerResourceUCS@@PAU12@0ABHULineLess@?A0xa493ca04@@@Z 100080dc f i LocalizerUCS.obj
 0001:000070f6       ??$make_heap@PAULine@LocalizerResourceUCS@@ULineLess@?A0xa493ca04@@@std@@YGXPAULine@LocalizerResourceUCS@@0ULineLess@?A0xa493ca04@@@Z 100080f6 f i LocalizerUCS.obj
 0001:0000711d       ??$move@AAULine@LocalizerResourceUCS@@@std@@YG$$QAULine@LocalizerResourceUCS@@AAU12@@Z 1000811d f i LocalizerUCS.obj
 0001:00007124       ??$sort@PAULine@LocalizerResourceUCS@@ULineLess@?A0xa493ca04@@@std@@YGXPAULine@LocalizerResourceUCS@@0ULineLess@?A0xa493ca04@@@Z 10008124 f i LocalizerUCS.obj
 0001:00007143       ??$sort_heap@PAULine@LocalizerResourceUCS@@ULineLess@?A0xa493ca04@@@std@@YGXPAULine@LocalizerResourceUCS@@0ULineLess@?A0xa493ca04@@@Z 10008143 f i LocalizerUCS.obj
 0001:00007157       ??$swap@ULine@LocalizerResourceUCS@@@std@@YGXAAULine@LocalizerResourceUCS@@0@Z 10008157 f i LocalizerUCS.obj
 0001:0000717a       ??$unwrap@P6G_NPB_W000PAI1@Z@_bi@boost@@YGAAP6G_NPB_W000PAI1@ZAAP6G_N000011@ZJ@Z 1000817a f i LocalizerUCS.obj
 0001:00007181       ??$unwrap@P6G_NPB_W000PAULine@LocalizerResourceUCS@@PAIPAPA_W@Z@_bi@boost@@YGAAP6G_NPB_W000PAULine@LocalizerResourceUCS@@PAIPAPA_W@ZAAP6G_N0000123@ZJ@Z 10008181 f i LocalizerUCS.obj
 0001:00007188       ??$upper_bound@PAULine@LocalizerResourceUCS@@HULineLess@?A0xa493ca04@@@std@@YGPAULine@LocalizerResourceUCS@@PAU12@0ABHULineLess@?A0xa493ca04@@@Z 10008188 f i LocalizerUCS.obj
 0001:000071a2       ??0?$auto_ptr@VFileBuffer@?A0xa493ca04@@@std@@QAE@PAVFileBuffer@?A0xa493ca04@@@Z 100081a2 f i LocalizerUCS.obj
 0001:000071ad       ??0?$auto_ptr@VLocalizerResourceUCS@@@std@@QAE@PAVLocalizerResourceUCS@@@Z 100081ad f i LocalizerUCS.obj
 0001:000071b8       ??0?$bind_t@_NP6G_NPB_W000PAI1@ZV?$list6@V?$arg@$00@boost@@V?$arg@$01@2@V?$arg@$02@2@V?$arg@$03@2@V?$value@PAI@_bi@2@V672@@_bi@boost@@@_bi@boost@@QAE@P6G_NPB_W000PAI1@ZABV?$list6@V?$arg@$00@boost@@V?$arg@$01@2@V?$arg@$02@2@V?$arg@$03@2@V?$value@PAI@_bi@2@V672@@12@@Z 100081b8 f i LocalizerUCS.obj
 0001:000071d1       ??0?$bind_t@_NP6G_NPB_W000PAULine@LocalizerResourceUCS@@PAIPAPA_W@ZV?$list7@V?$arg@$00@boost@@V?$arg@$01@2@V?$arg@$02@2@V?$arg@$03@2@V?$value@PAULine@LocalizerResourceUCS@@@_bi@2@V?$value@PAI@72@V?$value@PAPA_W@72@@_bi@boost@@@_bi@boost@@QAE@P6G_NPB_W000PAULine@LocalizerResourceUCS@@PAIPAPA_W@ZABV?$list7@V?$arg@$00@boost@@V?$arg@$01@2@V?$arg@$02@2@V?$arg@$03@2@V?$value@PAULine@LocalizerResourceUCS@@@_bi@2@V?$value@PAI@72@V?$value@PAPA_W@72@@12@@Z 100081d1 f i LocalizerUCS.obj
 0001:000071eb       ??0?$list4@AAPB_WAAPB_WAAPB_WAAPB_W@_bi@boost@@QAE@AAPB_W000@Z 100081eb f i LocalizerUCS.obj
 0001:0000720b       ??0?$list6@V?$arg@$00@boost@@V?$arg@$01@2@V?$arg@$02@2@V?$arg@$03@2@V?$value@PAI@_bi@2@V672@@_bi@boost@@QAE@V?$arg@$00@2@V?$arg@$01@2@V?$arg@$02@2@V?$arg@$03@2@V?$value@PAI@12@4@Z 1000820b f i LocalizerUCS.obj
 0001:0000721e       ??0?$list7@V?$arg@$00@boost@@V?$arg@$01@2@V?$arg@$02@2@V?$arg@$03@2@V?$value@PAULine@LocalizerResourceUCS@@@_bi@2@V?$value@PAI@72@V?$value@PAPA_W@72@@_bi@boost@@QAE@V?$arg@$00@2@V?$arg@$01@2@V?$arg@$02@2@V?$arg@$03@2@V?$value@PAULine@LocalizerResourceUCS@@@12@V?$value@PAI@12@V?$value@PAPA_W@12@@Z 1000821e f i LocalizerUCS.obj
 0001:00007238       ??0?$scoped_ptr@VFileBuffer@?A0xa493ca04@@@boost@@QAE@PAVFileBuffer@?A0xa493ca04@@@Z 10008238 f i LocalizerUCS.obj
 0001:00007243       ??0?$value@PAI@_bi@boost@@QAE@ABQAI@Z 10008243 f i LocalizerUCS.obj
 0001:00007250       ??0?$value@PAPA_W@_bi@boost@@QAE@ABQAPA_W@Z 10008250 f i LocalizerUCS.obj
 0001:0000725d       ??0?$value@PAULine@LocalizerResourceUCS@@@_bi@boost@@QAE@ABQAULine@LocalizerResourceUCS@@@Z 1000825d f i LocalizerUCS.obj
 0001:0000726a       ??0FileBuffer@?A0xa493ca04@@AAE@K@Z 1000826a f i LocalizerUCS.obj
 0001:00007288       ??0LocalizerResourceUCS@@AAE@PBDII@Z 10008288 f   LocalizerUCS.obj
 0001:000072f1       ??1?$auto_ptr@VFileBuffer@?A0xa493ca04@@@std@@QAE@XZ 100082f1 f i LocalizerUCS.obj
 0001:000072ff       ??1?$auto_ptr@VLocalizerResourceUCS@@@std@@QAE@XZ 100082ff f i LocalizerUCS.obj
 0001:0000730c       ??1?$scoped_ptr@VFileBuffer@?A0xa493ca04@@@boost@@QAE@XZ 1000830c f i LocalizerUCS.obj
 0001:0000731a       ??1FileBuffer@?A0xa493ca04@@QAE@XZ 1000831a f i LocalizerUCS.obj
 0001:00007329       ??1LocalizerResourceUCS@@UAE@XZ 10008329 f   LocalizerUCS.obj
 0001:00007391       ??7?$scoped_ptr@VFileBuffer@?A0xa493ca04@@@boost@@QBE_NXZ 10008391 f i LocalizerUCS.obj
 0001:00007399       ??A?$list4@AAPB_WAAPB_WAAPB_WAAPB_W@_bi@boost@@QBEAAPB_WV?$arg@$00@2@@Z 10008399 f i LocalizerUCS.obj
 0001:0000739e       ??A?$list4@AAPB_WAAPB_WAAPB_WAAPB_W@_bi@boost@@QBEAAPB_WV?$arg@$01@2@@Z 1000839e f i LocalizerUCS.obj
 0001:000073a4       ??A?$list4@AAPB_WAAPB_WAAPB_WAAPB_W@_bi@boost@@QBEAAPB_WV?$arg@$02@2@@Z 100083a4 f i LocalizerUCS.obj
 0001:000073aa       ??A?$list4@AAPB_WAAPB_WAAPB_WAAPB_W@_bi@boost@@QBEAAPB_WV?$arg@$03@2@@Z 100083aa f i LocalizerUCS.obj
 0001:000073b0       ??C?$auto_ptr@VFileBuffer@?A0xa493ca04@@@std@@QBEPAVFileBuffer@?A0xa493ca04@@XZ 100083b0 f i LocalizerUCS.obj
 0001:000073b3       ??C?$auto_ptr@VLocalizerResourceUCS@@@std@@QBEPAVLocalizerResourceUCS@@XZ 100083b3 f i LocalizerUCS.obj
 0001:000073b6       ??C?$scoped_ptr@VFileBuffer@?A0xa493ca04@@@boost@@QBEPAVFileBuffer@?A0xa493ca04@@XZ 100083b6 f i LocalizerUCS.obj
 0001:000073b9       ??RLineEqual@?A0xa493ca04@@QBE_NABULine@LocalizerResourceUCS@@0@Z 100083b9 f i LocalizerUCS.obj
 0001:000073cd       ??RLineLess@?A0xa493ca04@@QBE_NABULine@LocalizerResourceUCS@@0@Z 100083cd f i LocalizerUCS.obj
 0001:000073e1       ??RLineLess@?A0xa493ca04@@QBE_NABULine@LocalizerResourceUCS@@H@Z 100083e1 f i LocalizerUCS.obj
 0001:000073f3       ??RLineLess@?A0xa493ca04@@QBE_NHABULine@LocalizerResourceUCS@@@Z 100083f3 f i LocalizerUCS.obj
 0001:00007405       ??_GFileBuffer@?A0xa493ca04@@QAEPAXI@Z 10008405 f i LocalizerUCS.obj
 0001:0000742a       ??_GLocalizerResourceUCS@@UAEPAXI@Z 1000842a f i LocalizerUCS.obj
 0001:0000742a       ??_ELocalizerResourceUCS@@UAEPAXI@Z 1000842a f i LocalizerUCS.obj
 0001:00007462       ?Create@FileBuffer@?A0xa493ca04@@SGPAV12@PBD@Z 10008462 f i LocalizerUCS.obj
 0001:000075af       ?Get@FileBuffer@?A0xa493ca04@@QBEPB_WXZ 100085af f i LocalizerUCS.obj
 0001:000075b2       ?GetName@LocalizerResourceUCS@@UBEPBDXZ 100085b2 f   LocalizerUCS.obj
 0001:000075be       ?GetString@LocalizerResourceUCS@@UBE_NPA_WIH@Z 100085be f   LocalizerUCS.obj
 0001:00007696       ?Load@LocalizerResourceUCS@@SGPAVResource@LocalizerImp@@PBD@Z 10008696 f   LocalizerUCS.obj
 0001:000077d1       ?RangeMax@LocalizerResourceUCS@@UBEHXZ 100087d1 f   LocalizerUCS.obj
 0001:000077e3       ?RangeMin@LocalizerResourceUCS@@UBEHXZ 100087e3 f   LocalizerUCS.obj
 0001:000078f4       ?get@?$auto_ptr@VFileBuffer@?A0xa493ca04@@@std@@QBEPAVFileBuffer@?A0xa493ca04@@XZ 100088f4 f i LocalizerUCS.obj
 0001:000078f7       ?get@?$auto_ptr@VLocalizerResourceUCS@@@std@@QBEPAVLocalizerResourceUCS@@XZ 100088f7 f i LocalizerUCS.obj
 0001:000078fa       ?get@?$value@PAI@_bi@boost@@QBEABQAIXZ 100088fa f i LocalizerUCS.obj
 0001:000078fd       ?get@?$value@PAPA_W@_bi@boost@@QBEABQAPA_WXZ 100088fd f i LocalizerUCS.obj
 0001:00007900       ?get@?$value@PAULine@LocalizerResourceUCS@@@_bi@boost@@QBEABQAULine@LocalizerResourceUCS@@XZ 10008900 f i LocalizerUCS.obj
 0001:00007903       ?release@?$auto_ptr@VFileBuffer@?A0xa493ca04@@@std@@QAEPAVFileBuffer@?A0xa493ca04@@XZ 10008903 f i LocalizerUCS.obj
 0001:00007909       ?release@?$auto_ptr@VLocalizerResourceUCS@@@std@@QAEPAVLocalizerResourceUCS@@XZ 10008909 f i LocalizerUCS.obj
 0001:0000790f       ??0_Generic_error_category@std@@QAE@XZ 1000890f f i pch.obj
 0001:00007918       ??0_Ignore@std@@QAE@XZ     10008918 f i pch.obj
 0001:0000791b       ??0_Iostream_error_category@std@@QAE@XZ 1000891b f i pch.obj
 0001:00007924       ??0_System_error_category@std@@QAE@XZ 10008924 f i pch.obj
 0001:0000792d       ??0error_category@std@@QAE@XZ 1000892d f i pch.obj
 0001:00007936       ??0error_condition@std@@QAE@HABVerror_category@1@@Z 10008936 f i pch.obj
 0001:00007948       ??1_Generic_error_category@std@@UAE@XZ 10008948 f i pch.obj
 0001:0000794f       ??1_Iostream_error_category@std@@UAE@XZ 1000894f f i pch.obj
 0001:00007956       ??1_System_error_category@std@@UAE@XZ 10008956 f i pch.obj
 0001:0000795d       ??1error_category@std@@UAE@XZ 1000895d f i pch.obj
 0001:00007964       ??8error_category@std@@QBE_NABV01@@Z 10008964 f i pch.obj
 0001:00007970       ??8error_condition@std@@QBE_NABV01@@Z 10008970 f i pch.obj
 0001:0000798c       ??_E_Generic_error_category@std@@UAEPAXI@Z 1000898c f i pch.obj
 0001:0000798c       ??_G_Generic_error_category@std@@UAEPAXI@Z 1000898c f i pch.obj
 0001:000079a9       ??_E_Iostream_error_category@std@@UAEPAXI@Z 100089a9 f i pch.obj
 0001:000079a9       ??_G_Iostream_error_category@std@@UAEPAXI@Z 100089a9 f i pch.obj
 0001:000079c6       ??_E_System_error_category@std@@UAEPAXI@Z 100089c6 f i pch.obj
 0001:000079c6       ??_G_System_error_category@std@@UAEPAXI@Z 100089c6 f i pch.obj
 0001:000079e3       ??_Gerror_category@std@@UAEPAXI@Z 100089e3 f i pch.obj
 0001:000079e3       ??_Eerror_category@std@@UAEPAXI@Z 100089e3 f i pch.obj
 0001:00007a00       ?category@error_code@std@@QBEABVerror_category@2@XZ 10008a00 f i pch.obj
 0001:00007a04       ?category@error_condition@std@@QBEABVerror_category@2@XZ 10008a04 f i pch.obj
 0001:00007a08       ?default_error_condition@_System_error_category@std@@UBE?AVerror_condition@2@H@Z 10008a08 f i pch.obj
 0001:00007a33       ?default_error_condition@error_category@std@@UBE?AVerror_condition@2@H@Z 10008a33 f i pch.obj
 0001:00007a43       ?equivalent@error_category@std@@UBE_NABVerror_code@2@H@Z 10008a43 f i pch.obj
 0001:00007a5e       ?equivalent@error_category@std@@UBE_NHABVerror_condition@2@@Z 10008a5e f i pch.obj
 0001:00007a7d       ?generic_category@std@@YGABVerror_category@1@XZ 10008a7d f i pch.obj
 0001:00007a83       ?message@_Generic_error_category@std@@UBE?AV?$basic_string@DU?$char_traits@D@std@@V?$allocator@D@2@@2@H@Z 10008a83 f i pch.obj
 0001:00007aaf       ?message@_Iostream_error_category@std@@UBE?AV?$basic_string@DU?$char_traits@D@std@@V?$allocator@D@2@@2@H@Z 10008aaf f i pch.obj
 0001:00007ade       ?message@_System_error_category@std@@UBE?AV?$basic_string@DU?$char_traits@D@std@@V?$allocator@D@2@@2@H@Z 10008ade f i pch.obj
 0001:00007b0a       ?name@_Generic_error_category@std@@UBEPBDXZ 10008b0a f i pch.obj
 0001:00007b10       ?name@_Iostream_error_category@std@@UBEPBDXZ 10008b10 f i pch.obj
 0001:00007b16       ?name@_System_error_category@std@@UBEPBDXZ 10008b16 f i pch.obj
 0001:00007b1c       ?system_category@std@@YGABVerror_category@1@XZ 10008b1c f i pch.obj
 0001:00007b22       ?value@error_code@std@@QBEHXZ 10008b22 f i pch.obj
 0001:00007b25       ?value@error_condition@std@@QBEHXZ 10008b25 f i pch.obj
 0001:00007b28       ??0MemoryPoolObj@@QAE@PBDI@Z 10008b28 f   memory:Memory.dll
 0001:00007b2e       ??1MemoryPoolObj@@QAE@XZ   10008b2e f   memory:Memory.dll
 0001:00007b34       ?MemPoolAlloc@@YGPAXPAU_HMEMPOOL@@I@Z 10008b34 f   memory:Memory.dll
 0001:00007b3a       ?MemPoolFree@@YGXPAU_HMEMPOOL@@PAX@Z 10008b3a f   memory:Memory.dll
 0001:00007b40       ??0FileStream@@QAE@XZ      10008b40 f   fileio:FileIO.dll
 0001:00007b46       ??1FileStream@@UAE@XZ      10008b46 f   fileio:FileIO.dll
 0001:00007b4c       ?Write@FileStream@@UAEKPBXK@Z 10008b4c f   fileio:FileIO.dll
 0001:00007b52       ?GetPos@FileStream@@UAEKXZ 10008b52 f   fileio:FileIO.dll
 0001:00007b58       ?GetLen@FileStream@@UAEKXZ 10008b58 f   fileio:FileIO.dll
 0001:00007b5e       ?Open@FileStream@@QAEJPBDW4StreamMode@@@Z 10008b5e f   fileio:FileIO.dll
 0001:00007b64       ?Close@FileStream@@QAEJXZ  10008b64 f   fileio:FileIO.dll
 0001:00007b6a       ?ReadLine@FileStream@@QAEKPADK@Z 10008b6a f   fileio:FileIO.dll
 0001:00007b70       ?Read@FileStream@@UAEKPAXK@Z 10008b70 f   fileio:FileIO.dll
 0001:00007b76       ?dbTracefAux@@YAXPBDZZ     10008b76 f   debug:Debug.dll
 0001:00007b7c       _GetLocalTime@4            10008b7c f   kernel32:KERNEL32.dll
 0001:00007b82       _GetVersionExA@4           10008b82 f   kernel32:KERNEL32.dll
 0001:00007b88       _GetDateFormatA@24         10008b88 f   kernel32:KERNEL32.dll
 0001:00007b8e       _GetTimeFormatA@24         10008b8e f   kernel32:KERNEL32.dll
 0001:00007b94       _CompareStringW@24         10008b94 f   kernel32:KERNEL32.dll
 0001:00007b9a       _MultiByteToWideChar@24    10008b9a f   kernel32:KERNEL32.dll
 0001:00007ba0       _WideCharToMultiByte@32    10008ba0 f   kernel32:KERNEL32.dll
 0001:00007ba6       _GetACP@0                  10008ba6 f   kernel32:KERNEL32.dll
 0001:00007bac       _CompareStringA@24         10008bac f   kernel32:KERNEL32.dll
 0001:00007bb2       _GetStringTypeA@20         10008bb2 f   kernel32:KERNEL32.dll
 0001:00007bb8       _InterlockedExchange@8     10008bb8 f   kernel32:KERNEL32.dll
 0001:00007bbe       _Sleep@4                   10008bbe f   kernel32:KERNEL32.dll
 0001:00007bc4       _CompareFileTime@8         10008bc4 f   kernel32:KERNEL32.dll
 0001:00007bca       _CreateFileA@28            10008bca f   kernel32:KERNEL32.dll
 0001:00007bd0       _FindClose@4               10008bd0 f   kernel32:KERNEL32.dll
 0001:00007bd6       _FindFirstFileA@8          10008bd6 f   kernel32:KERNEL32.dll
 0001:00007bdc       _FindNextFileA@8           10008bdc f   kernel32:KERNEL32.dll
 0001:00007be2       _GetFileTime@16            10008be2 f   kernel32:KERNEL32.dll
 0001:00007be8       _CloseHandle@4             10008be8 f   kernel32:KERNEL32.dll
 0001:00007bee       _CharNextA@4               10008bee f   user32:USER32.dll
 0001:00007bf4       ??_U@YAPAXI@Z              10008bf4 f   msvcprt:newaop_s.obj
 0001:00007bfe       ?_Orphan_all@_Container_base0@std@@QAEXXZ 10008bfe f   msvcprt:MSVCP110.dll
 0001:00007c04       ?_Xbad_alloc@std@@YAXXZ    10008c04 f   msvcprt:MSVCP110.dll
 0001:00007c0a       ?_Xlength_error@std@@YAXPBD@Z 10008c0a f   msvcprt:MSVCP110.dll
 0001:00007c10       ?_Xout_of_range@std@@YAXPBD@Z 10008c10 f   msvcprt:MSVCP110.dll
 0001:00007c16       ?_Swap_all@_Container_base0@std@@QAEXAAU12@@Z 10008c16 f   msvcprt:MSVCP110.dll
 0001:00007c1c       ??0id@locale@std@@QAE@I@Z  10008c1c f   msvcprt:MSVCP110.dll
 0001:00007c22       ?_Syserror_map@std@@YAPBDH@Z 10008c22 f   msvcprt:MSVCP110.dll
 0001:00007c28       ?_Winerror_map@std@@YAPBDH@Z 10008c28 f   msvcprt:MSVCP110.dll
 0001:00007c2e       ??_M@YGXPAXIHP6EX0@Z@Z     10008c2e f   MSVCRT:ehvecdtr.obj
 0001:00007cb6       ?__ArrayUnwind@@YGXPAXIHP6EX0@Z@Z 10008cb6 f   MSVCRT:ehvecdtr.obj
 0001:00007d14       __purecall                 10008d14 f   MSVCRT:MSVCR110.dll
 0001:00007d1a       ??2@YAPAXI@Z               10008d1a f   MSVCRT:MSVCR110.dll
 0001:00007d20       ??3@YAXPAX@Z               10008d20 f   MSVCRT:MSVCR110.dll
 0001:00007d26       _memcpy                    10008d26 f   MSVCRT:MSVCR110.dll
 0001:00007d2c       _wcstol                    10008d2c f   MSVCRT:MSVCR110.dll
 0001:00007d32       _strlen                    10008d32 f   MSVCRT:MSVCR110.dll
 0001:00007d38       _memmove                   10008d38 f   MSVCRT:MSVCR110.dll
 0001:00007d3e       _wcschr                    10008d3e f   MSVCRT:MSVCR110.dll
 0001:00007d44       _wcscmp                    10008d44 f   MSVCRT:MSVCR110.dll
 0001:00007d4a       _wcscpy                    10008d4a f   MSVCRT:MSVCR110.dll
 0001:00007d50       _wcslen                    10008d50 f   MSVCRT:MSVCR110.dll
 0001:00007d56       _wcsncpy                   10008d56 f   MSVCRT:MSVCR110.dll
 0001:00007d5c       ??_V@YAXPAX@Z              10008d5c f   MSVCRT:MSVCR110.dll
 0001:00007d62       __snwprintf                10008d62 f   MSVCRT:MSVCR110.dll
 0001:00007d68       __CxxThrowException@8      10008d68 f   MSVCRT:MSVCR110.dll
 0001:00007d70       __EH_prolog                10008d70 f   MSVCRT:ehprolog.obj
 0001:00007d90       ___CxxFrameHandler3        10008d90 f   MSVCRT:MSVCR110.dll
 0001:00007da0       __chkstk                   10008da0 f   MSVCRT:chkstk.obj
 0001:00007da0       __alloca_probe             10008da0     MSVCRT:chkstk.obj
 0001:00007dcc       _memset                    10008dcc f   MSVCRT:MSVCR110.dll
 0001:00007dd2       ??0type_info@@AAE@ABV0@@Z  10008dd2 f   MSVCRT:ti_inst.obj
 0001:00007ddd       ??4type_info@@AAEAAV0@ABV0@@Z 10008ddd f   MSVCRT:ti_inst.obj
 0001:00007de2       ??_Etype_info@@UAEPAXI@Z   10008de2 f i MSVCRT:ti_inst.obj
 0001:00007e2c       ___atonexitinit            10008e2c f   MSVCRT:atonexit.obj
 0001:00007e68       __onexit                   10008e68 f   MSVCRT:atonexit.obj
 0001:00007f0d       _atexit                    10008f0d f   MSVCRT:atonexit.obj
 0001:00007f22       __stricmp                  10008f22 f   MSVCRT:MSVCR110.dll
 0001:00007f28       ??0exception@std@@QAE@XZ   10008f28 f   MSVCRT:MSVCR110.dll
 0001:00007f2e       ??0exception@std@@QAE@ABV01@@Z 10008f2e f   MSVCRT:MSVCR110.dll
 0001:00007f34       ??1exception@std@@UAE@XZ   10008f34 f   MSVCRT:MSVCR110.dll
 0001:00007f3a       ??8type_info@@QBE_NABV0@@Z 10008f3a f   MSVCRT:MSVCR110.dll
 0001:00007f40       ___RTDynamicCast           10008f40 f   MSVCRT:MSVCR110.dll
 0001:00007f46       _strcpy                    10008f46 f   MSVCRT:MSVCR110.dll
 0001:00007f4c       _strncmp                   10008f4c f   MSVCRT:MSVCR110.dll
 0001:00007f52       _sscanf                    10008f52 f   MSVCRT:MSVCR110.dll
 0001:00007f58       __snscanf                  10008f58 f   MSVCRT:MSVCR110.dll
 0001:00007f5e       _sprintf                   10008f5e f   MSVCRT:MSVCR110.dll
 0001:00007f64       _wcsstr                    10008f64 f   MSVCRT:MSVCR110.dll
 0001:00007f6a       __snwscanf                 10008f6a f   MSVCRT:MSVCR110.dll
 0001:00007fbc       _NtCurrentTeb              10008fbc f i MSVCRT:crtdll.obj
 0001:00007fc3       __CRT_INIT@12              10008fc3 f   MSVCRT:crtdll.obj
 0001:000081b8       __DllMainCRTStartup@12     100091b8 f   MSVCRT:crtdll.obj
 0001:0000830e       ?terminate@@YAXXZ          1000930e f   MSVCRT:MSVCR110.dll
 0001:00008320       __SEH_prolog4              10009320 f   MSVCRT:sehprolg4.obj
 0001:00008365       __SEH_epilog4              10009365 f   MSVCRT:sehprolg4.obj
 0001:00008379       __except_handler4          10009379 f   MSVCRT:chandler4gs.obj
 0001:0000839c       ??1type_info@@UAE@XZ       1000939c f   MSVCRT:MSVCR110.dll
 0001:000083a2       __lock                     100093a2 f   MSVCRT:MSVCR110.dll
 0001:000083a8       __unlock                   100093a8 f   MSVCRT:MSVCR110.dll
 0001:000083ae       __calloc_crt               100093ae f   MSVCRT:MSVCR110.dll
 0001:000083b4       ___dllonexit               100093b4 f   MSVCRT:MSVCR110.dll
 0001:000083ba       ___CppXcptFilter           100093ba f   MSVCRT:MSVCR110.dll
 0001:000083c0       __amsg_exit                100093c0 f   MSVCRT:MSVCR110.dll
 0001:000083d0       __FindPESection            100093d0 f   MSVCRT:pesect.obj
 0001:00008420       __IsNonwritableInCurrentImage 10009420 f   MSVCRT:pesect.obj
 0001:000084e0       __ValidateImageBase        100094e0 f   MSVCRT:pesect.obj
 0001:00008512       _free                      10009512 f   MSVCRT:MSVCR110.dll
 0001:00008518       ___security_init_cookie    10009518 f   MSVCRT:gs_support.obj
 0001:000085b2       _DllMain@12                100095b2 f   MSVCRT:dllmain.obj
 0001:000085d4       __malloc_crt               100095d4 f   MSVCRT:MSVCR110.dll
 0001:000085da       __RTC_Initialize           100095da f   MSVCRT:initsect.obj
 0001:000085fa       __RTC_Terminate            100095fa f   MSVCRT:initsect.obj
 0001:0000861a       __initterm                 1000961a f   MSVCRT:MSVCR110.dll
 0001:00008620       __initterm_e               10009620 f   MSVCRT:MSVCR110.dll
 0001:00008626       ___clean_type_info_names   10009626 f   MSVCRT:tncleanup.obj
 0001:00008632       @__security_check_cookie@4 10009632 f   MSVCRT:secchk.obj
 0001:00008642       __except_handler4_common   10009642 f   MSVCRT:MSVCR110.dll
 0001:00008648       ___clean_type_info_names_internal 10009648 f   MSVCRT:MSVCR110.dll
 0001:0000864e       ___raise_securityfailure   1000964e f   MSVCRT:gs_report.obj
 0001:0000868b       ___report_gsfailure        1000968b f   MSVCRT:gs_report.obj
 0001:00008784       ___report_rangecheckfailure 10009784 f   MSVCRT:gs_report.obj
 0001:00008790       ___report_securityfailure  10009790 f   MSVCRT:gs_report.obj
 0001:0000885e       ___report_securityfailureEx 1000985e f   MSVCRT:gs_report.obj
 0001:00008972       __crt_debugger_hook        10009972 f   MSVCRT:MSVCR110.dll
 0001:00008978       ___crtUnhandledException   10009978 f   MSVCRT:MSVCR110.dll
 0001:0000897e       ___crtTerminateProcess     1000997e f   MSVCRT:MSVCR110.dll
 0001:00008984       _EncodePointer@4           10009984 f   kernel32:KERNEL32.dll
 0001:0000898a       _DecodePointer@4           1000998a f   kernel32:KERNEL32.dll
 0001:00008990       _QueryPerformanceCounter@4 10009990 f   kernel32:KERNEL32.dll
 0001:00008996       _GetCurrentProcessId@0     10009996 f   kernel32:KERNEL32.dll
 0001:0000899c       _GetCurrentThreadId@0      1000999c f   kernel32:KERNEL32.dll
 0001:000089a2       _GetSystemTimeAsFileTime@4 100099a2 f   kernel32:KERNEL32.dll
 0001:000089a8       _DisableThreadLibraryCalls@4 100099a8 f   kernel32:KERNEL32.dll
 0001:000089ae       _IsDebuggerPresent@0       100099ae f   kernel32:KERNEL32.dll
 0001:000089b4       _IsProcessorFeaturePresent@4 100099b4 f   kernel32:KERNEL32.dll
 0002:00000000       __imp_?dbTracefAux@@YAXPBDZZ 1000a000     debug:Debug.dll
 0002:00000004       \177Debug_NULL_THUNK_DATA  1000a004     debug:Debug.dll
 0002:00000008       __imp_?Read@FileStream@@UAEKPAXK@Z 1000a008     fileio:FileIO.dll
 0002:0000000c       __imp_?ReadLine@FileStream@@QAEKPADK@Z 1000a00c     fileio:FileIO.dll
 0002:00000010       __imp_??0FileStream@@QAE@XZ 1000a010     fileio:FileIO.dll
 0002:00000014       __imp_??1FileStream@@UAE@XZ 1000a014     fileio:FileIO.dll
 0002:00000018       __imp_?Write@FileStream@@UAEKPBXK@Z 1000a018     fileio:FileIO.dll
 0002:0000001c       __imp_?GetPos@FileStream@@UAEKXZ 1000a01c     fileio:FileIO.dll
 0002:00000020       __imp_?GetLen@FileStream@@UAEKXZ 1000a020     fileio:FileIO.dll
 0002:00000024       __imp_?Open@FileStream@@QAEJPBDW4StreamMode@@@Z 1000a024     fileio:FileIO.dll
 0002:00000028       __imp_?Close@FileStream@@QAEJXZ 1000a028     fileio:FileIO.dll
 0002:0000002c       \177FileIO_NULL_THUNK_DATA 1000a02c     fileio:FileIO.dll
 0002:00000030       __imp__GetSystemTimeAsFileTime@4 1000a030     kernel32:KERNEL32.dll
 0002:00000034       __imp__DisableThreadLibraryCalls@4 1000a034     kernel32:KERNEL32.dll
 0002:00000038       __imp__IsDebuggerPresent@0 1000a038     kernel32:KERNEL32.dll
 0002:0000003c       __imp__IsProcessorFeaturePresent@4 1000a03c     kernel32:KERNEL32.dll
 0002:00000040       __imp__GetCurrentThreadId@0 1000a040     kernel32:KERNEL32.dll
 0002:00000044       __imp__GetLocalTime@4      1000a044     kernel32:KERNEL32.dll
 0002:00000048       __imp__GetVersionExA@4     1000a048     kernel32:KERNEL32.dll
 0002:0000004c       __imp__GetDateFormatA@24   1000a04c     kernel32:KERNEL32.dll
 0002:00000050       __imp__GetTimeFormatA@24   1000a050     kernel32:KERNEL32.dll
 0002:00000054       __imp__CompareStringW@24   1000a054     kernel32:KERNEL32.dll
 0002:00000058       __imp__MultiByteToWideChar@24 1000a058     kernel32:KERNEL32.dll
 0002:0000005c       __imp__WideCharToMultiByte@32 1000a05c     kernel32:KERNEL32.dll
 0002:00000060       __imp__GetACP@0            1000a060     kernel32:KERNEL32.dll
 0002:00000064       __imp__CompareStringA@24   1000a064     kernel32:KERNEL32.dll
 0002:00000068       __imp__GetStringTypeA@20   1000a068     kernel32:KERNEL32.dll
 0002:0000006c       __imp__InterlockedExchange@8 1000a06c     kernel32:KERNEL32.dll
 0002:00000070       __imp__Sleep@4             1000a070     kernel32:KERNEL32.dll
 0002:00000074       __imp__CompareFileTime@8   1000a074     kernel32:KERNEL32.dll
 0002:00000078       __imp__CreateFileA@28      1000a078     kernel32:KERNEL32.dll
 0002:0000007c       __imp__FindClose@4         1000a07c     kernel32:KERNEL32.dll
 0002:00000080       __imp__FindFirstFileA@8    1000a080     kernel32:KERNEL32.dll
 0002:00000084       __imp__FindNextFileA@8     1000a084     kernel32:KERNEL32.dll
 0002:00000088       __imp__GetFileTime@16      1000a088     kernel32:KERNEL32.dll
 0002:0000008c       __imp__CloseHandle@4       1000a08c     kernel32:KERNEL32.dll
 0002:00000090       __imp__GetCurrentProcessId@0 1000a090     kernel32:KERNEL32.dll
 0002:00000094       __imp__QueryPerformanceCounter@4 1000a094     kernel32:KERNEL32.dll
 0002:00000098       __imp__EncodePointer@4     1000a098     kernel32:KERNEL32.dll
 0002:0000009c       __imp__DecodePointer@4     1000a09c     kernel32:KERNEL32.dll
 0002:000000a0       \177KERNEL32_NULL_THUNK_DATA 1000a0a0     kernel32:KERNEL32.dll
 0002:000000a4       __imp_?_Xlength_error@std@@YAXPBD@Z 1000a0a4     msvcprt:MSVCP110.dll
 0002:000000a8       __imp_?_Xout_of_range@std@@YAXPBD@Z 1000a0a8     msvcprt:MSVCP110.dll
 0002:000000ac       __imp_?_Swap_all@_Container_base0@std@@QAEXAAU12@@Z 1000a0ac     msvcprt:MSVCP110.dll
 0002:000000b0       __imp_??0id@locale@std@@QAE@I@Z 1000a0b0     msvcprt:MSVCP110.dll
 0002:000000b4       __imp_?_Syserror_map@std@@YAPBDH@Z 1000a0b4     msvcprt:MSVCP110.dll
 0002:000000b8       __imp_?_Winerror_map@std@@YAPBDH@Z 1000a0b8     msvcprt:MSVCP110.dll
 0002:000000bc       __imp_?_Orphan_all@_Container_base0@std@@QAEXXZ 1000a0bc     msvcprt:MSVCP110.dll
 0002:000000c0       __imp_?_Xbad_alloc@std@@YAXXZ 1000a0c0     msvcprt:MSVCP110.dll
 0002:000000c4       \177MSVCP110_NULL_THUNK_DATA 1000a0c4     msvcprt:MSVCP110.dll
 0002:000000c8       __imp_??3@YAXPAX@Z         1000a0c8     MSVCRT:MSVCR110.dll
 0002:000000cc       __imp__memcpy              1000a0cc     MSVCRT:MSVCR110.dll
 0002:000000d0       __imp__wcstol              1000a0d0     MSVCRT:MSVCR110.dll
 0002:000000d4       __imp__strlen              1000a0d4     MSVCRT:MSVCR110.dll
 0002:000000d8       __imp__memmove             1000a0d8     MSVCRT:MSVCR110.dll
 0002:000000dc       __imp__wcschr              1000a0dc     MSVCRT:MSVCR110.dll
 0002:000000e0       __imp__wcscmp              1000a0e0     MSVCRT:MSVCR110.dll
 0002:000000e4       __imp__wcscpy              1000a0e4     MSVCRT:MSVCR110.dll
 0002:000000e8       __imp__wcslen              1000a0e8     MSVCRT:MSVCR110.dll
 0002:000000ec       __imp__wcsncpy             1000a0ec     MSVCRT:MSVCR110.dll
 0002:000000f0       __imp_??_V@YAXPAX@Z        1000a0f0     MSVCRT:MSVCR110.dll
 0002:000000f4       __imp___snwprintf          1000a0f4     MSVCRT:MSVCR110.dll
 0002:000000f8       __imp___CxxThrowException@8 1000a0f8     MSVCRT:MSVCR110.dll
 0002:000000fc       __imp____CxxFrameHandler3  1000a0fc     MSVCRT:MSVCR110.dll
 0002:00000100       __imp__memset              1000a100     MSVCRT:MSVCR110.dll
 0002:00000104       __imp___stricmp            1000a104     MSVCRT:MSVCR110.dll
 0002:00000108       __imp_??0exception@std@@QAE@XZ 1000a108     MSVCRT:MSVCR110.dll
 0002:0000010c       __imp_??0exception@std@@QAE@ABV01@@Z 1000a10c     MSVCRT:MSVCR110.dll
 0002:00000110       __imp_??1exception@std@@UAE@XZ 1000a110     MSVCRT:MSVCR110.dll
 0002:00000114       __imp___purecall           1000a114     MSVCRT:MSVCR110.dll
 0002:00000118       __imp____RTDynamicCast     1000a118     MSVCRT:MSVCR110.dll
 0002:0000011c       __imp__strcpy              1000a11c     MSVCRT:MSVCR110.dll
 0002:00000120       __imp__strncmp             1000a120     MSVCRT:MSVCR110.dll
 0002:00000124       __imp__sscanf              1000a124     MSVCRT:MSVCR110.dll
 0002:00000128       __imp___snscanf            1000a128     MSVCRT:MSVCR110.dll
 0002:0000012c       __imp__sprintf             1000a12c     MSVCRT:MSVCR110.dll
 0002:00000130       __imp__wcsstr              1000a130     MSVCRT:MSVCR110.dll
 0002:00000134       __imp___snwscanf           1000a134     MSVCRT:MSVCR110.dll
 0002:00000138       __imp_?terminate@@YAXXZ    1000a138     MSVCRT:MSVCR110.dll
 0002:0000013c       __imp_??1type_info@@UAE@XZ 1000a13c     MSVCRT:MSVCR110.dll
 0002:00000140       __imp___lock               1000a140     MSVCRT:MSVCR110.dll
 0002:00000144       __imp___unlock             1000a144     MSVCRT:MSVCR110.dll
 0002:00000148       __imp___calloc_crt         1000a148     MSVCRT:MSVCR110.dll
 0002:0000014c       __imp____dllonexit         1000a14c     MSVCRT:MSVCR110.dll
 0002:00000150       __imp___onexit             1000a150     MSVCRT:MSVCR110.dll
 0002:00000154       __imp____CppXcptFilter     1000a154     MSVCRT:MSVCR110.dll
 0002:00000158       __imp___amsg_exit          1000a158     MSVCRT:MSVCR110.dll
 0002:0000015c       __imp__free                1000a15c     MSVCRT:MSVCR110.dll
 0002:00000160       __imp___malloc_crt         1000a160     MSVCRT:MSVCR110.dll
 0002:00000164       __imp___initterm           1000a164     MSVCRT:MSVCR110.dll
 0002:00000168       __imp___initterm_e         1000a168     MSVCRT:MSVCR110.dll
 0002:0000016c       __imp___except_handler4_common 1000a16c     MSVCRT:MSVCR110.dll
 0002:00000170       __imp____clean_type_info_names_internal 1000a170     MSVCRT:MSVCR110.dll
 0002:00000174       __imp___crt_debugger_hook  1000a174     MSVCRT:MSVCR110.dll
 0002:00000178       __imp____crtUnhandledException 1000a178     MSVCRT:MSVCR110.dll
 0002:0000017c       __imp____crtTerminateProcess 1000a17c     MSVCRT:MSVCR110.dll
 0002:00000180       __imp_??8type_info@@QBE_NABV0@@Z 1000a180     MSVCRT:MSVCR110.dll
 0002:00000184       __imp_??2@YAPAXI@Z         1000a184     MSVCRT:MSVCR110.dll
 0002:00000188       \177MSVCR110_NULL_THUNK_DATA 1000a188     MSVCRT:MSVCR110.dll
 0002:0000018c       __imp_??1MemoryPoolObj@@QAE@XZ 1000a18c     memory:Memory.dll
 0002:00000190       __imp_?MemPoolFree@@YGXPAU_HMEMPOOL@@PAX@Z 1000a190     memory:Memory.dll
 0002:00000194       __imp_?MemPoolAlloc@@YGPAXPAU_HMEMPOOL@@I@Z 1000a194     memory:Memory.dll
 0002:00000198       __imp_??0MemoryPoolObj@@QAE@PBDI@Z 1000a198     memory:Memory.dll
 0002:0000019c       \177Memory_NULL_THUNK_DATA 1000a19c     memory:Memory.dll
 0002:000001a0       __imp__CharNextA@4         1000a1a0     user32:USER32.dll
 0002:000001a4       \177USER32_NULL_THUNK_DATA 1000a1a4     user32:USER32.dll
 0002:000001a8       ___xc_a                    1000a1a8     MSVCRT:cinitexe.obj
 0002:000001c0       ___xc_z                    1000a1c0     MSVCRT:cinitexe.obj
 0002:000001c4       ___xi_a                    1000a1c4     MSVCRT:cinitexe.obj
 0002:000001d0       ___xi_z                    1000a1d0     MSVCRT:cinitexe.obj
 0002:00000218       ??_C@_15KNBIKKIN@?$AA?$CF?$AAd?$AA?$AA@ 1000a218     Localizer.obj
 0002:00000220       ??_C@_0BI@CFPLBAOH@invalid?5string?5position?$AA@ 1000a220     Localizer.obj
 0002:00000238       ??_C@_0BA@JFNIOLAK@string?5too?5long?$AA@ 1000a238     Localizer.obj
 0002:0000024c       ??_7Resource@LocalizerImp@@6B@ 1000a24c     Localizer.obj
 0002:00000260       ??_C@_17EMELIOL@?$AA$?$AA?$CF?$AAd?$AA?$AA@ 1000a260     Localizer.obj
 0002:00000268       ??_C@_17PGKOGADG@?$AA$?$AA?$CF?$AAi?$AA?$AA@ 1000a268     Localizer.obj
 0002:00000274       ??_7bad_weak_ptr@boost@@6B@ 1000a274     LocalizerImp.obj
 0002:0000027c       ??_C@_0BE@GLILEGNA@boost?3?3bad_weak_ptr?$AA@ 1000a27c     LocalizerImp.obj
 0002:00000294       ??_7sp_counted_base@detail@boost@@6B@ 1000a294     LocalizerImp.obj
 0002:000002a4       ??_C@_02KHDDNBB@?2?$CK?$AA@ 1000a2a4     LocalizerImp.obj
 0002:000002a8       ??_C@_09NEAPFGIB@Localizer?$AA@ 1000a2a8     LocalizerImp.obj
 0002:000002b4       ??_C@_0DK@FKDLBNFG@LOCALIZER?5?9?9?5Failed?5to?5load?5file@ 1000a2b4     LocalizerImp.obj
 0002:000002f0       ??_C@_0EF@CPMBJHNI@LOCALIZER?5?9?9?5Failed?5to?5load?5file@ 1000a2f0     LocalizerImp.obj
 0002:00000338       ??_C@_0DI@LPJFJOCM@LOCALIZER?5?9?9?5Requested?5string?5ra@ 1000a338     LocalizerImp.obj
 0002:00000370       ??_C@_0BD@OLBABOEK@vector?$DMT?$DO?5too?5long?$AA@ 1000a370     LocalizerImp.obj
 0002:00000388       ??_7?$sp_counted_base_impl@PAVResource@LocalizerImp@@U?$checked_deleter@VResource@LocalizerImp@@@boost@@@detail@boost@@6B@ 1000a388     LocalizerImp.obj
 0002:00000398       ??_C@_04PBCOOEDG@?4dat?$AA@ 1000a398     LocalizerTxt.obj
 0002:000003c7       ??_C@_00CNPNBAHC@?$AA@     1000a3c7     LocalizerTxt.obj
 0002:000003c8       ??_C@_02GMHACPFF@?$CFu?$AA@ 1000a3c8     LocalizerTxt.obj
 0002:000003d0       ??_7LocalizerResourceTxt@@6B@ 1000a3d0     LocalizerTxt.obj
 0002:000003e4       ??_C@_0BA@KFGLKMOM@filerange?5?$CFd?5?$CFd?$AA@ 1000a3e4     LocalizerTxt.obj
 0002:000003f4       ??_C@_0BB@PKDOMNNC@rangestart?5?$CFd?5?$CFd?$AA@ 1000a3f4     LocalizerTxt.obj
 0002:00000408       ??_C@_0CM@EEMHJDAE@LOCALIZER?5?9?9?5Parsing?5error?5on?5li@ 1000a408     LocalizerTxt.obj
 0002:00000434       ??_C@_01EEMJAFIK@?6?$AA@   1000a434     LocalizerTxt.obj
 0002:00000438       ??_C@_0CM@IEKELENB@LOCALIZER?5?9?9?5Duplicate?5string?5li@ 1000a438     LocalizerTxt.obj
 0002:00000464       ??_C@_0CP@ENCALGHF@LOCALIZER?5?9?9?5String?5out?5of?5range@ 1000a464     LocalizerTxt.obj
 0002:00000494       ??_C@_0CP@JPLHEIDJ@LOCALIZER?5?9?9?5Unexpected?5error?5on@ 1000a494     LocalizerTxt.obj
 0002:000004c4       ??_C@_0DC@POLICJFP@LOCALIZER?5?9?9?5Duplicate?5filerange@ 1000a4c4     LocalizerTxt.obj
 0002:000004f8       ??_C@_0DA@JJILFKME@LOCALIZER?5?9?9?5Invalid?5filerange?5a@ 1000a4f8     LocalizerTxt.obj
 0002:00000528       ??_C@_0DA@DGIIHOG@LOCALIZER?5?9?9?5Missing?5filerange?5a@ 1000a528     LocalizerTxt.obj
 0002:00000558       ??_C@_0CM@GEDFBKPK@LOCALIZER?5?9?9?5Invalid?5range?5at?5li@ 1000a558     LocalizerTxt.obj
 0002:00000584       ??_C@_0DJ@CIBCIKBE@LOCALIZER?5?9?9?5Range?5outside?5of?5fi@ 1000a584     LocalizerTxt.obj
 0002:000005c0       ??_C@_0CO@LOPBCOHK@LOCALIZER?5?9?9?5Colliding?5range?5at?5@ 1000a5c0     LocalizerTxt.obj
 0002:000005f0       ??_C@_0CL@IDFONOGB@LOCALIZER?5?9?9?5Missing?5final?5range@ 1000a5f0     LocalizerTxt.obj
 0002:0000061c       ??_C@_0CO@DKJKHGGK@LOCALIZER?5?9?9?5File?5is?5missing?5fil@ 1000a61c     LocalizerTxt.obj
 0002:0000064c       ??_C@_11LOCGONAA@?$AA?$AA@ 1000a64c     LocalizerTxt.obj
 0002:00000650       ??_C@_0N@HAGGIOCE@?$CFs?$CFs?5?$CFi?5?$CFi?$AN?6?$AA@ 1000a650     LocalizerTxt.obj
 0002:00000660       ??_C@_08HHJFPBJJ@?$CFs?$CFi?7?$CFs?6?$AA@ 1000a660     LocalizerTxt.obj
 0002:0000066c       ??_C@_03OFAPEBGM@?$CFs?6?$AA@ 1000a66c     LocalizerTxt.obj
 0002:00000670       ??_C@_04FFEOJGGF@?4ucs?$AA@ 1000a670     LocalizerUCS.obj
 0002:00000678       ??_C@_15EFLNJKHH@?$AA?$CF?$AAu?$AA?$AA@ 1000a678     LocalizerUCS.obj
 0002:00000684       ??_7LocalizerResourceUCS@@6B@ 1000a684     LocalizerUCS.obj
 0002:00000698       ??_C@_15JNBOKNOG@?$AA?$AN?$AA?6?$AA?$AA@ 1000a698     LocalizerUCS.obj
 0002:0000069e       ?is_signed@?$numeric_limits@E@std@@2_NB 1000a69e     pch.obj
 0002:000006a0       ?digits@?$numeric_limits@E@std@@2HB 1000a6a0     pch.obj
 0002:000006a4       ?digits10@?$numeric_limits@E@std@@2HB 1000a6a4     pch.obj
 0002:000006a8       ?is_signed@?$numeric_limits@F@std@@2_NB 1000a6a8     pch.obj
 0002:000006ac       ?digits@?$numeric_limits@F@std@@2HB 1000a6ac     pch.obj
 0002:000006b0       ?digits10@?$numeric_limits@F@std@@2HB 1000a6b0     pch.obj
 0002:000006b4       ?value@?$integral_constant@I$0A@@std@@2IB 1000a6b4     pch.obj
 0002:000006b8       ?is_signed@?$numeric_limits@G@std@@2_NB 1000a6b8     pch.obj
 0002:000006bc       ?digits@?$numeric_limits@G@std@@2HB 1000a6bc     pch.obj
 0002:000006c0       ?digits10@?$numeric_limits@G@std@@2HB 1000a6c0     pch.obj
 0002:000006c4       ?value@?$ice_and@$00$00$00$00$00$00$00@type_traits@boost@@2_NB 1000a6c4     pch.obj
 0002:000006c5       ?is_signed@?$numeric_limits@H@std@@2_NB 1000a6c5     pch.obj
 0002:000006c8       ?digits@?$numeric_limits@H@std@@2HB 1000a6c8     pch.obj
 0002:000006cc       ?collate@?$_Locbase@H@std@@2HB 1000a6cc     pch.obj
 0002:000006d0       ?ctype@?$_Locbase@H@std@@2HB 1000a6d0     pch.obj
 0002:000006d4       ?digits10@?$numeric_limits@H@std@@2HB 1000a6d4     pch.obj
 0002:000006d8       ?monetary@?$_Locbase@H@std@@2HB 1000a6d8     pch.obj
 0002:000006dc       ?numeric@?$_Locbase@H@std@@2HB 1000a6dc     pch.obj
 0002:000006e0       ?value@?$ice_not@$00@type_traits@boost@@2_NB 1000a6e0     pch.obj
 0002:000006e4       ?time@?$_Locbase@H@std@@2HB 1000a6e4     pch.obj
 0002:000006e8       ?messages@?$_Locbase@H@std@@2HB 1000a6e8     pch.obj
 0002:000006ec       ?all@?$_Locbase@H@std@@2HB 1000a6ec     pch.obj
 0002:000006f0       ?none@?$_Locbase@H@std@@2HB 1000a6f0     pch.obj
 0002:000006f4       ?is_signed@?$numeric_limits@I@std@@2_NB 1000a6f4     pch.obj
 0002:000006f8       ?digits@?$numeric_limits@I@std@@2HB 1000a6f8     pch.obj
 0002:000006fc       ?digits10@?$numeric_limits@I@std@@2HB 1000a6fc     pch.obj
 0002:00000700       ?value@?$is_convertible_impl@XX@detail@boost@@2_NB 1000a700     pch.obj
 0002:00000701       ?is_signed@?$numeric_limits@J@std@@2_NB 1000a701     pch.obj
 0002:00000702       ?value@?$is_convertible_impl@X$$CBX@detail@boost@@2_NB 1000a702     pch.obj
 0002:00000704       ?digits@?$numeric_limits@J@std@@2HB 1000a704     pch.obj
 0002:00000708       ?digits10@?$numeric_limits@J@std@@2HB 1000a708     pch.obj
 0002:0000070c       ?value@?$is_convertible_impl@X$$CCX@detail@boost@@2_NB 1000a70c     pch.obj
 0002:0000070d       ?value@?$is_convertible_impl@X$$CDX@detail@boost@@2_NB 1000a70d     pch.obj
 0002:00000710       ?value@?$_Sizeof@U_Nil@std@@U12@U12@U12@U12@U12@U12@U12@@std@@2IB 1000a710     pch.obj
 0002:00000714       ?value@?$is_convertible_impl@$$CBXX@detail@boost@@2_NB 1000a714     pch.obj
 0002:00000715       ?is_signed@?$numeric_limits@K@std@@2_NB 1000a715     pch.obj
 0002:00000718       ?digits@?$numeric_limits@K@std@@2HB 1000a718     pch.obj
 0002:0000071c       ?value@?$is_convertible_impl@$$CBX$$CBX@detail@boost@@2_NB 1000a71c     pch.obj
 0002:00000720       ?digits10@?$numeric_limits@K@std@@2HB 1000a720     pch.obj
 0002:00000724       ?value@?$is_convertible_impl@$$CBX$$CCX@detail@boost@@2_NB 1000a724     pch.obj
 0002:00000725       ?value@?$is_convertible_impl@$$CBX$$CDX@detail@boost@@2_NB 1000a725     pch.obj
 0002:00000726       ?is_signed@?$numeric_limits@_J@std@@2_NB 1000a726     pch.obj
 0002:00000727       ?value@?$is_convertible_impl@$$CCXX@detail@boost@@2_NB 1000a727     pch.obj
 0002:00000728       ?digits@?$numeric_limits@_J@std@@2HB 1000a728     pch.obj
 0002:0000072c       ?digits10@?$numeric_limits@_J@std@@2HB 1000a72c     pch.obj
 0002:00000730       ?value@?$is_convertible_impl@$$CCX$$CBX@detail@boost@@2_NB 1000a730     pch.obj
 0002:00000731       ?value@?$is_convertible_impl@$$CCX$$CCX@detail@boost@@2_NB 1000a731     pch.obj
 0002:00000732       ?value@?$is_convertible_impl@$$CCX$$CDX@detail@boost@@2_NB 1000a732     pch.obj
 0002:00000733       ?is_signed@?$numeric_limits@_K@std@@2_NB 1000a733     pch.obj
 0002:00000734       ?digits@?$numeric_limits@_K@std@@2HB 1000a734     pch.obj
 0002:00000738       ?digits10@?$numeric_limits@_K@std@@2HB 1000a738     pch.obj
 0002:0000073c       ?value@?$is_convertible_impl@$$CDXX@detail@boost@@2_NB 1000a73c     pch.obj
 0002:0000073d       ?value@?$is_convertible_impl@$$CDX$$CBX@detail@boost@@2_NB 1000a73d     pch.obj
 0002:0000073e       ?value@?$integral_constant@_N$0A@@std@@2_NB 1000a73e     pch.obj
 0002:0000073f       ?value@?$is_convertible_impl@$$CDX$$CCX@detail@boost@@2_NB 1000a73f     pch.obj
 0002:00000740       ?digits@?$numeric_limits@M@std@@2HB 1000a740     pch.obj
 0002:00000744       ?value@?$integral_constant@_N$00@std@@2_NB 1000a744     pch.obj
 0002:00000748       ?digits10@?$numeric_limits@M@std@@2HB 1000a748     pch.obj
 0002:0000074c       ?value@?$is_convertible_impl@$$CDX$$CDX@detail@boost@@2_NB 1000a74c     pch.obj
 0002:00000750       ?max_digits10@?$numeric_limits@M@std@@2HB 1000a750     pch.obj
 0002:00000754       ?max_exponent@?$numeric_limits@M@std@@2HB 1000a754     pch.obj
 0002:00000758       ?max_exponent10@?$numeric_limits@M@std@@2HB 1000a758     pch.obj
 0002:0000075c       ?min_exponent@?$numeric_limits@M@std@@2HB 1000a75c     pch.obj
 0002:00000760       ?min_exponent10@?$numeric_limits@M@std@@2HB 1000a760     pch.obj
 0002:00000764       ?digits@?$numeric_limits@N@std@@2HB 1000a764     pch.obj
 0002:00000768       ?digits10@?$numeric_limits@N@std@@2HB 1000a768     pch.obj
 0002:0000076c       ?max_digits10@?$numeric_limits@N@std@@2HB 1000a76c     pch.obj
 0002:00000770       ?max_exponent@?$numeric_limits@N@std@@2HB 1000a770     pch.obj
 0002:00000774       ?max_exponent10@?$numeric_limits@N@std@@2HB 1000a774     pch.obj
 0002:00000778       ?value@?$bool_@$0A@@mpl@boost@@2_NB 1000a778     pch.obj
 0002:0000077c       ?min_exponent@?$numeric_limits@N@std@@2HB 1000a77c     pch.obj
 0002:00000780       ?min_exponent10@?$numeric_limits@N@std@@2HB 1000a780     pch.obj
 0002:00000784       ?value@?$bool_@$00@mpl@boost@@2_NB 1000a784     pch.obj
 0002:00000788       ?digits@?$numeric_limits@O@std@@2HB 1000a788     pch.obj
 0002:0000078c       ?digits10@?$numeric_limits@O@std@@2HB 1000a78c     pch.obj
 0002:00000790       ?max_digits10@?$numeric_limits@O@std@@2HB 1000a790     pch.obj
 0002:00000794       ?max_exponent@?$numeric_limits@O@std@@2HB 1000a794     pch.obj
 0002:00000798       ?max_exponent10@?$numeric_limits@O@std@@2HB 1000a798     pch.obj
 0002:0000079c       ?min_exponent@?$numeric_limits@O@std@@2HB 1000a79c     pch.obj
 0002:000007a0       ?min_exponent10@?$numeric_limits@O@std@@2HB 1000a7a0     pch.obj
 0002:000007a4       ?value@?$is_enum_impl@M@detail@boost@@2_NB 1000a7a4     pch.obj
 0002:000007a5       ?value@?$is_enum_impl@N@detail@boost@@2_NB 1000a7a5     pch.obj
 0002:000007a6       ?value@?$is_enum_impl@O@detail@boost@@2_NB 1000a7a6     pch.obj
 0002:000007a7       ?value@?$is_enum_impl@X@detail@boost@@2_NB 1000a7a7     pch.obj
 0002:000007a8       ?value@?$is_enum_impl@$$CBX@detail@boost@@2_NB 1000a7a8     pch.obj
 0002:000007a9       ?value@?$is_enum_impl@$$CCX@detail@boost@@2_NB 1000a7a9     pch.obj
 0002:000007aa       ?value@?$is_enum_impl@$$CDX@detail@boost@@2_NB 1000a7aa     pch.obj
 0002:000007ac       ?has_denorm@_Num_base@std@@2W4float_denorm_style@2@B 1000a7ac     pch.obj
 0002:000007b0       ?has_denorm_loss@_Num_base@std@@2_NB 1000a7b0     pch.obj
 0002:000007b1       ?has_infinity@_Num_base@std@@2_NB 1000a7b1     pch.obj
 0002:000007b2       ?has_quiet_NaN@_Num_base@std@@2_NB 1000a7b2     pch.obj
 0002:000007b3       ?has_signaling_NaN@_Num_base@std@@2_NB 1000a7b3     pch.obj
 0002:000007b4       ?is_bounded@_Num_base@std@@2_NB 1000a7b4     pch.obj
 0002:000007b5       ?is_exact@_Num_base@std@@2_NB 1000a7b5     pch.obj
 0002:000007b6       ?is_iec559@_Num_base@std@@2_NB 1000a7b6     pch.obj
 0002:000007b7       ?is_integer@_Num_base@std@@2_NB 1000a7b7     pch.obj
 0002:000007b8       ?value@?$integral_constant@H$0A@@std@@2HB 1000a7b8     pch.obj
 0002:000007bc       ?is_modulo@_Num_base@std@@2_NB 1000a7bc     pch.obj
 0002:000007bd       ?is_signed@_Num_base@std@@2_NB 1000a7bd     pch.obj
 0002:000007be       ?is_specialized@_Num_base@std@@2_NB 1000a7be     pch.obj
 0002:000007bf       ?tinyness_before@_Num_base@std@@2_NB 1000a7bf     pch.obj
 0002:000007c0       ?traps@_Num_base@std@@2_NB 1000a7c0     pch.obj
 0002:000007c4       ?round_style@_Num_base@std@@2W4float_round_style@2@B 1000a7c4     pch.obj
 0002:000007c8       ?digits@_Num_base@std@@2HB 1000a7c8     pch.obj
 0002:000007cc       ?digits10@_Num_base@std@@2HB 1000a7cc     pch.obj
 0002:000007d0       ?max_digits10@_Num_base@std@@2HB 1000a7d0     pch.obj
 0002:000007d4       ?max_exponent@_Num_base@std@@2HB 1000a7d4     pch.obj
 0002:000007d8       ?max_exponent10@_Num_base@std@@2HB 1000a7d8     pch.obj
 0002:000007dc       ?min_exponent@_Num_base@std@@2HB 1000a7dc     pch.obj
 0002:000007e0       ?min_exponent10@_Num_base@std@@2HB 1000a7e0     pch.obj
 0002:000007e4       ?radix@_Num_base@std@@2HB  1000a7e4     pch.obj
 0002:000007e8       ?is_bounded@_Num_int_base@std@@2_NB 1000a7e8     pch.obj
 0002:000007e9       ?is_exact@_Num_int_base@std@@2_NB 1000a7e9     pch.obj
 0002:000007ea       ?is_integer@_Num_int_base@std@@2_NB 1000a7ea     pch.obj
 0002:000007eb       ?is_modulo@_Num_int_base@std@@2_NB 1000a7eb     pch.obj
 0002:000007ec       ?is_specialized@_Num_int_base@std@@2_NB 1000a7ec     pch.obj
 0002:000007f0       ?radix@_Num_int_base@std@@2HB 1000a7f0     pch.obj
 0002:000007f4       ?value@?$_Sizeof@HU_Nil@std@@U12@U12@U12@U12@U12@U12@@std@@2IB 1000a7f4     pch.obj
 0002:000007f8       ?has_denorm@_Num_float_base@std@@2W4float_denorm_style@2@B 1000a7f8     pch.obj
 0002:000007fc       ?has_denorm_loss@_Num_float_base@std@@2_NB 1000a7fc     pch.obj
 0002:000007fd       ?has_infinity@_Num_float_base@std@@2_NB 1000a7fd     pch.obj
 0002:000007fe       ?has_quiet_NaN@_Num_float_base@std@@2_NB 1000a7fe     pch.obj
 0002:00000800       ?skipws@?$_Iosb@H@std@@2W4_Fmtflags@12@B 1000a800     pch.obj
 0002:00000804       ?has_signaling_NaN@_Num_float_base@std@@2_NB 1000a804     pch.obj
 0002:00000808       ?unitbuf@?$_Iosb@H@std@@2W4_Fmtflags@12@B 1000a808     pch.obj
 0002:0000080c       ?is_bounded@_Num_float_base@std@@2_NB 1000a80c     pch.obj
 0002:00000810       ?uppercase@?$_Iosb@H@std@@2W4_Fmtflags@12@B 1000a810     pch.obj
 0002:00000814       ?is_exact@_Num_float_base@std@@2_NB 1000a814     pch.obj
 0002:00000818       ?showbase@?$_Iosb@H@std@@2W4_Fmtflags@12@B 1000a818     pch.obj
 0002:0000081c       ?is_iec559@_Num_float_base@std@@2_NB 1000a81c     pch.obj
 0002:00000820       ?showpoint@?$_Iosb@H@std@@2W4_Fmtflags@12@B 1000a820     pch.obj
 0002:00000824       ?is_integer@_Num_float_base@std@@2_NB 1000a824     pch.obj
 0002:00000828       ?showpos@?$_Iosb@H@std@@2W4_Fmtflags@12@B 1000a828     pch.obj
 0002:0000082c       ?is_modulo@_Num_float_base@std@@2_NB 1000a82c     pch.obj
 0002:00000830       ?left@?$_Iosb@H@std@@2W4_Fmtflags@12@B 1000a830     pch.obj
 0002:00000834       ?is_signed@_Num_float_base@std@@2_NB 1000a834     pch.obj
 0002:00000838       ?right@?$_Iosb@H@std@@2W4_Fmtflags@12@B 1000a838     pch.obj
 0002:0000083c       ?is_specialized@_Num_float_base@std@@2_NB 1000a83c     pch.obj
 0002:00000840       ?internal@?$_Iosb@H@std@@2W4_Fmtflags@12@B 1000a840     pch.obj
 0002:00000844       ?tinyness_before@_Num_float_base@std@@2_NB 1000a844     pch.obj
 0002:00000848       ?dec@?$_Iosb@H@std@@2W4_Fmtflags@12@B 1000a848     pch.obj
 0002:0000084c       ?traps@_Num_float_base@std@@2_NB 1000a84c     pch.obj
 0002:00000850       ?oct@?$_Iosb@H@std@@2W4_Fmtflags@12@B 1000a850     pch.obj
 0002:00000854       ?round_style@_Num_float_base@std@@2W4float_round_style@2@B 1000a854     pch.obj
 0002:00000858       ?hex@?$_Iosb@H@std@@2W4_Fmtflags@12@B 1000a858     pch.obj
 0002:0000085c       ?radix@_Num_float_base@std@@2HB 1000a85c     pch.obj
 0002:00000860       ?scientific@?$_Iosb@H@std@@2W4_Fmtflags@12@B 1000a860     pch.obj
 0002:00000864       ?fixed@?$_Iosb@H@std@@2W4_Fmtflags@12@B 1000a864     pch.obj
 0002:00000868       ?hexfloat@?$_Iosb@H@std@@2W4_Fmtflags@12@B 1000a868     pch.obj
 0002:0000086c       ?boolalpha@?$_Iosb@H@std@@2W4_Fmtflags@12@B 1000a86c     pch.obj
 0002:00000870       ?_Stdio@?$_Iosb@H@std@@2W4_Fmtflags@12@B 1000a870     pch.obj
 0002:00000874       ?adjustfield@?$_Iosb@H@std@@2W4_Fmtflags@12@B 1000a874     pch.obj
 0002:00000878       ?basefield@?$_Iosb@H@std@@2W4_Fmtflags@12@B 1000a878     pch.obj
 0002:0000087c       ?is_signed@?$numeric_limits@D@std@@2_NB 1000a87c     pch.obj
 0002:00000880       ?floatfield@?$_Iosb@H@std@@2W4_Fmtflags@12@B 1000a880     pch.obj
 0002:00000884       ?digits@?$numeric_limits@D@std@@2HB 1000a884     pch.obj
 0002:00000888       ?digits10@?$numeric_limits@D@std@@2HB 1000a888     pch.obj
 0002:0000088c       ?goodbit@?$_Iosb@H@std@@2W4_Iostate@12@B 1000a88c     pch.obj
 0002:00000890       ?eofbit@?$_Iosb@H@std@@2W4_Iostate@12@B 1000a890     pch.obj
 0002:00000894       ?failbit@?$_Iosb@H@std@@2W4_Iostate@12@B 1000a894     pch.obj
 0002:00000898       ?badbit@?$_Iosb@H@std@@2W4_Iostate@12@B 1000a898     pch.obj
 0002:0000089c       ?_Hardfail@?$_Iosb@H@std@@2W4_Iostate@12@B 1000a89c     pch.obj
 0002:000008a0       ?in@?$_Iosb@H@std@@2W4_Openmode@12@B 1000a8a0     pch.obj
 0002:000008a4       ?out@?$_Iosb@H@std@@2W4_Openmode@12@B 1000a8a4     pch.obj
 0002:000008a8       ?ate@?$_Iosb@H@std@@2W4_Openmode@12@B 1000a8a8     pch.obj
 0002:000008ac       ?app@?$_Iosb@H@std@@2W4_Openmode@12@B 1000a8ac     pch.obj
 0002:000008b0       ?is_signed@?$numeric_limits@_W@std@@2_NB 1000a8b0     pch.obj
 0002:000008b4       ?trunc@?$_Iosb@H@std@@2W4_Openmode@12@B 1000a8b4     pch.obj
 0002:000008b8       ?_Nocreate@?$_Iosb@H@std@@2W4_Openmode@12@B 1000a8b8     pch.obj
 0002:000008bc       ?digits@?$numeric_limits@_W@std@@2HB 1000a8bc     pch.obj
 0002:000008c0       ?_Noreplace@?$_Iosb@H@std@@2W4_Openmode@12@B 1000a8c0     pch.obj
 0002:000008c4       ?digits10@?$numeric_limits@_W@std@@2HB 1000a8c4     pch.obj
 0002:000008c8       ?binary@?$_Iosb@H@std@@2W4_Openmode@12@B 1000a8c8     pch.obj
 0002:000008cc       ?beg@?$_Iosb@H@std@@2W4_Seekdir@12@B 1000a8cc     pch.obj
 0002:000008d0       ?cur@?$_Iosb@H@std@@2W4_Seekdir@12@B 1000a8d0     pch.obj
 0002:000008d4       ?end@?$_Iosb@H@std@@2W4_Seekdir@12@B 1000a8d4     pch.obj
 0002:000008d8       ?is_modulo@?$numeric_limits@_N@std@@2_NB 1000a8d8     pch.obj
 0002:000008d9       ?is_signed@?$numeric_limits@_N@std@@2_NB 1000a8d9     pch.obj
 0002:000008dc       ?digits@?$numeric_limits@_N@std@@2HB 1000a8dc     pch.obj
 0002:000008e0       ?_Stream_err@failure@ios_base@std@@0W4io_errc@43@B 1000a8e0     pch.obj
 0002:000008e4       ?digits10@?$numeric_limits@_N@std@@2HB 1000a8e4     pch.obj
 0002:000008e8       ?value@?$ice_or@$0A@$0A@$0A@$0A@$0A@$0A@$0A@@type_traits@boost@@2_NB 1000a8e8     pch.obj
 0002:000008e9       ?is_signed@?$numeric_limits@C@std@@2_NB 1000a8e9     pch.obj
 0002:000008ec       ?digits@?$numeric_limits@C@std@@2HB 1000a8ec     pch.obj
 0002:000008f0       ?digits10@?$numeric_limits@C@std@@2HB 1000a8f0     pch.obj
 0002:000008f8       ??_7error_category@std@@6B@ 1000a8f8     pch.obj
 0002:00000914       ??_7_Generic_error_category@std@@6B@ 1000a914     pch.obj
 0002:0000092c       ??_C@_07DCLBNMLN@generic?$AA@ 1000a92c     pch.obj
 0002:00000934       ??_C@_0O@BFJCFAAK@unknown?5error?$AA@ 1000a934     pch.obj
 0002:00000948       ??_7_Iostream_error_category@std@@6B@ 1000a948     pch.obj
 0002:00000960       ??_C@_08LLGCOLLL@iostream?$AA@ 1000a960     pch.obj
 0002:0000096c       ??_C@_0BG@PADBLCHM@iostream?5stream?5error?$AA@ 1000a96c     pch.obj
 0002:00000988       ??_7_System_error_category@std@@6B@ 1000a988     pch.obj
 0002:000009a0       ??_C@_06FHFOAHML@system?$AA@ 1000a9a0     pch.obj
 0002:000009ac       ??_7type_info@@6B@         1000a9ac     MSVCRT:ti_inst.obj
 0002:000009b0       __pDefaultRawDllMain       1000a9b0     MSVCRT:crtdll.obj
 0002:000009b0       __pRawDllMain              1000a9b0     MSVCRT:crtdll.obj
 0002:000009b4       ?ProcessDetach@NativeDll@<CrtImplementationDetails>@@0IB 1000a9b4     MSVCRT:initsect.obj
 0002:000009b8       ?ProcessAttach@NativeDll@<CrtImplementationDetails>@@0IB 1000a9b8     MSVCRT:initsect.obj
 0002:000009bc       ?ThreadAttach@NativeDll@<CrtImplementationDetails>@@0IB 1000a9bc     MSVCRT:initsect.obj
 0002:000009c0       ?ThreadDetach@NativeDll@<CrtImplementationDetails>@@0IB 1000a9c0     MSVCRT:initsect.obj
 0002:000009c4       ?ProcessVerifier@NativeDll@<CrtImplementationDetails>@@0IB 1000a9c4     MSVCRT:initsect.obj
 0002:000009d0       __load_config_used         1000a9d0     MSVCRT:loadcfg.obj
 0002:00000a88       ??_R4Resource@LocalizerImp@@6B@ 1000aa88     Localizer.obj
 0002:00000a9c       ??_R3Resource@LocalizerImp@@8 1000aa9c     Localizer.obj
 0002:00000aac       ??_R2Resource@LocalizerImp@@8 1000aaac     Localizer.obj
 0002:00000ab4       ??_R1A@?0A@EA@Resource@LocalizerImp@@8 1000aab4     Localizer.obj
 0002:00000ad0       ??_R1A@?0A@EA@exception@std@@8 1000aad0     LocalizerImp.obj
 0002:00000aec       ??_R3exception@std@@8      1000aaec     LocalizerImp.obj
 0002:00000afc       ??_R2exception@std@@8      1000aafc     LocalizerImp.obj
 0002:00000b04       ??_R4bad_weak_ptr@boost@@6B@ 1000ab04     LocalizerImp.obj
 0002:00000b18       ??_R3bad_weak_ptr@boost@@8 1000ab18     LocalizerImp.obj
 0002:00000b28       ??_R2bad_weak_ptr@boost@@8 1000ab28     LocalizerImp.obj
 0002:00000b34       ??_R1A@?0A@EA@bad_weak_ptr@boost@@8 1000ab34     LocalizerImp.obj
 0002:00000b50       ??_R4sp_counted_base@detail@boost@@6B@ 1000ab50     LocalizerImp.obj
 0002:00000b64       ??_R3sp_counted_base@detail@boost@@8 1000ab64     LocalizerImp.obj
 0002:00000b74       ??_R2sp_counted_base@detail@boost@@8 1000ab74     LocalizerImp.obj
 0002:00000b7c       ??_R1A@?0A@EA@sp_counted_base@detail@boost@@8 1000ab7c     LocalizerImp.obj
 0002:00000b98       ??_R4?$sp_counted_base_impl@PAVResource@LocalizerImp@@U?$checked_deleter@VResource@LocalizerImp@@@boost@@@detail@boost@@6B@ 1000ab98     LocalizerImp.obj
 0002:00000bac       ??_R3?$sp_counted_base_impl@PAVResource@LocalizerImp@@U?$checked_deleter@VResource@LocalizerImp@@@boost@@@detail@boost@@8 1000abac     LocalizerImp.obj
 0002:00000bbc       ??_R2?$sp_counted_base_impl@PAVResource@LocalizerImp@@U?$checked_deleter@VResource@LocalizerImp@@@boost@@@detail@boost@@8 1000abbc     LocalizerImp.obj
 0002:00000bc8       ??_R1A@?0A@EA@?$sp_counted_base_impl@PAVResource@LocalizerImp@@U?$checked_deleter@VResource@LocalizerImp@@@boost@@@detail@boost@@8 1000abc8     LocalizerImp.obj
 0002:00000be4       ??_R4LocalizerResourceTxt@@6B@ 1000abe4     LocalizerTxt.obj
 0002:00000bf8       ??_R3LocalizerResourceTxt@@8 1000abf8     LocalizerTxt.obj
 0002:00000c08       ??_R2LocalizerResourceTxt@@8 1000ac08     LocalizerTxt.obj
 0002:00000c14       ??_R1A@?0A@EA@LocalizerResourceTxt@@8 1000ac14     LocalizerTxt.obj
 0002:00000c30       ??_R4LocalizerResourceUCS@@6B@ 1000ac30     LocalizerUCS.obj
 0002:00000c44       ??_R3LocalizerResourceUCS@@8 1000ac44     LocalizerUCS.obj
 0002:00000c54       ??_R2LocalizerResourceUCS@@8 1000ac54     LocalizerUCS.obj
 0002:00000c60       ??_R1A@?0A@EA@LocalizerResourceUCS@@8 1000ac60     LocalizerUCS.obj
 0002:00000c7c       ??_R4error_category@std@@6B@ 1000ac7c     pch.obj
 0002:00000c90       ??_R3error_category@std@@8 1000ac90     pch.obj
 0002:00000ca0       ??_R2error_category@std@@8 1000aca0     pch.obj
 0002:00000ca8       ??_R1A@?0A@EA@error_category@std@@8 1000aca8     pch.obj
 0002:00000cc4       ??_R4_Generic_error_category@std@@6B@ 1000acc4     pch.obj
 0002:00000cd8       ??_R3_Generic_error_category@std@@8 1000acd8     pch.obj
 0002:00000ce8       ??_R2_Generic_error_category@std@@8 1000ace8     pch.obj
 0002:00000cf4       ??_R1A@?0A@EA@_Generic_error_category@std@@8 1000acf4     pch.obj
 0002:00000d10       ??_R4_Iostream_error_category@std@@6B@ 1000ad10     pch.obj
 0002:00000d24       ??_R3_Iostream_error_category@std@@8 1000ad24     pch.obj
 0002:00000d34       ??_R2_Iostream_error_category@std@@8 1000ad34     pch.obj
 0002:00000d44       ??_R1A@?0A@EA@_Iostream_error_category@std@@8 1000ad44     pch.obj
 0002:00000d60       ??_R4_System_error_category@std@@6B@ 1000ad60     pch.obj
 0002:00000d74       ??_R3_System_error_category@std@@8 1000ad74     pch.obj
 0002:00000d84       ??_R2_System_error_category@std@@8 1000ad84     pch.obj
 0002:00000d94       ??_R1A@?0A@EA@_System_error_category@std@@8 1000ad94     pch.obj
 0002:00000db0       ??_R4type_info@@6B@        1000adb0     MSVCRT:ti_inst.obj
 0002:00000dc4       ??_R3type_info@@8          1000adc4     MSVCRT:ti_inst.obj
 0002:00000dd4       ??_R2type_info@@8          1000add4     MSVCRT:ti_inst.obj
 0002:00000ddc       ??_R1A@?0A@EA@type_info@@8 1000addc     MSVCRT:ti_inst.obj
 0002:00000e00       ___safe_se_handler_table   1000ae00     <linker-defined>
 0002:00000e88       ___rtc_iaa                 1000ae88     MSVCRT:initsect.obj
 0002:00000e8c       ___rtc_izz                 1000ae8c     MSVCRT:initsect.obj
 0002:00000e90       ___rtc_taa                 1000ae90     MSVCRT:initsect.obj
 0002:00000e94       ___rtc_tzz                 1000ae94     MSVCRT:initsect.obj
 0002:00001408       __CT??_R0?AVexception@std@@@8??0exception@std@@QAE@ABV01@@Z12 1000b408     LocalizerImp.obj
 0002:00001424       __TI2?AVbad_weak_ptr@boost@@ 1000b424     LocalizerImp.obj
 0002:00001434       __CTA2?AVbad_weak_ptr@boost@@ 1000b434     LocalizerImp.obj
 0002:00001440       __CT??_R0?AVbad_weak_ptr@boost@@@8??0bad_weak_ptr@boost@@QAE@ABV01@@Z12 1000b440     LocalizerImp.obj
 0002:000017c4       __IMPORT_DESCRIPTOR_Memory 1000b7c4     memory:Memory.dll
 0002:000017d8       __IMPORT_DESCRIPTOR_FileIO 1000b7d8     fileio:FileIO.dll
 0002:000017ec       __IMPORT_DESCRIPTOR_Debug  1000b7ec     debug:Debug.dll
 0002:00001800       __IMPORT_DESCRIPTOR_KERNEL32 1000b800     kernel32:KERNEL32.dll
 0002:00001814       __IMPORT_DESCRIPTOR_USER32 1000b814     user32:USER32.dll
 0002:00001828       __IMPORT_DESCRIPTOR_MSVCP110 1000b828     msvcprt:MSVCP110.dll
 0002:0000183c       __IMPORT_DESCRIPTOR_MSVCR110 1000b83c     MSVCRT:MSVCR110.dll
 0002:00001850       __NULL_IMPORT_DESCRIPTOR   1000b850     memory:Memory.dll
 0003:00000000       ??_R0?AVResource@LocalizerImp@@@8 1000d000     Localizer.obj
 0003:00000024       ??_R0?AVexception@std@@@8  1000d024     LocalizerImp.obj
 0003:00000040       ??_R0?AVbad_weak_ptr@boost@@@8 1000d040     LocalizerImp.obj
 0003:00000064       ??_R0?AVsp_counted_base@detail@boost@@@8 1000d064     LocalizerImp.obj
 0003:00000090       ??_R0?AVLocalizerResourceTxt@@@8 1000d090     LocalizerImp.obj
 0003:000000b4       ??_R0?AVLocalizerResourceUCS@@@8 1000d0b4     LocalizerImp.obj
 0003:000000d8       ??_R0?AU?$checked_deleter@VResource@LocalizerImp@@@boost@@@8 1000d0d8     LocalizerImp.obj
 0003:00000118       ??_R0?AV?$sp_counted_base_impl@PAVResource@LocalizerImp@@U?$checked_deleter@VResource@LocalizerImp@@@boost@@@detail@boost@@@8 1000d118     LocalizerImp.obj
 0003:00000198       ?FileExtension@LocalizerResourceTxt@@2PBDB 1000d198     LocalizerTxt.obj
 0003:0000019c       ?FileExtension@LocalizerResourceUCS@@2PBDB 1000d19c     LocalizerUCS.obj
 0003:000001a0       ?_Generic_object@?$_Error_objects@H@std@@2V_Generic_error_category@2@A 1000d1a0     pch.obj
 0003:000001a4       ?_Iostream_object@?$_Error_objects@H@std@@2V_Iostream_error_category@2@A 1000d1a4     pch.obj
 0003:000001a8       ?_System_object@?$_Error_objects@H@std@@2V_System_error_category@2@A 1000d1a8     pch.obj
 0003:000001ac       ??_R0?AVerror_category@std@@@8 1000d1ac     pch.obj
 0003:000001d0       ??_R0?AV_Generic_error_category@std@@@8 1000d1d0     pch.obj
 0003:000001fc       ??_R0?AV_Iostream_error_category@std@@@8 1000d1fc     pch.obj
 0003:00000228       ??_R0?AV_System_error_category@std@@@8 1000d228     pch.obj
 0003:00000260       ??_R0?AVtype_info@@@8      1000d260     MSVCRT:ti_inst.obj
 0003:00000280       ___native_dllmain_reason   1000d280     MSVCRT:natstart.obj
 0003:00000284       ___security_cookie         1000d284     MSVCRT:gs_cookie.obj
 0003:00000288       ___security_cookie_complement 1000d288     MSVCRT:gs_cookie.obj
 0003:00000290       ?_1@?A0x5d8973ec@@3V?$arg@$00@boost@@A 1000d290     Localizer.obj
 0003:00000291       ?_2@?A0x5d8973ec@@3V?$arg@$01@boost@@A 1000d291     Localizer.obj
 0003:00000292       ?_3@?A0x5d8973ec@@3V?$arg@$02@boost@@A 1000d292     Localizer.obj
 0003:00000293       ?_4@?A0x5d8973ec@@3V?$arg@$03@boost@@A 1000d293     Localizer.obj
 0003:00000294       ?_5@?A0x5d8973ec@@3V?$arg@$04@boost@@A 1000d294     Localizer.obj
 0003:00000295       ?_6@?A0x5d8973ec@@3V?$arg@$05@boost@@A 1000d295     Localizer.obj
 0003:00000296       ?_7@?A0x5d8973ec@@3V?$arg@$06@boost@@A 1000d296     Localizer.obj
 0003:00000297       ?_8@?A0x5d8973ec@@3V?$arg@$07@boost@@A 1000d297     Localizer.obj
 0003:00000298       ?_9@?A0x5d8973ec@@3V?$arg@$08@boost@@A 1000d298     Localizer.obj
 0003:000042a0       ?_1@?A0x592ce793@@3V?$arg@$00@boost@@A 100112a0     LocalizerImp.obj
 0003:000042a1       ?_2@?A0x592ce793@@3V?$arg@$01@boost@@A 100112a1     LocalizerImp.obj
 0003:000042a2       ?_3@?A0x592ce793@@3V?$arg@$02@boost@@A 100112a2     LocalizerImp.obj
 0003:000042a3       ?_4@?A0x592ce793@@3V?$arg@$03@boost@@A 100112a3     LocalizerImp.obj
 0003:000042a4       ?_5@?A0x592ce793@@3V?$arg@$04@boost@@A 100112a4     LocalizerImp.obj
 0003:000042a5       ?_6@?A0x592ce793@@3V?$arg@$05@boost@@A 100112a5     LocalizerImp.obj
 0003:000042a6       ?_7@?A0x592ce793@@3V?$arg@$06@boost@@A 100112a6     LocalizerImp.obj
 0003:000042a7       ?_8@?A0x592ce793@@3V?$arg@$07@boost@@A 100112a7     LocalizerImp.obj
 0003:000042a8       ?_9@?A0x592ce793@@3V?$arg@$08@boost@@A 100112a8     LocalizerImp.obj
 0003:000042c4       ?_3@?A0xa493ca04@@3V?$arg@$02@boost@@A 100112c4     LocalizerUCS.obj
 0003:000042c5       ?_4@?A0xa493ca04@@3V?$arg@$03@boost@@A 100112c5     LocalizerUCS.obj
 0003:000042c6       ?_5@?A0xa493ca04@@3V?$arg@$04@boost@@A 100112c6     LocalizerUCS.obj
 0003:000042c7       ?_6@?A0xa493ca04@@3V?$arg@$05@boost@@A 100112c7     LocalizerUCS.obj
 0003:000042c8       ?_7@?A0xa493ca04@@3V?$arg@$06@boost@@A 100112c8     LocalizerUCS.obj
 0003:000042c9       ?_8@?A0xa493ca04@@3V?$arg@$07@boost@@A 100112c9     LocalizerUCS.obj
 0003:000042ca       ?_9@?A0xa493ca04@@3V?$arg@$08@boost@@A 100112ca     LocalizerUCS.obj
 0003:000042cb       ?_1@?A0xa493ca04@@3V?$arg@$00@boost@@A 100112cb     LocalizerUCS.obj
 0003:000042cc       ?_2@?A0xa493ca04@@3V?$arg@$01@boost@@A 100112cc     LocalizerUCS.obj
 0003:000042d0       ___@@_PchSym_@00@UsrxplibRkxhsrkUslnvdliowCxozhhrxUhixUrmgvinvwrzgvUhszivwUolxzoraviUivovzhvUlyqUkxsOlyq@5DD7BEB794714209 100112d0     pch.obj
 0003:000042d8       ?id@?$num_put@DV?$back_insert_iterator@V?$basic_string@DU?$char_traits@D@std@@V?$allocator@D@2@@std@@@std@@@std@@2V0locale@2@A 100112d8     pch.obj
 0003:000042dc       ?id@?$num_put@_WV?$back_insert_iterator@V?$basic_string@_WU?$char_traits@_W@std@@V?$allocator@_W@2@@std@@@std@@@std@@2V0locale@2@A 100112dc     pch.obj
 0003:000042e4       ?__type_info_root_node@@3U__type_info_node@@A 100112e4     MSVCRT:tncleanup.obj
 0003:00004610       ___native_startup_lock     10011610     <common>
 0003:00004614       ___native_startup_state    10011614     <common>
 0003:00004618       ___dyn_tls_init_callback   10011618     <common>
 0003:0000461c       ___onexitend               1001161c     <common>
 0003:00004620       ___onexitbegin             10011620     <common>

 entry point at        0001:000081b8

 Static symbols

 0000:fffec000       .debug$S                   10000000     MSVCRT:MSVCR110.dll
 0000:fffec000       .debug$S                   10000000     MSVCRT:MSVCR110.dll
 0000:fffec000       .debug$S                   10000000     MSVCRT:MSVCR110.dll
 0000:fffec000       .debug$S                   10000000     MSVCRT:MSVCR110.dll
 0000:fffec000       .debug$S                   10000000     MSVCRT:MSVCR110.dll
 0000:fffec000       .debug$S                   10000000     MSVCRT:MSVCR110.dll
 0000:fffec000       .debug$S                   10000000     MSVCRT:MSVCR110.dll
 0000:fffec000       .debug$S                   10000000     MSVCRT:MSVCR110.dll
 0000:fffec000       .debug$S                   10000000     MSVCRT:MSVCR110.dll
 0000:fffec000       .debug$S                   10000000     MSVCRT:MSVCR110.dll
 0000:fffec000       .debug$S                   10000000     MSVCRT:MSVCR110.dll
 0000:fffec000       .debug$S                   10000000     MSVCRT:MSVCR110.dll
 0000:fffec000       .debug$S                   10000000     MSVCRT:MSVCR110.dll
 0000:fffec000       .debug$S                   10000000     MSVCRT:MSVCR110.dll
 0000:fffec000       .debug$S                   10000000     MSVCRT:MSVCR110.dll
 0000:fffec000       .debug$S                   10000000     MSVCRT:MSVCR110.dll
 0000:fffec000       .debug$S                   10000000     MSVCRT:MSVCR110.dll
 0000:fffec000       .debug$S                   10000000     MSVCRT:MSVCR110.dll
 0000:fffec000       .debug$S                   10000000     MSVCRT:MSVCR110.dll
 0000:fffec000       .debug$S                   10000000     MSVCRT:MSVCR110.dll
 0000:fffec000       .debug$S                   10000000     MSVCRT:MSVCR110.dll
 0000:fffec000       .debug$S                   10000000     MSVCRT:MSVCR110.dll
 0000:fffec000       .debug$S                   10000000     MSVCRT:MSVCR110.dll
 0000:fffec000       .debug$S                   10000000     MSVCRT:MSVCR110.dll
 0000:fffec000       .debug$S                   10000000     MSVCRT:MSVCR110.dll
 0000:fffec000       .debug$S                   10000000     MSVCRT:MSVCR110.dll
 0000:fffec000       .debug$S                   10000000     MSVCRT:MSVCR110.dll
 0000:fffec000       .debug$S                   10000000     MSVCRT:MSVCR110.dll
 0000:fffec000       .debug$S                   10000000     MSVCRT:MSVCR110.dll
 0000:fffec000       .debug$S                   10000000     MSVCRT:MSVCR110.dll
 0000:fffec000       .debug$S                   10000000     MSVCRT:MSVCR110.dll
 0000:fffec000       .debug$S                   10000000     MSVCRT:MSVCR110.dll
 0000:fffec000       .debug$S                   10000000     MSVCRT:MSVCR110.dll
 0000:fffec000       .debug$S                   10000000     MSVCRT:MSVCR110.dll
 0000:fffec000       .debug$S                   10000000     MSVCRT:MSVCR110.dll
 0000:fffec000       .debug$S                   10000000     MSVCRT:MSVCR110.dll
 0000:fffec000       .debug$S                   10000000     MSVCRT:MSVCR110.dll
 0000:fffec000       .debug$S                   10000000     MSVCRT:MSVCR110.dll
 0000:fffec000       .debug$S                   10000000     MSVCRT:MSVCR110.dll
 0000:fffec000       .debug$S                   10000000     MSVCRT:MSVCR110.dll
 0000:fffec000       .debug$S                   10000000     MSVCRT:MSVCR110.dll
 0000:fffec000       .debug$S                   10000000     MSVCRT:MSVCR110.dll
 0000:fffec000       .debug$S                   10000000     MSVCRT:MSVCR110.dll
 0000:fffec000       .debug$S                   10000000     MSVCRT:MSVCR110.dll
 0000:fffec000       .debug$S                   10000000     MSVCRT:MSVCR110.dll
 0000:fffec000       .debug$S                   10000000     MSVCRT:MSVCR110.dll
 0000:fffec000       .debug$S                   10000000     MSVCRT:MSVCR110.dll
 0000:fffec000       .debug$S                   10000000     MSVCRT:MSVCR110.dll
 0001:fffff000       __ehhandler$?_Copy@?$basic_string@DU?$char_traits@D@std@@V?$allocator@D@2@@std@@QAEXII@Z 10000000 f   LocalizerImp.obj
 0000:fffec000       .debug$S                   10000000     fileio:FileIO.dll
 0000:fffec000       .debug$S                   10000000     fileio:FileIO.dll
 0000:fffec000       .debug$S                   10000000     fileio:FileIO.dll
 0000:fffec000       .debug$S                   10000000     fileio:FileIO.dll
 0002:ffff6000       __catchsym$?_Copy@?$basic_string@DU?$char_traits@D@std@@V?$allocator@D@2@@std@@QAEXII@Z$5 10000000     LocalizerImp.obj
 0000:fffec000       .debug$S                   10000000     msvcprt:MSVCP110.dll
 0000:fffec000       .debug$S                   10000000     msvcprt:MSVCP110.dll
 0000:fffec000       .debug$S                   10000000     msvcprt:MSVCP110.dll
 0001:fffff000       __ehhandler$?_Copy@?$basic_string@DU?$char_traits@D@std@@V?$allocator@D@2@@std@@QAEXII@Z 10000000 f   pch.obj
 0002:ffff6000       __catchsym$?_Copy@?$basic_string@DU?$char_traits@D@std@@V?$allocator@D@2@@std@@QAEXII@Z$5 10000000     LocalizerTxt.obj
 0000:fffec000       .debug$S                   10000000     fileio:FileIO.dll
 0000:fffec000       .debug$S                   10000000     fileio:FileIO.dll
 0001:fffff000       __ehhandler$?_Copy@?$basic_string@DU?$char_traits@D@std@@V?$allocator@D@2@@std@@QAEXII@Z 10000000 f   LocalizerTxt.obj
 0000:fffec000       .debug$S                   10000000     fileio:FileIO.dll
 0000:fffec000       .debug$S                   10000000     debug:Debug.dll
 0002:ffff6000       __catchsym$?_Copy@?$basic_string@DU?$char_traits@D@std@@V?$allocator@D@2@@std@@QAEXII@Z$5 10000000     pch.obj
 0000:fffec000       .debug$S                   10000000     msvcprt:MSVCP110.dll
 0000:fffec000       .debug$S                   10000000     msvcprt:MSVCP110.dll
 0000:fffec000       .debug$S                   10000000     msvcprt:MSVCP110.dll
 0000:fffec000       .debug$S                   10000000     msvcprt:MSVCP110.dll
 0000:fffec000       .debug$S                   10000000     msvcprt:MSVCP110.dll
 0000:fffec000       .debug$S                   10000000     user32:USER32.dll
 0000:fffec000       .debug$S                   10000000     kernel32:KERNEL32.dll
 0000:fffec000       .debug$S                   10000000     kernel32:KERNEL32.dll
 0000:fffec000       .debug$S                   10000000     kernel32:KERNEL32.dll
 0000:fffec000       .debug$S                   10000000     kernel32:KERNEL32.dll
 0000:fffec000       .debug$S                   10000000     kernel32:KERNEL32.dll
 0000:fffec000       .debug$S                   10000000     kernel32:KERNEL32.dll
 0000:fffec000       .debug$S                   10000000     memory:Memory.dll
 0000:fffec000       .debug$S                   10000000     memory:Memory.dll
 0000:fffec000       .debug$S                   10000000     memory:Memory.dll
 0000:fffec000       .debug$S                   10000000     memory:Memory.dll
 0001:fffff000       __ehhandler$?_Copy@?$basic_string@DU?$char_traits@D@std@@V?$allocator@D@2@@std@@QAEXII@Z 10000000 f   LocalizerUCS.obj
 0000:fffec000       .debug$S                   10000000     fileio:FileIO.dll
 0000:fffec000       .debug$S                   10000000     fileio:FileIO.dll
 0000:fffec000       .debug$S                   10000000     kernel32:KERNEL32.dll
 0000:fffec000       .debug$S                   10000000     kernel32:KERNEL32.dll
 0000:fffec000       .debug$S                   10000000     kernel32:KERNEL32.dll
 0000:fffec000       .debug$S                   10000000     kernel32:KERNEL32.dll
 0000:fffec000       .debug$S                   10000000     kernel32:KERNEL32.dll
 0000:fffec000       .debug$S                   10000000     kernel32:KERNEL32.dll
 0000:fffec000       .debug$S                   10000000     kernel32:KERNEL32.dll
 0000:fffec000       .debug$S                   10000000     kernel32:KERNEL32.dll
 0000:fffec000       .debug$S                   10000000     kernel32:KERNEL32.dll
 0000:fffec000       .debug$S                   10000000     kernel32:KERNEL32.dll
 0000:fffec000       .debug$S                   10000000     kernel32:KERNEL32.dll
 0000:fffec000       .debug$S                   10000000     kernel32:KERNEL32.dll
 0000:fffec000       .debug$S                   10000000     kernel32:KERNEL32.dll
 0000:fffec000       .debug$S                   10000000     kernel32:KERNEL32.dll
 0000:fffec000       .debug$S                   10000000     kernel32:KERNEL32.dll
 0000:fffec000       .debug$S                   10000000     kernel32:KERNEL32.dll
 0000:fffec000       .debug$S                   10000000     kernel32:KERNEL32.dll
 0000:fffec000       .debug$S                   10000000     kernel32:KERNEL32.dll
 0002:ffff6000       __catchsym$?_Copy@?$basic_string@DU?$char_traits@D@std@@V?$allocator@D@2@@std@@QAEXII@Z$5 10000000     LocalizerUCS.obj
 0000:fffec000       .debug$S                   10000000     kernel32:KERNEL32.dll
 0000:fffec000       .debug$S                   10000000     kernel32:KERNEL32.dll
 0000:fffec000       .debug$S                   10000000     kernel32:KERNEL32.dll
 0000:fffec000       .debug$S                   10000000     kernel32:KERNEL32.dll
 0002:ffff6010       __catchsym$?_Copy@?$basic_string@DU?$char_traits@D@std@@V?$allocator@D@2@@std@@QAEXII@Z$4 10000010     pch.obj
 0002:ffff6010       __catchsym$?_Copy@?$basic_string@DU?$char_traits@D@std@@V?$allocator@D@2@@std@@QAEXII@Z$4 10000010     LocalizerTxt.obj
 0002:ffff6010       __catchsym$?_Copy@?$basic_string@DU?$char_traits@D@std@@V?$allocator@D@2@@std@@QAEXII@Z$4 10000010     LocalizerImp.obj
 0002:ffff6010       __catchsym$?_Copy@?$basic_string@DU?$char_traits@D@std@@V?$allocator@D@2@@std@@QAEXII@Z$4 10000010     LocalizerUCS.obj
 0002:ffff6020       __unwindtable$?_Copy@?$basic_string@DU?$char_traits@D@std@@V?$allocator@D@2@@std@@QAEXII@Z 10000020     LocalizerTxt.obj
 0002:ffff6020       __unwindtable$?_Copy@?$basic_string@DU?$char_traits@D@std@@V?$allocator@D@2@@std@@QAEXII@Z 10000020     pch.obj
 0002:ffff6020       __unwindtable$?_Copy@?$basic_string@DU?$char_traits@D@std@@V?$allocator@D@2@@std@@QAEXII@Z 10000020     LocalizerUCS.obj
 0002:ffff6020       __unwindtable$?_Copy@?$basic_string@DU?$char_traits@D@std@@V?$allocator@D@2@@std@@QAEXII@Z 10000020     LocalizerImp.obj
 0002:ffff6040       __ehfuncinfo$?_Copy@?$basic_string@DU?$char_traits@D@std@@V?$allocator@D@2@@std@@QAEXII@Z 10000040     pch.obj
 0002:ffff6040       __ehfuncinfo$?_Copy@?$basic_string@DU?$char_traits@D@std@@V?$allocator@D@2@@std@@QAEXII@Z 10000040     LocalizerTxt.obj
 0002:ffff6040       __ehfuncinfo$?_Copy@?$basic_string@DU?$char_traits@D@std@@V?$allocator@D@2@@std@@QAEXII@Z 10000040     LocalizerUCS.obj
 0002:ffff6040       __ehfuncinfo$?_Copy@?$basic_string@DU?$char_traits@D@std@@V?$allocator@D@2@@std@@QAEXII@Z 10000040     LocalizerImp.obj
 0002:ffff6064       __tryblocktable$?_Copy@?$basic_string@DU?$char_traits@D@std@@V?$allocator@D@2@@std@@QAEXII@Z 10000064     LocalizerUCS.obj
 0002:ffff6064       __tryblocktable$?_Copy@?$basic_string@DU?$char_traits@D@std@@V?$allocator@D@2@@std@@QAEXII@Z 10000064     LocalizerImp.obj
 0002:ffff6064       __tryblocktable$?_Copy@?$basic_string@DU?$char_traits@D@std@@V?$allocator@D@2@@std@@QAEXII@Z 10000064     pch.obj
 0002:ffff6064       __tryblocktable$?_Copy@?$basic_string@DU?$char_traits@D@std@@V?$allocator@D@2@@std@@QAEXII@Z 10000064     LocalizerTxt.obj
 0001:fffff068       __catch$?_Copy@?$basic_string@DU?$char_traits@D@std@@V?$allocator@D@2@@std@@QAEXII@Z$0 10000068 f   LocalizerImp.obj
 0001:fffff068       __catch$?_Copy@?$basic_string@DU?$char_traits@D@std@@V?$allocator@D@2@@std@@QAEXII@Z$0 10000068 f   LocalizerUCS.obj
 0001:fffff068       __catch$?_Copy@?$basic_string@DU?$char_traits@D@std@@V?$allocator@D@2@@std@@QAEXII@Z$0 10000068 f   LocalizerTxt.obj
 0001:fffff068       __catch$?_Copy@?$basic_string@DU?$char_traits@D@std@@V?$allocator@D@2@@std@@QAEXII@Z$0 10000068 f   pch.obj
 0001:fffff0ee       __catch$?_Copy@?$basic_string@DU?$char_traits@D@std@@V?$allocator@D@2@@std@@QAEXII@Z$1 100000ee f   LocalizerUCS.obj
 0001:fffff0ee       __catch$?_Copy@?$basic_string@DU?$char_traits@D@std@@V?$allocator@D@2@@std@@QAEXII@Z$1 100000ee f   pch.obj
 0001:fffff0ee       __catch$?_Copy@?$basic_string@DU?$char_traits@D@std@@V?$allocator@D@2@@std@@QAEXII@Z$1 100000ee f   LocalizerTxt.obj
 0001:fffff0ee       __catch$?_Copy@?$basic_string@DU?$char_traits@D@std@@V?$allocator@D@2@@std@@QAEXII@Z$1 100000ee f   LocalizerImp.obj
 0001:000009f0       ?ConvertToMultiByte@@YG_NPADIPB_W@Z 100019f0 f   Localizer.obj
 0001:00000a24       ?FormatArgsExtract@@YG_NQAPB_WQBIIPAH@Z 10001a24 f   Localizer.obj
 0001:00000a73       ?FormatArgsUsed@@YG_NQAIAAIPB_W@Z 10001a73 f   Localizer.obj
 0001:00000b06       ?FormatInternal@@YG_NPA_WIPB_WQAPB_W@Z 10001b06 f   Localizer.obj
 0001:00000eb9       ?IsAllowed@Pred@?7??CheckString@Localizer@@SG_NPB_WK0@Z@SG_N_W0@Z 10001eb9 f   Localizer.obj
 0001:00000ed2       ?IsNT@@YG_NXZ              10001ed2 f   Localizer.obj
 0001:00001219       __catch$?_Copy@?$basic_string@DU?$char_traits@D@std@@V?$allocator@D@2@@std@@QAEXII@Z$0 10002219 f i Localizer.obj
 0001:0000129f       __catch$?_Copy@?$basic_string@DU?$char_traits@D@std@@V?$allocator@D@2@@std@@QAEXII@Z$1 1000229f f i Localizer.obj
 0001:0000132b       __catch$?_Copy@?$basic_string@_WU?$char_traits@_W@std@@V?$allocator@_W@2@@std@@QAEXII@Z$0 1000232b f i Localizer.obj
 0001:000013a8       __catch$?_Copy@?$basic_string@_WU?$char_traits@_W@std@@V?$allocator@_W@2@@std@@QAEXII@Z$1 100023a8 f i Localizer.obj
 0001:00001c89       __catch$??$?0PAVResource@LocalizerImp@@U?$checked_deleter@VResource@LocalizerImp@@@boost@@@shared_count@detail@boost@@QAE@PAVResource@LocalizerImp@@U?$checked_deleter@VResource@LocalizerImp@@@2@@Z$0 10002c89 f i LocalizerImp.obj
 0001:00001ea6       __catch$??$_Uninit_move@PAVResEntry@LocalizerImp@@PAV12@V?$allocator@VResEntry@LocalizerImp@@@std@@V12@@std@@YGPAVResEntry@LocalizerImp@@PAV12@00AAU?$_Wrap_alloc@V?$allocator@VResEntry@LocalizerImp@@@std@@@0@0U_Nonscalar_ptr_iterator_tag@0@@Z$0 10002ea6 f i LocalizerImp.obj
 0001:00002748       ?CheckName@S@?4??InternalResUnload@LocalizerImp@@AAE_NPBD@Z@SG_NABVResEntry@3@0@Z 10003748 f   LocalizerImp.obj
 0001:00002a93       ?ListFiles@@YGXAAV?$vector@V?$basic_string@DU?$char_traits@D@std@@V?$allocator@D@2@@std@@V?$allocator@V?$basic_string@DU?$char_traits@D@std@@V?$allocator@D@2@@std@@@2@@std@@PBD1@Z 10003a93 f   LocalizerImp.obj
 0001:00002bcf       ?ListFilesTime@@YGXABV?$vector@V?$basic_string@DU?$char_traits@D@std@@V?$allocator@D@2@@std@@V?$allocator@V?$basic_string@DU?$char_traits@D@std@@V?$allocator@D@2@@std@@@2@@std@@_NAAU_FILETIME@@@Z 10003bcf f   LocalizerImp.obj
 0001:00002ca3       ?RangeOverlap@@YG_NHHH@Z   10003ca3 f   LocalizerImp.obj
 0001:00003210       __catch$?_Reallocate@?$vector@V?$basic_string@DU?$char_traits@D@std@@V?$allocator@D@2@@std@@V?$allocator@V?$basic_string@DU?$char_traits@D@std@@V?$allocator@D@2@@std@@@2@@std@@IAEXI@Z$0 10004210 f i LocalizerImp.obj
 0001:000032ad       __catch$?_Reallocate@?$vector@VResEntry@LocalizerImp@@V?$allocator@VResEntry@LocalizerImp@@@std@@@std@@IAEXI@Z$0 100042ad f i LocalizerImp.obj
 0001:0000533b       ?LineIsWSChar@@YG_ND@Z     1000633b f   LocalizerTxt.obj
 0001:00005351       ?LineParse@@YGXPBDAAUParseOut@?A0x10e53216@@@Z 10006351 f   LocalizerTxt.obj
 0001:000053e5       ?LineParseComment@@YG_NPBDAAUParseOut@?A0x10e53216@@@Z 100063e5 f   LocalizerTxt.obj
 0001:0000542e       ?LineParseFileRange@@YG_NPBDAAUParseOut@?A0x10e53216@@@Z 1000642e f   LocalizerTxt.obj
 0001:00005470       ?LineParseRangeEnd@@YG_NPBDAAUParseOut@?A0x10e53216@@@Z 10006470 f   LocalizerTxt.obj
 0001:000054c8       ?LineParseRangeStart@@YG_NPBDAAUParseOut@?A0x10e53216@@@Z 100064c8 f   LocalizerTxt.obj
 0001:00005508       ?LineParseText@@YG_NPBDAAUParseOut@?A0x10e53216@@@Z 10006508 f   LocalizerTxt.obj
 0001:000055b9       ?LinePrep@@YGXPAD@Z        100065b9 f   LocalizerTxt.obj
 0001:00005b06       ?RangeDuplicate@@YG_NABV?$vector@URange@LocalizerResourceTxt@@V?$mempool_alloc@URange@LocalizerResourceTxt@@@@@std@@HH@Z 10006b06 f   LocalizerTxt.obj
 0001:00005b79       ?RangeReset@@YGXAAURange@LocalizerResourceTxt@@@Z 10006b79 f   LocalizerTxt.obj
 0001:00005b9b       ?RangeSetup@@YGXAAURange@LocalizerResourceTxt@@PBDHH@Z 10006b9b f   LocalizerTxt.obj
 0001:00005df9       ?TxtLineDuplicate@@YG_NABV?$vector@U?$pair@HULine@LocalizerResourceTxt@@@std@@V?$mempool_alloc@U?$pair@HULine@LocalizerResourceTxt@@@std@@@@@std@@H@Z 10006df9 f   LocalizerTxt.obj
 0001:00005e1c       ?TxtLineFind@@YG?AV?$_Vector_const_iterator@V?$_Vector_val@U?$_Simple_types@U?$pair@HULine@LocalizerResourceTxt@@@std@@@std@@@std@@@std@@ABV?$vector@U?$pair@HULine@LocalizerResourceTxt@@@std@@V?$mempool_alloc@U?$pair@HULine@LocalizerResourceTxt@@@std@@@@@2@H@Z 10006e1c f   LocalizerTxt.obj
 0001:00005e54       ?TxtLineFind@@YG?AV?$_Vector_iterator@V?$_Vector_val@U?$_Simple_types@U?$pair@HULine@LocalizerResourceTxt@@@std@@@std@@@std@@@std@@AAV?$vector@U?$pair@HULine@LocalizerResourceTxt@@@std@@V?$mempool_alloc@U?$pair@HULine@LocalizerResourceTxt@@@std@@@@@2@H@Z 10006e54 f   LocalizerTxt.obj
 0001:00005e8c       ?TxtLineInsert@@YG?AV?$_Vector_iterator@V?$_Vector_val@U?$_Simple_types@U?$pair@HULine@LocalizerResourceTxt@@@std@@@std@@@std@@@std@@AAV?$vector@U?$pair@HULine@LocalizerResourceTxt@@@std@@V?$mempool_alloc@U?$pair@HULine@LocalizerResourceTxt@@@std@@@@@2@HULine@LocalizerResourceTxt@@@Z 10006e8c f   LocalizerTxt.obj
 0001:00005eda       ?TxtLineReset@@YGXAAULine@LocalizerResourceTxt@@@Z 10006eda f   LocalizerTxt.obj
 0001:00005f27       ?TxtLineSetup@@YGXAAULine@LocalizerResourceTxt@@PBD1@Z 10006f27 f   LocalizerTxt.obj
 0001:00005f68       ?TxtLineSetup@@YGXAAULine@LocalizerResourceTxt@@PBDPB_W1@Z 10006f68 f   LocalizerTxt.obj
 0001:00005fec       ?TxtLineUpdate@@YGXAAULine@LocalizerResourceTxt@@PBDPB_W@Z 10006fec f   LocalizerTxt.obj
 0001:00006009       ?TxtLineUpdate@@YGXAAULine@LocalizerResourceTxt@@PB_W@Z 10007009 f   LocalizerTxt.obj
 0001:00006176       __catch$?_Reallocate@?$vector@U?$pair@HULine@LocalizerResourceTxt@@@std@@V?$mempool_alloc@U?$pair@HULine@LocalizerResourceTxt@@@std@@@@@std@@IAEXI@Z$0 10007176 f i LocalizerTxt.obj
 0001:00006226       __catch$?_Reallocate@?$vector@URange@LocalizerResourceTxt@@V?$mempool_alloc@URange@LocalizerResourceTxt@@@@@std@@IAEXI@Z$0 10007226 f i LocalizerTxt.obj
 0001:000064ea       ?destroy@clearall@?1???1LocalizerResourceTxt@@UAE@XZ@SGXAAU?$pair@HULine@LocalizerResourceTxt@@@std@@@Z 100074ea f   LocalizerTxt.obj
 0001:0000679b       ??$WBufParse@V?$bind_t@_NP6G_NPB_W000PAI1@ZV?$list6@V?$arg@$00@boost@@V?$arg@$01@2@V?$arg@$02@2@V?$arg@$03@2@V?$value@PAI@_bi@2@V672@@_bi@boost@@@_bi@boost@@@@YG_NPB_WV?$bind_t@_NP6G_NPB_W000PAI1@ZV?$list6@V?$arg@$00@boost@@V?$arg@$01@2@V?$arg@$02@2@V?$arg@$03@2@V?$value@PAI@_bi@2@V672@@_bi@boost@@@_bi@boost@@@Z 1000779b f   LocalizerUCS.obj
 0001:00006810       ??$WBufParse@V?$bind_t@_NP6G_NPB_W000PAULine@LocalizerResourceUCS@@PAIPAPA_W@ZV?$list7@V?$arg@$00@boost@@V?$arg@$01@2@V?$arg@$02@2@V?$arg@$03@2@V?$value@PAULine@LocalizerResourceUCS@@@_bi@2@V?$value@PAI@72@V?$value@PAPA_W@72@@_bi@boost@@@_bi@boost@@@@YG_NPB_WV?$bind_t@_NP6G_NPB_W000PAULine@LocalizerResourceUCS@@PAIPAPA_W@ZV?$list7@V?$arg@$00@boost@@V?$arg@$01@2@V?$arg@$02@2@V?$arg@$03@2@V?$value@PAULine@LocalizerResourceUCS@@@_bi@2@V?$value@PAI@72@V?$value@PAPA_W@72@@_bi@boost@@@_bi@boost@@@Z 10007810 f   LocalizerUCS.obj
 0001:00007446       ?Counter@S@?1??WBufCount@@YG_NPB_WAAI1@Z@SG_N0000PAI2@Z 10008446 f   LocalizerUCS.obj
 0001:00007612       ?Liner@S@?1??WBufParseAll@@YG_NPB_WPBIPAULine@LocalizerResourceUCS@@PA_W@Z@SG_N00002PAIPAPA_W@Z 10008612 f   LocalizerUCS.obj
 0001:000077f0       ?WBufCount@@YG_NPB_WAAI1@Z 100087f0 f   LocalizerUCS.obj
 0001:00007839       ?WBufParseAll@@YG_NPB_WPBIPAULine@LocalizerResourceUCS@@PA_W@Z 10008839 f   LocalizerUCS.obj
 0001:00007899       ?WBufParseLine@@YGXPB_W0PAPB_W111@Z 10008899 f   LocalizerUCS.obj
 0001:00007c9d       ?ArrayUnwindFilter@@YAHPAU_EXCEPTION_POINTERS@@@Z 10008c9d f   MSVCRT:ehvecdtr.obj
 0001:00007d70       $$000000                   10008d70     MSVCRT:ehprolog.obj
 0001:00007da0       $$000000                   10008da0     MSVCRT:chkstk.obj
 0001:00007f70       _pre_c_init                10008f70 f   MSVCRT:crtdll.obj
 0001:000081db       ___DllMainCRTStartup       100091db f   MSVCRT:crtdll.obj
 0001:00008320       $$000000                   10009320     MSVCRT:sehprolg4.obj
 0001:000089ba       __unwindfunclet$?CheckString@Localizer@@SG_NPB_WK0@Z$0 100099ba f   Localizer.obj
 0001:000089c2       __unwindfunclet$?CheckString@Localizer@@SG_NPB_WK0@Z$1 100099c2 f   Localizer.obj
 0001:000089ca       __ehhandler$?CheckString@Localizer@@SG_NPB_WK0@Z 100099ca f   Localizer.obj
 0001:000089d4       __ehhandler$?_Copy@?$basic_string@DU?$char_traits@D@std@@V?$allocator@D@2@@std@@QAEXII@Z 100099d4 f   Localizer.obj
 0001:000089de       __ehhandler$?_Copy@?$basic_string@_WU?$char_traits@_W@std@@V?$allocator@_W@2@@std@@QAEXII@Z 100099de f   Localizer.obj
 0001:000089e8       __ehhandler$??$?0PAVResource@LocalizerImp@@U?$checked_deleter@VResource@LocalizerImp@@@boost@@@shared_count@detail@boost@@QAE@PAVResource@LocalizerImp@@U?$checked_deleter@VResource@LocalizerImp@@@2@@Z 100099e8 f   LocalizerImp.obj
 0001:000089f2       __ehhandler$??$_Uninit_move@PAVResEntry@LocalizerImp@@PAV12@V?$allocator@VResEntry@LocalizerImp@@@std@@V12@@std@@YGPAVResEntry@LocalizerImp@@PAV12@00AAU?$_Wrap_alloc@V?$allocator@VResEntry@LocalizerImp@@@std@@@0@0U_Nonscalar_ptr_iterator_tag@0@@Z 100099f2 f   LocalizerImp.obj
 0001:000089fc       __unwindfunclet$??$construct@V?$basic_string@DU?$char_traits@D@std@@V?$allocator@D@2@@std@@AAV12@@?$_Wrap_alloc@V?$allocator@V?$basic_string@DU?$char_traits@D@std@@V?$allocator@D@2@@std@@@std@@@std@@QAEXPAV?$basic_string@DU?$char_traits@D@std@@V?$allocator@D@2@@1@AAV21@@Z$0 100099fc f   LocalizerImp.obj
 0001:00008a0a       __ehhandler$??$construct@V?$basic_string@DU?$char_traits@D@std@@V?$allocator@D@2@@std@@AAV12@@?$_Wrap_alloc@V?$allocator@V?$basic_string@DU?$char_traits@D@std@@V?$allocator@D@2@@std@@@std@@@std@@QAEXPAV?$basic_string@DU?$char_traits@D@std@@V?$allocator@D@2@@1@AAV21@@Z 10009a0a f   LocalizerImp.obj
 0001:00008a14       __unwindfunclet$??$construct@V?$basic_string@DU?$char_traits@D@std@@V?$allocator@D@2@@std@@AAV12@@?$allocator@V?$basic_string@DU?$char_traits@D@std@@V?$allocator@D@2@@std@@@std@@QAEXPAV?$basic_string@DU?$char_traits@D@std@@V?$allocator@D@2@@1@AAV21@@Z$0 10009a14 f   LocalizerImp.obj
 0001:00008a22       __ehhandler$??$construct@V?$basic_string@DU?$char_traits@D@std@@V?$allocator@D@2@@std@@AAV12@@?$allocator@V?$basic_string@DU?$char_traits@D@std@@V?$allocator@D@2@@std@@@std@@QAEXPAV?$basic_string@DU?$char_traits@D@std@@V?$allocator@D@2@@1@AAV21@@Z 10009a22 f   LocalizerImp.obj
 0001:00008a2c       __unwindfunclet$??$construct@V?$basic_string@DU?$char_traits@D@std@@V?$allocator@D@2@@std@@AAV12@@?$allocator_traits@V?$allocator@V?$basic_string@DU?$char_traits@D@std@@V?$allocator@D@2@@std@@@std@@@std@@SGXAAV?$allocator@V?$basic_string@DU?$char_traits@D@std@@V?$allocator@D@2@@std@@@1@PAV?$basic_string@DU?$char_traits@D@std@@V?$allocator@D@2@@1@AAV31@@Z$0 10009a2c f   LocalizerImp.obj
 0001:00008a3a       __ehhandler$??$construct@V?$basic_string@DU?$char_traits@D@std@@V?$allocator@D@2@@std@@AAV12@@?$allocator_traits@V?$allocator@V?$basic_string@DU?$char_traits@D@std@@V?$allocator@D@2@@std@@@std@@@std@@SGXAAV?$allocator@V?$basic_string@DU?$char_traits@D@std@@V?$allocator@D@2@@std@@@1@PAV?$basic_string@DU?$char_traits@D@std@@V?$allocator@D@2@@1@AAV31@@Z 10009a3a f   LocalizerImp.obj
 0001:00008a44       __unwindfunclet$??$construct@V?$basic_string@DU?$char_traits@D@std@@V?$allocator@D@2@@std@@ABV12@@?$_Wrap_alloc@V?$allocator@V?$basic_string@DU?$char_traits@D@std@@V?$allocator@D@2@@std@@@std@@@std@@QAEXPAV?$basic_string@DU?$char_traits@D@std@@V?$allocator@D@2@@1@ABV21@@Z$0 10009a44 f   LocalizerImp.obj
 0001:00008a52       __ehhandler$??$construct@V?$basic_string@DU?$char_traits@D@std@@V?$allocator@D@2@@std@@ABV12@@?$_Wrap_alloc@V?$allocator@V?$basic_string@DU?$char_traits@D@std@@V?$allocator@D@2@@std@@@std@@@std@@QAEXPAV?$basic_string@DU?$char_traits@D@std@@V?$allocator@D@2@@1@ABV21@@Z 10009a52 f   LocalizerImp.obj
 0001:00008a5c       __unwindfunclet$??$construct@V?$basic_string@DU?$char_traits@D@std@@V?$allocator@D@2@@std@@ABV12@@?$allocator_traits@V?$allocator@V?$basic_string@DU?$char_traits@D@std@@V?$allocator@D@2@@std@@@std@@@std@@SGXAAV?$allocator@V?$basic_string@DU?$char_traits@D@std@@V?$allocator@D@2@@std@@@1@PAV?$basic_string@DU?$char_traits@D@std@@V?$allocator@D@2@@1@ABV31@@Z$0 10009a5c f   LocalizerImp.obj
 0001:00008a6a       __ehhandler$??$construct@V?$basic_string@DU?$char_traits@D@std@@V?$allocator@D@2@@std@@ABV12@@?$allocator_traits@V?$allocator@V?$basic_string@DU?$char_traits@D@std@@V?$allocator@D@2@@std@@@std@@@std@@SGXAAV?$allocator@V?$basic_string@DU?$char_traits@D@std@@V?$allocator@D@2@@std@@@1@PAV?$basic_string@DU?$char_traits@D@std@@V?$allocator@D@2@@1@ABV31@@Z 10009a6a f   LocalizerImp.obj
 0001:00008a74       __unwindfunclet$??$construct@VResEntry@LocalizerImp@@AAV12@@?$allocator@VResEntry@LocalizerImp@@@std@@QAEXPAVResEntry@LocalizerImp@@AAV23@@Z$0 10009a74 f   LocalizerImp.obj
 0001:00008a82       __ehhandler$??$construct@VResEntry@LocalizerImp@@AAV12@@?$allocator@VResEntry@LocalizerImp@@@std@@QAEXPAVResEntry@LocalizerImp@@AAV23@@Z 10009a82 f   LocalizerImp.obj
 0001:00008a8c       __unwindfunclet$??$construct@VResEntry@LocalizerImp@@V12@@?$allocator@VResEntry@LocalizerImp@@@std@@QAEXPAVResEntry@LocalizerImp@@$$QAV23@@Z$0 10009a8c f   LocalizerImp.obj
 0001:00008a9a       __ehhandler$??$construct@VResEntry@LocalizerImp@@V12@@?$allocator@VResEntry@LocalizerImp@@@std@@QAEXPAVResEntry@LocalizerImp@@$$QAV23@@Z 10009a9a f   LocalizerImp.obj
 0001:00008aa4       __unwindfunclet$?Allocator@LocalizerImp@@SGPAU_HMEMPOOL@@XZ$0 10009aa4 f   LocalizerImp.obj
 0001:00008ab2       __ehhandler$?Allocator@LocalizerImp@@SGPAU_HMEMPOOL@@XZ 10009ab2 f   LocalizerImp.obj
 0001:00008abc       __unwindfunclet$?InternalResLoad@LocalizerImp@@AAE_NPBDP6GPAVResource@1@0@Z@Z$0 10009abc f   LocalizerImp.obj
 0001:00008ac4       __unwindfunclet$?InternalResLoad@LocalizerImp@@AAE_NPBDP6GPAVResource@1@0@Z@Z$1 10009ac4 f   LocalizerImp.obj
 0001:00008acc       __ehhandler$?InternalResLoad@LocalizerImp@@AAE_NPBDP6GPAVResource@1@0@Z@Z 10009acc f   LocalizerImp.obj
 0001:00008ad6       __unwindfunclet$?ListFiles@@YGXAAV?$vector@V?$basic_string@DU?$char_traits@D@std@@V?$allocator@D@2@@std@@V?$allocator@V?$basic_string@DU?$char_traits@D@std@@V?$allocator@D@2@@std@@@2@@std@@PBD1@Z$0 10009ad6 f   LocalizerImp.obj
 0001:00008ade       __unwindfunclet$?ListFiles@@YGXAAV?$vector@V?$basic_string@DU?$char_traits@D@std@@V?$allocator@D@2@@std@@V?$allocator@V?$basic_string@DU?$char_traits@D@std@@V?$allocator@D@2@@std@@@2@@std@@PBD1@Z$1 10009ade f   LocalizerImp.obj
 0001:00008ae6       __ehhandler$?ListFiles@@YGXAAV?$vector@V?$basic_string@DU?$char_traits@D@std@@V?$allocator@D@2@@std@@V?$allocator@V?$basic_string@DU?$char_traits@D@std@@V?$allocator@D@2@@std@@@2@@std@@PBD1@Z 10009ae6 f   LocalizerImp.obj
 0001:00008af0       __unwindfunclet$?ResLoadFolder@LocalizerImp@@QAE?AV?$vector@V?$basic_string@DU?$char_traits@D@std@@V?$allocator@D@2@@std@@V?$allocator@V?$basic_string@DU?$char_traits@D@std@@V?$allocator@D@2@@std@@@2@@std@@PBD@Z$0 10009af0 f   LocalizerImp.obj
 0001:00008af8       __unwindfunclet$?ResLoadFolder@LocalizerImp@@QAE?AV?$vector@V?$basic_string@DU?$char_traits@D@std@@V?$allocator@D@2@@std@@V?$allocator@V?$basic_string@DU?$char_traits@D@std@@V?$allocator@D@2@@std@@@2@@std@@PBD@Z$1 10009af8 f   LocalizerImp.obj
 0001:00008b00       __unwindfunclet$?ResLoadFolder@LocalizerImp@@QAE?AV?$vector@V?$basic_string@DU?$char_traits@D@std@@V?$allocator@D@2@@std@@V?$allocator@V?$basic_string@DU?$char_traits@D@std@@V?$allocator@D@2@@std@@@2@@std@@PBD@Z$2 10009b00 f   LocalizerImp.obj
 0001:00008b19       __ehhandler$?ResLoadFolder@LocalizerImp@@QAE?AV?$vector@V?$basic_string@DU?$char_traits@D@std@@V?$allocator@D@2@@std@@V?$allocator@V?$basic_string@DU?$char_traits@D@std@@V?$allocator@D@2@@std@@@2@@std@@PBD@Z 10009b19 f   LocalizerImp.obj
 0001:00008b23       __ehhandler$?_Reallocate@?$vector@V?$basic_string@DU?$char_traits@D@std@@V?$allocator@D@2@@std@@V?$allocator@V?$basic_string@DU?$char_traits@D@std@@V?$allocator@D@2@@std@@@2@@std@@IAEXI@Z 10009b23 f   LocalizerImp.obj
 0001:00008b2d       __ehhandler$?_Reallocate@?$vector@VResEntry@LocalizerImp@@V?$allocator@VResEntry@LocalizerImp@@@std@@@std@@IAEXI@Z 10009b2d f   LocalizerImp.obj
 0001:00008b37       __unwindfunclet$?add_ref@sp_counted_base@detail@boost@@QAEXXZ$0 10009b37 f   LocalizerImp.obj
 0001:00008b3f       __unwindfunclet$?add_ref@sp_counted_base@detail@boost@@QAEXXZ$1 10009b3f f   LocalizerImp.obj
 0001:00008b47       __ehhandler$?add_ref@sp_counted_base@detail@boost@@QAEXXZ 10009b47 f   LocalizerImp.obj
 0001:00008b51       __unwindfunclet$?construct@?$allocator@V?$basic_string@DU?$char_traits@D@std@@V?$allocator@D@2@@std@@@std@@QAEXPAV?$basic_string@DU?$char_traits@D@std@@V?$allocator@D@2@@2@ABV32@@Z$0 10009b51 f   LocalizerImp.obj
 0001:00008b5f       __ehhandler$?construct@?$allocator@V?$basic_string@DU?$char_traits@D@std@@V?$allocator@D@2@@std@@@std@@QAEXPAV?$basic_string@DU?$char_traits@D@std@@V?$allocator@D@2@@2@ABV32@@Z 10009b5f f   LocalizerImp.obj
 0001:00008b69       __unwindfunclet$?construct@?$allocator@VResEntry@LocalizerImp@@@std@@QAEXPAVResEntry@LocalizerImp@@ABV34@@Z$0 10009b69 f   LocalizerImp.obj
 0001:00008b77       __ehhandler$?construct@?$allocator@VResEntry@LocalizerImp@@@std@@QAEXPAVResEntry@LocalizerImp@@ABV34@@Z 10009b77 f   LocalizerImp.obj
 0001:00008b81       __unwindfunclet$?push_back@?$vector@V?$basic_string@DU?$char_traits@D@std@@V?$allocator@D@2@@std@@V?$allocator@V?$basic_string@DU?$char_traits@D@std@@V?$allocator@D@2@@std@@@2@@std@@QAEXABV?$basic_string@DU?$char_traits@D@std@@V?$allocator@D@2@@2@@Z$0 10009b81 f   LocalizerImp.obj
 0001:00008b8f       __unwindfunclet$?push_back@?$vector@V?$basic_string@DU?$char_traits@D@std@@V?$allocator@D@2@@std@@V?$allocator@V?$basic_string@DU?$char_traits@D@std@@V?$allocator@D@2@@std@@@2@@std@@QAEXABV?$basic_string@DU?$char_traits@D@std@@V?$allocator@D@2@@2@@Z$1 10009b8f f   LocalizerImp.obj
 0001:00008b9d       __ehhandler$?push_back@?$vector@V?$basic_string@DU?$char_traits@D@std@@V?$allocator@D@2@@std@@V?$allocator@V?$basic_string@DU?$char_traits@D@std@@V?$allocator@D@2@@std@@@2@@std@@QAEXABV?$basic_string@DU?$char_traits@D@std@@V?$allocator@D@2@@2@@Z 10009b9d f   LocalizerImp.obj
 0001:00008ba7       __unwindfunclet$??$?HDU?$char_traits@D@std@@V?$allocator@D@1@@std@@YG?AV?$basic_string@DU?$char_traits@D@std@@V?$allocator@D@2@@0@ABV10@PBD@Z$0 10009ba7 f   LocalizerTxt.obj
 0001:00008bc0       __ehhandler$??$?HDU?$char_traits@D@std@@V?$allocator@D@1@@std@@YG?AV?$basic_string@DU?$char_traits@D@std@@V?$allocator@D@2@@0@ABV10@PBD@Z 10009bc0 f   LocalizerTxt.obj
 0001:00008bca       __unwindfunclet$??0LocalizerResourceTxt@@AAE@PBD@Z$0 10009bca f   LocalizerTxt.obj
 0001:00008bd2       __unwindfunclet$??0LocalizerResourceTxt@@AAE@PBD@Z$1 10009bd2 f   LocalizerTxt.obj
 0001:00008bdd       __unwindfunclet$??0LocalizerResourceTxt@@AAE@PBD@Z$2 10009bdd f   LocalizerTxt.obj
 0001:00008be8       __ehhandler$??0LocalizerResourceTxt@@AAE@PBD@Z 10009be8 f   LocalizerTxt.obj
 0001:00008bf2       __unwindfunclet$??1LocalizerResourceTxt@@UAE@XZ$0 10009bf2 f   LocalizerTxt.obj
 0001:00008bfa       __unwindfunclet$??1LocalizerResourceTxt@@UAE@XZ$1 10009bfa f   LocalizerTxt.obj
 0001:00008c05       __unwindfunclet$??1LocalizerResourceTxt@@UAE@XZ$2 10009c05 f   LocalizerTxt.obj
 0001:00008c10       __unwindfunclet$??1LocalizerResourceTxt@@UAE@XZ$3 10009c10 f   LocalizerTxt.obj
 0001:00008c1b       __ehhandler$??1LocalizerResourceTxt@@UAE@XZ 10009c1b f   LocalizerTxt.obj
 0001:00008c25       __unwindfunclet$?Load@LocalizerResourceTxt@@SGPAVResource@LocalizerImp@@PBD@Z$0 10009c25 f   LocalizerTxt.obj
 0001:00008c31       __unwindfunclet$?Load@LocalizerResourceTxt@@SGPAVResource@LocalizerImp@@PBD@Z$1 10009c31 f   LocalizerTxt.obj
 0001:00008c3e       __unwindfunclet$?Load@LocalizerResourceTxt@@SGPAVResource@LocalizerImp@@PBD@Z$2 10009c3e f   LocalizerTxt.obj
 0001:00008c49       __unwindfunclet$?Load@LocalizerResourceTxt@@SGPAVResource@LocalizerImp@@PBD@Z$3 10009c49 f   LocalizerTxt.obj
 0001:00008c54       __unwindfunclet$?Load@LocalizerResourceTxt@@SGPAVResource@LocalizerImp@@PBD@Z$4 10009c54 f   LocalizerTxt.obj
 0001:00008c5f       __unwindfunclet$?Load@LocalizerResourceTxt@@SGPAVResource@LocalizerImp@@PBD@Z$5 10009c5f f   LocalizerTxt.obj
 0001:00008c6a       __unwindfunclet$?Load@LocalizerResourceTxt@@SGPAVResource@LocalizerImp@@PBD@Z$6 10009c6a f   LocalizerTxt.obj
 0001:00008c75       __ehhandler$?Load@LocalizerResourceTxt@@SGPAVResource@LocalizerImp@@PBD@Z 10009c75 f   LocalizerTxt.obj
 0001:00008c7f       __unwindfunclet$?Save@LocalizerResourceTxt@@QAE_NPBD@Z$0 10009c7f f   LocalizerTxt.obj
 0001:00008c8b       __ehhandler$?Save@LocalizerResourceTxt@@QAE_NPBD@Z 10009c8b f   LocalizerTxt.obj
 0001:00008c95       __ehhandler$?_Reallocate@?$vector@U?$pair@HULine@LocalizerResourceTxt@@@std@@V?$mempool_alloc@U?$pair@HULine@LocalizerResourceTxt@@@std@@@@@std@@IAEXI@Z 10009c95 f   LocalizerTxt.obj
 0001:00008c9f       __ehhandler$?_Reallocate@?$vector@URange@LocalizerResourceTxt@@V?$mempool_alloc@URange@LocalizerResourceTxt@@@@@std@@IAEXI@Z 10009c9f f   LocalizerTxt.obj
 0001:00008ca9       __unwindfunclet$??0LocalizerResourceUCS@@AAE@PBDII@Z$0 10009ca9 f   LocalizerUCS.obj
 0001:00008cb1       __unwindfunclet$??0LocalizerResourceUCS@@AAE@PBDII@Z$1 10009cb1 f   LocalizerUCS.obj
 0001:00008cbc       __ehhandler$??0LocalizerResourceUCS@@AAE@PBDII@Z 10009cbc f   LocalizerUCS.obj
 0001:00008cc6       __unwindfunclet$??1LocalizerResourceUCS@@UAE@XZ$0 10009cc6 f   LocalizerUCS.obj
 0001:00008cce       __unwindfunclet$??1LocalizerResourceUCS@@UAE@XZ$1 10009cce f   LocalizerUCS.obj
 0001:00008cd9       __ehhandler$??1LocalizerResourceUCS@@UAE@XZ 10009cd9 f   LocalizerUCS.obj
 0001:00008ce3       __unwindfunclet$?Create@FileBuffer@?A0xa493ca04@@SGPAV12@PBD@Z$0 10009ce3 f   LocalizerUCS.obj
 0001:00008cef       __unwindfunclet$?Create@FileBuffer@?A0xa493ca04@@SGPAV12@PBD@Z$1 10009cef f   LocalizerUCS.obj
 0001:00008cf9       __unwindfunclet$?Create@FileBuffer@?A0xa493ca04@@SGPAV12@PBD@Z$2 10009cf9 f   LocalizerUCS.obj
 0001:00008d01       __ehhandler$?Create@FileBuffer@?A0xa493ca04@@SGPAV12@PBD@Z 10009d01 f   LocalizerUCS.obj
 0001:00008d0b       __unwindfunclet$?Load@LocalizerResourceUCS@@SGPAVResource@LocalizerImp@@PBD@Z$0 10009d0b f   LocalizerUCS.obj
 0001:00008d13       __unwindfunclet$?Load@LocalizerResourceUCS@@SGPAVResource@LocalizerImp@@PBD@Z$1 10009d13 f   LocalizerUCS.obj
 0001:00008d1d       __unwindfunclet$?Load@LocalizerResourceUCS@@SGPAVResource@LocalizerImp@@PBD@Z$2 10009d1d f   LocalizerUCS.obj
 0001:00008d25       __ehhandler$?Load@LocalizerResourceUCS@@SGPAVResource@LocalizerImp@@PBD@Z 10009d25 f   LocalizerUCS.obj
 0001:00008d2f       ??__E?_Generic_object@?$_Error_objects@H@std@@2V_Generic_error_category@2@A@@YAXXZ 10009d2f f   pch.obj
 0001:00008d3b       ??__E?_Iostream_object@?$_Error_objects@H@std@@2V_Iostream_error_category@2@A@@YAXXZ 10009d3b f   pch.obj
 0001:00008d47       ??__E?_System_object@?$_Error_objects@H@std@@2V_System_error_category@2@A@@YAXXZ 10009d47 f   pch.obj
 0001:00008d53       ??__E?id@?$num_put@DV?$back_insert_iterator@V?$basic_string@DU?$char_traits@D@std@@V?$allocator@D@2@@std@@@std@@@std@@2V0locale@2@A@@YAXXZ 10009d53 f   pch.obj
 0001:00008d61       ??__E?id@?$num_put@_WV?$back_insert_iterator@V?$basic_string@_WU?$char_traits@_W@std@@V?$allocator@_W@2@@std@@@std@@@std@@2V0locale@2@A@@YAXXZ 10009d61 f   pch.obj
 0001:00008d6f       ??__Fs_pool@?1??Allocator@LocalizerImp@@SGPAU_HMEMPOOL@@XZ@YAXXZ 10009d6f f   LocalizerImp.obj
 0001:00008d7a       ??__F?_Generic_object@?$_Error_objects@H@std@@2V_Generic_error_category@2@A@@YAXXZ 10009d7a f   pch.obj
 0001:00008d85       ??__F?_Iostream_object@?$_Error_objects@H@std@@2V_Iostream_error_category@2@A@@YAXXZ 10009d85 f   pch.obj
 0001:00008d90       ??__F?_System_object@?$_Error_objects@H@std@@2V_System_error_category@2@A@@YAXXZ 10009d90 f   pch.obj
 0002:000001ac       ?_Generic_object$initializer$@?$_Error_objects@H@std@@2P6AXXZA 1000a1ac     pch.obj
 0002:000001b0       ?_Iostream_object$initializer$@?$_Error_objects@H@std@@2P6AXXZA 1000a1b0     pch.obj
 0002:000001b4       ?_System_object$initializer$@?$_Error_objects@H@std@@2P6AXXZA 1000a1b4     pch.obj
 0002:000001b8       ?id$initializer$@?$num_put@DV?$back_insert_iterator@V?$basic_string@DU?$char_traits@D@std@@V?$allocator@D@2@@std@@@std@@@std@@2P6AXXZA 1000a1b8     pch.obj
 0002:000001bc       ?id$initializer$@?$num_put@_WV?$back_insert_iterator@V?$basic_string@_WU?$char_traits@_W@std@@V?$allocator@_W@2@@std@@@std@@@std@@2P6AXXZA 1000a1bc     pch.obj
 0002:000001c8       _pcinit                    1000a1c8     MSVCRT:crtdll.obj
 0002:000001cc       _pinit                     1000a1cc     MSVCRT:atonexit.obj
 0002:000003a0       _TOKEN_FILERANGE           1000a3a0     LocalizerTxt.obj
 0002:000003ac       _TOKEN_RANGE_START         1000a3ac     LocalizerTxt.obj
 0002:000003b8       _TOKEN_RANGE_END           1000a3b8     LocalizerTxt.obj
 0002:000003c4       _TOKEN_COMMENT             1000a3c4     LocalizerTxt.obj
 0002:000009c8       _GS_ExceptionPointers      1000a9c8     MSVCRT:gs_report.obj
 0002:00000e98       __catchsym$?_Copy@?$basic_string@DU?$char_traits@D@std@@V?$allocator@D@2@@std@@QAEXII@Z$5 1000ae98     Localizer.obj
 0002:00000ea8       __catchsym$?_Copy@?$basic_string@DU?$char_traits@D@std@@V?$allocator@D@2@@std@@QAEXII@Z$4 1000aea8     Localizer.obj
 0002:00000eb8       __unwindtable$?_Copy@?$basic_string@DU?$char_traits@D@std@@V?$allocator@D@2@@std@@QAEXII@Z 1000aeb8     Localizer.obj
 0002:00000ed8       __ehfuncinfo$?_Copy@?$basic_string@DU?$char_traits@D@std@@V?$allocator@D@2@@std@@QAEXII@Z 1000aed8     Localizer.obj
 0002:00000efc       __tryblocktable$?_Copy@?$basic_string@DU?$char_traits@D@std@@V?$allocator@D@2@@std@@QAEXII@Z 1000aefc     Localizer.obj
 0002:00000f24       __catchsym$?_Copy@?$basic_string@_WU?$char_traits@_W@std@@V?$allocator@_W@2@@std@@QAEXII@Z$5 1000af24     Localizer.obj
 0002:00000f34       __catchsym$?_Copy@?$basic_string@_WU?$char_traits@_W@std@@V?$allocator@_W@2@@std@@QAEXII@Z$4 1000af34     Localizer.obj
 0002:00000f44       __unwindtable$?_Copy@?$basic_string@_WU?$char_traits@_W@std@@V?$allocator@_W@2@@std@@QAEXII@Z 1000af44     Localizer.obj
 0002:00000f64       __ehfuncinfo$?_Copy@?$basic_string@_WU?$char_traits@_W@std@@V?$allocator@_W@2@@std@@QAEXII@Z 1000af64     Localizer.obj
 0002:00000f88       __tryblocktable$?_Copy@?$basic_string@_WU?$char_traits@_W@std@@V?$allocator@_W@2@@std@@QAEXII@Z 1000af88     Localizer.obj
 0002:00000fb0       __unwindtable$?CheckString@Localizer@@SG_NPB_WK0@Z 1000afb0     Localizer.obj
 0002:00000fc0       __ehfuncinfo$?CheckString@Localizer@@SG_NPB_WK0@Z 1000afc0     Localizer.obj
 0002:00000fe4       __unwindtable$?add_ref@sp_counted_base@detail@boost@@QAEXXZ 1000afe4     LocalizerImp.obj
 0002:00000ff4       __ehfuncinfo$?add_ref@sp_counted_base@detail@boost@@QAEXXZ 1000aff4     LocalizerImp.obj
 0002:00001018       __unwindtable$?Allocator@LocalizerImp@@SGPAU_HMEMPOOL@@XZ 1000b018     LocalizerImp.obj
 0002:00001020       __ehfuncinfo$?Allocator@LocalizerImp@@SGPAU_HMEMPOOL@@XZ 1000b020     LocalizerImp.obj
 0002:00001044       __unwindtable$?ResLoadFolder@LocalizerImp@@QAE?AV?$vector@V?$basic_string@DU?$char_traits@D@std@@V?$allocator@D@2@@std@@V?$allocator@V?$basic_string@DU?$char_traits@D@std@@V?$allocator@D@2@@std@@@2@@std@@PBD@Z 1000b044     LocalizerImp.obj
 0002:0000105c       __ehfuncinfo$?ResLoadFolder@LocalizerImp@@QAE?AV?$vector@V?$basic_string@DU?$char_traits@D@std@@V?$allocator@D@2@@std@@V?$allocator@V?$basic_string@DU?$char_traits@D@std@@V?$allocator@D@2@@std@@@2@@std@@PBD@Z 1000b05c     LocalizerImp.obj
 0002:00001080       __unwindtable$?construct@?$allocator@VResEntry@LocalizerImp@@@std@@QAEXPAVResEntry@LocalizerImp@@ABV34@@Z 1000b080     LocalizerImp.obj
 0002:00001088       __ehfuncinfo$?construct@?$allocator@VResEntry@LocalizerImp@@@std@@QAEXPAVResEntry@LocalizerImp@@ABV34@@Z 1000b088     LocalizerImp.obj
 0002:000010ac       __catchsym$?_Reallocate@?$vector@VResEntry@LocalizerImp@@V?$allocator@VResEntry@LocalizerImp@@@std@@@std@@IAEXI@Z$2 1000b0ac     LocalizerImp.obj
 0002:000010bc       __unwindtable$?_Reallocate@?$vector@VResEntry@LocalizerImp@@V?$allocator@VResEntry@LocalizerImp@@@std@@@std@@IAEXI@Z 1000b0bc     LocalizerImp.obj
 0002:000010cc       __tryblocktable$?_Reallocate@?$vector@VResEntry@LocalizerImp@@V?$allocator@VResEntry@LocalizerImp@@@std@@@std@@IAEXI@Z 1000b0cc     LocalizerImp.obj
 0002:000010e0       __ehfuncinfo$?_Reallocate@?$vector@VResEntry@LocalizerImp@@V?$allocator@VResEntry@LocalizerImp@@@std@@@std@@IAEXI@Z 1000b0e0     LocalizerImp.obj
 0002:00001104       __unwindtable$?InternalResLoad@LocalizerImp@@AAE_NPBDP6GPAVResource@1@0@Z@Z 1000b104     LocalizerImp.obj
 0002:00001114       __ehfuncinfo$?InternalResLoad@LocalizerImp@@AAE_NPBDP6GPAVResource@1@0@Z@Z 1000b114     LocalizerImp.obj
 0002:00001138       __unwindtable$?ListFiles@@YGXAAV?$vector@V?$basic_string@DU?$char_traits@D@std@@V?$allocator@D@2@@std@@V?$allocator@V?$basic_string@DU?$char_traits@D@std@@V?$allocator@D@2@@std@@@2@@std@@PBD1@Z 1000b138     LocalizerImp.obj
 0002:00001148       __ehfuncinfo$?ListFiles@@YGXAAV?$vector@V?$basic_string@DU?$char_traits@D@std@@V?$allocator@D@2@@std@@V?$allocator@V?$basic_string@DU?$char_traits@D@std@@V?$allocator@D@2@@std@@@2@@std@@PBD1@Z 1000b148     LocalizerImp.obj
 0002:0000116c       __unwindtable$?construct@?$allocator@V?$basic_string@DU?$char_traits@D@std@@V?$allocator@D@2@@std@@@std@@QAEXPAV?$basic_string@DU?$char_traits@D@std@@V?$allocator@D@2@@2@ABV32@@Z 1000b16c     LocalizerImp.obj
 0002:00001174       __ehfuncinfo$?construct@?$allocator@V?$basic_string@DU?$char_traits@D@std@@V?$allocator@D@2@@std@@@std@@QAEXPAV?$basic_string@DU?$char_traits@D@std@@V?$allocator@D@2@@2@ABV32@@Z 1000b174     LocalizerImp.obj
 0002:00001198       __unwindtable$?push_back@?$vector@V?$basic_string@DU?$char_traits@D@std@@V?$allocator@D@2@@std@@V?$allocator@V?$basic_string@DU?$char_traits@D@std@@V?$allocator@D@2@@std@@@2@@std@@QAEXABV?$basic_string@DU?$char_traits@D@std@@V?$allocator@D@2@@2@@Z 1000b198     LocalizerImp.obj
 0002:000011a8       __ehfuncinfo$?push_back@?$vector@V?$basic_string@DU?$char_traits@D@std@@V?$allocator@D@2@@std@@V?$allocator@V?$basic_string@DU?$char_traits@D@std@@V?$allocator@D@2@@std@@@2@@std@@QAEXABV?$basic_string@DU?$char_traits@D@std@@V?$allocator@D@2@@2@@Z 1000b1a8     LocalizerImp.obj
 0002:000011cc       __catchsym$?_Reallocate@?$vector@V?$basic_string@DU?$char_traits@D@std@@V?$allocator@D@2@@std@@V?$allocator@V?$basic_string@DU?$char_traits@D@std@@V?$allocator@D@2@@std@@@2@@std@@IAEXI@Z$2 1000b1cc     LocalizerImp.obj
 0002:000011dc       __unwindtable$?_Reallocate@?$vector@V?$basic_string@DU?$char_traits@D@std@@V?$allocator@D@2@@std@@V?$allocator@V?$basic_string@DU?$char_traits@D@std@@V?$allocator@D@2@@std@@@2@@std@@IAEXI@Z 1000b1dc     LocalizerImp.obj
 0002:000011ec       __tryblocktable$?_Reallocate@?$vector@V?$basic_string@DU?$char_traits@D@std@@V?$allocator@D@2@@std@@V?$allocator@V?$basic_string@DU?$char_traits@D@std@@V?$allocator@D@2@@std@@@2@@std@@IAEXI@Z 1000b1ec     LocalizerImp.obj
 0002:00001200       __ehfuncinfo$?_Reallocate@?$vector@V?$basic_string@DU?$char_traits@D@std@@V?$allocator@D@2@@std@@V?$allocator@V?$basic_string@DU?$char_traits@D@std@@V?$allocator@D@2@@std@@@2@@std@@IAEXI@Z 1000b200     LocalizerImp.obj
 0002:00001224       __unwindtable$??$construct@V?$basic_string@DU?$char_traits@D@std@@V?$allocator@D@2@@std@@AAV12@@?$_Wrap_alloc@V?$allocator@V?$basic_string@DU?$char_traits@D@std@@V?$allocator@D@2@@std@@@std@@@std@@QAEXPAV?$basic_string@DU?$char_traits@D@std@@V?$allocator@D@2@@1@AAV21@@Z 1000b224     LocalizerImp.obj
 0002:0000122c       __ehfuncinfo$??$construct@V?$basic_string@DU?$char_traits@D@std@@V?$allocator@D@2@@std@@AAV12@@?$_Wrap_alloc@V?$allocator@V?$basic_string@DU?$char_traits@D@std@@V?$allocator@D@2@@std@@@std@@@std@@QAEXPAV?$basic_string@DU?$char_traits@D@std@@V?$allocator@D@2@@1@AAV21@@Z 1000b22c     LocalizerImp.obj
 0002:00001250       __unwindtable$??$construct@V?$basic_string@DU?$char_traits@D@std@@V?$allocator@D@2@@std@@ABV12@@?$_Wrap_alloc@V?$allocator@V?$basic_string@DU?$char_traits@D@std@@V?$allocator@D@2@@std@@@std@@@std@@QAEXPAV?$basic_string@DU?$char_traits@D@std@@V?$allocator@D@2@@1@ABV21@@Z 1000b250     LocalizerImp.obj
 0002:00001258       __ehfuncinfo$??$construct@V?$basic_string@DU?$char_traits@D@std@@V?$allocator@D@2@@std@@ABV12@@?$_Wrap_alloc@V?$allocator@V?$basic_string@DU?$char_traits@D@std@@V?$allocator@D@2@@std@@@std@@@std@@QAEXPAV?$basic_string@DU?$char_traits@D@std@@V?$allocator@D@2@@1@ABV21@@Z 1000b258     LocalizerImp.obj
 0002:0000127c       __unwindtable$??$construct@V?$basic_string@DU?$char_traits@D@std@@V?$allocator@D@2@@std@@AAV12@@?$allocator_traits@V?$allocator@V?$basic_string@DU?$char_traits@D@std@@V?$allocator@D@2@@std@@@std@@@std@@SGXAAV?$allocator@V?$basic_string@DU?$char_traits@D@std@@V?$allocator@D@2@@std@@@1@PAV?$basic_string@DU?$char_traits@D@std@@V?$allocator@D@2@@1@AAV31@@Z 1000b27c     LocalizerImp.obj
 0002:00001284       __ehfuncinfo$??$construct@V?$basic_string@DU?$char_traits@D@std@@V?$allocator@D@2@@std@@AAV12@@?$allocator_traits@V?$allocator@V?$basic_string@DU?$char_traits@D@std@@V?$allocator@D@2@@std@@@std@@@std@@SGXAAV?$allocator@V?$basic_string@DU?$char_traits@D@std@@V?$allocator@D@2@@std@@@1@PAV?$basic_string@DU?$char_traits@D@std@@V?$allocator@D@2@@1@AAV31@@Z 1000b284     LocalizerImp.obj
 0002:000012a8       __unwindtable$??$construct@V?$basic_string@DU?$char_traits@D@std@@V?$allocator@D@2@@std@@ABV12@@?$allocator_traits@V?$allocator@V?$basic_string@DU?$char_traits@D@std@@V?$allocator@D@2@@std@@@std@@@std@@SGXAAV?$allocator@V?$basic_string@DU?$char_traits@D@std@@V?$allocator@D@2@@std@@@1@PAV?$basic_string@DU?$char_traits@D@std@@V?$allocator@D@2@@1@ABV31@@Z 1000b2a8     LocalizerImp.obj
 0002:000012b0       __ehfuncinfo$??$construct@V?$basic_string@DU?$char_traits@D@std@@V?$allocator@D@2@@std@@ABV12@@?$allocator_traits@V?$allocator@V?$basic_string@DU?$char_traits@D@std@@V?$allocator@D@2@@std@@@std@@@std@@SGXAAV?$allocator@V?$basic_string@DU?$char_traits@D@std@@V?$allocator@D@2@@std@@@1@PAV?$basic_string@DU?$char_traits@D@std@@V?$allocator@D@2@@1@ABV31@@Z 1000b2b0     LocalizerImp.obj
 0002:000012d4       __catchsym$??$?0PAVResource@LocalizerImp@@U?$checked_deleter@VResource@LocalizerImp@@@boost@@@shared_count@detail@boost@@QAE@PAVResource@LocalizerImp@@U?$checked_deleter@VResource@LocalizerImp@@@2@@Z$3 1000b2d4     LocalizerImp.obj
 0002:000012e4       __unwindtable$??$?0PAVResource@LocalizerImp@@U?$checked_deleter@VResource@LocalizerImp@@@boost@@@shared_count@detail@boost@@QAE@PAVResource@LocalizerImp@@U?$checked_deleter@VResource@LocalizerImp@@@2@@Z 1000b2e4     LocalizerImp.obj
 0002:000012f4       __tryblocktable$??$?0PAVResource@LocalizerImp@@U?$checked_deleter@VResource@LocalizerImp@@@boost@@@shared_count@detail@boost@@QAE@PAVResource@LocalizerImp@@U?$checked_deleter@VResource@LocalizerImp@@@2@@Z 1000b2f4     LocalizerImp.obj
 0002:00001308       __ehfuncinfo$??$?0PAVResource@LocalizerImp@@U?$checked_deleter@VResource@LocalizerImp@@@boost@@@shared_count@detail@boost@@QAE@PAVResource@LocalizerImp@@U?$checked_deleter@VResource@LocalizerImp@@@2@@Z 1000b308     LocalizerImp.obj
 0002:0000132c       __unwindtable$??$construct@VResEntry@LocalizerImp@@AAV12@@?$allocator@VResEntry@LocalizerImp@@@std@@QAEXPAVResEntry@LocalizerImp@@AAV23@@Z 1000b32c     LocalizerImp.obj
 0002:00001334       __ehfuncinfo$??$construct@VResEntry@LocalizerImp@@AAV12@@?$allocator@VResEntry@LocalizerImp@@@std@@QAEXPAVResEntry@LocalizerImp@@AAV23@@Z 1000b334     LocalizerImp.obj
 0002:00001358       __unwindtable$??$construct@V?$basic_string@DU?$char_traits@D@std@@V?$allocator@D@2@@std@@AAV12@@?$allocator@V?$basic_string@DU?$char_traits@D@std@@V?$allocator@D@2@@std@@@std@@QAEXPAV?$basic_string@DU?$char_traits@D@std@@V?$allocator@D@2@@1@AAV21@@Z 1000b358     LocalizerImp.obj
 0002:00001360       __ehfuncinfo$??$construct@V?$basic_string@DU?$char_traits@D@std@@V?$allocator@D@2@@std@@AAV12@@?$allocator@V?$basic_string@DU?$char_traits@D@std@@V?$allocator@D@2@@std@@@std@@QAEXPAV?$basic_string@DU?$char_traits@D@std@@V?$allocator@D@2@@1@AAV21@@Z 1000b360     LocalizerImp.obj
 0002:00001384       __catchsym$??$_Uninit_move@PAVResEntry@LocalizerImp@@PAV12@V?$allocator@VResEntry@LocalizerImp@@@std@@V12@@std@@YGPAVResEntry@LocalizerImp@@PAV12@00AAU?$_Wrap_alloc@V?$allocator@VResEntry@LocalizerImp@@@std@@@0@0U_Nonscalar_ptr_iterator_tag@0@@Z$2 1000b384     LocalizerImp.obj
 0002:00001394       __unwindtable$??$_Uninit_move@PAVResEntry@LocalizerImp@@PAV12@V?$allocator@VResEntry@LocalizerImp@@@std@@V12@@std@@YGPAVResEntry@LocalizerImp@@PAV12@00AAU?$_Wrap_alloc@V?$allocator@VResEntry@LocalizerImp@@@std@@@0@0U_Nonscalar_ptr_iterator_tag@0@@Z 1000b394     LocalizerImp.obj
 0002:000013a4       __tryblocktable$??$_Uninit_move@PAVResEntry@LocalizerImp@@PAV12@V?$allocator@VResEntry@LocalizerImp@@@std@@V12@@std@@YGPAVResEntry@LocalizerImp@@PAV12@00AAU?$_Wrap_alloc@V?$allocator@VResEntry@LocalizerImp@@@std@@@0@0U_Nonscalar_ptr_iterator_tag@0@@Z 1000b3a4     LocalizerImp.obj
 0002:000013b8       __ehfuncinfo$??$_Uninit_move@PAVResEntry@LocalizerImp@@PAV12@V?$allocator@VResEntry@LocalizerImp@@@std@@V12@@std@@YGPAVResEntry@LocalizerImp@@PAV12@00AAU?$_Wrap_alloc@V?$allocator@VResEntry@LocalizerImp@@@std@@@0@0U_Nonscalar_ptr_iterator_tag@0@@Z 1000b3b8     LocalizerImp.obj
 0002:000013dc       __unwindtable$??$construct@VResEntry@LocalizerImp@@V12@@?$allocator@VResEntry@LocalizerImp@@@std@@QAEXPAVResEntry@LocalizerImp@@$$QAV23@@Z 1000b3dc     LocalizerImp.obj
 0002:000013e4       __ehfuncinfo$??$construct@VResEntry@LocalizerImp@@V12@@?$allocator@VResEntry@LocalizerImp@@@std@@QAEXPAVResEntry@LocalizerImp@@$$QAV23@@Z 1000b3e4     LocalizerImp.obj
 0002:0000145c       __unwindtable$??0LocalizerResourceTxt@@AAE@PBD@Z 1000b45c     LocalizerTxt.obj
 0002:00001474       __ehfuncinfo$??0LocalizerResourceTxt@@AAE@PBD@Z 1000b474     LocalizerTxt.obj
 0002:00001498       __ehfuncinfo$?Load@LocalizerResourceTxt@@SGPAVResource@LocalizerImp@@PBD@Z 1000b498     LocalizerTxt.obj
 0002:000014bc       __unwindtable$?Load@LocalizerResourceTxt@@SGPAVResource@LocalizerImp@@PBD@Z 1000b4bc     LocalizerTxt.obj
 0002:000014f4       __unwindtable$??1LocalizerResourceTxt@@UAE@XZ 1000b4f4     LocalizerTxt.obj
 0002:00001514       __ehfuncinfo$??1LocalizerResourceTxt@@UAE@XZ 1000b514     LocalizerTxt.obj
 0002:00001538       __unwindtable$?Save@LocalizerResourceTxt@@QAE_NPBD@Z 1000b538     LocalizerTxt.obj
 0002:00001540       __ehfuncinfo$?Save@LocalizerResourceTxt@@QAE_NPBD@Z 1000b540     LocalizerTxt.obj
 0002:00001564       __catchsym$?_Reallocate@?$vector@U?$pair@HULine@LocalizerResourceTxt@@@std@@V?$mempool_alloc@U?$pair@HULine@LocalizerResourceTxt@@@std@@@@@std@@IAEXI@Z$2 1000b564     LocalizerTxt.obj
 0002:00001574       __unwindtable$?_Reallocate@?$vector@U?$pair@HULine@LocalizerResourceTxt@@@std@@V?$mempool_alloc@U?$pair@HULine@LocalizerResourceTxt@@@std@@@@@std@@IAEXI@Z 1000b574     LocalizerTxt.obj
 0002:00001584       __tryblocktable$?_Reallocate@?$vector@U?$pair@HULine@LocalizerResourceTxt@@@std@@V?$mempool_alloc@U?$pair@HULine@LocalizerResourceTxt@@@std@@@@@std@@IAEXI@Z 1000b584     LocalizerTxt.obj
 0002:00001598       __ehfuncinfo$?_Reallocate@?$vector@U?$pair@HULine@LocalizerResourceTxt@@@std@@V?$mempool_alloc@U?$pair@HULine@LocalizerResourceTxt@@@std@@@@@std@@IAEXI@Z 1000b598     LocalizerTxt.obj
 0002:000015bc       __catchsym$?_Reallocate@?$vector@URange@LocalizerResourceTxt@@V?$mempool_alloc@URange@LocalizerResourceTxt@@@@@std@@IAEXI@Z$2 1000b5bc     LocalizerTxt.obj
 0002:000015cc       __unwindtable$?_Reallocate@?$vector@URange@LocalizerResourceTxt@@V?$mempool_alloc@URange@LocalizerResourceTxt@@@@@std@@IAEXI@Z 1000b5cc     LocalizerTxt.obj
 0002:000015dc       __tryblocktable$?_Reallocate@?$vector@URange@LocalizerResourceTxt@@V?$mempool_alloc@URange@LocalizerResourceTxt@@@@@std@@IAEXI@Z 1000b5dc     LocalizerTxt.obj
 0002:000015f0       __ehfuncinfo$?_Reallocate@?$vector@URange@LocalizerResourceTxt@@V?$mempool_alloc@URange@LocalizerResourceTxt@@@@@std@@IAEXI@Z 1000b5f0     LocalizerTxt.obj
 0002:00001614       __unwindtable$??$?HDU?$char_traits@D@std@@V?$allocator@D@1@@std@@YG?AV?$basic_string@DU?$char_traits@D@std@@V?$allocator@D@2@@0@ABV10@PBD@Z 1000b614     LocalizerTxt.obj
 0002:0000161c       __ehfuncinfo$??$?HDU?$char_traits@D@std@@V?$allocator@D@1@@std@@YG?AV?$basic_string@DU?$char_traits@D@std@@V?$allocator@D@2@@0@ABV10@PBD@Z 1000b61c     LocalizerTxt.obj
 0002:00001640       __unwindtable$??0LocalizerResourceUCS@@AAE@PBDII@Z 1000b640     LocalizerUCS.obj
 0002:00001650       __ehfuncinfo$??0LocalizerResourceUCS@@AAE@PBDII@Z 1000b650     LocalizerUCS.obj
 0002:00001674       __unwindtable$?Load@LocalizerResourceUCS@@SGPAVResource@LocalizerImp@@PBD@Z 1000b674     LocalizerUCS.obj
 0002:0000168c       __ehfuncinfo$?Load@LocalizerResourceUCS@@SGPAVResource@LocalizerImp@@PBD@Z 1000b68c     LocalizerUCS.obj
 0002:000016b0       __unwindtable$??1LocalizerResourceUCS@@UAE@XZ 1000b6b0     LocalizerUCS.obj
 0002:000016c0       __ehfuncinfo$??1LocalizerResourceUCS@@UAE@XZ 1000b6c0     LocalizerUCS.obj
 0002:000016e4       __unwindtable$?Create@FileBuffer@?A0xa493ca04@@SGPAV12@PBD@Z 1000b6e4     LocalizerUCS.obj
 0002:000016fc       __ehfuncinfo$?Create@FileBuffer@?A0xa493ca04@@SGPAV12@PBD@Z 1000b6fc     LocalizerUCS.obj
 0002:00001720       __sehtable$??_M@YGXPAXIHP6EX0@Z@Z 1000b720     MSVCRT:ehvecdtr.obj
 0002:00001740       __sehtable$?__ArrayUnwind@@YGXPAXIHP6EX0@Z@Z 1000b740     MSVCRT:ehvecdtr.obj
 0002:00001760       __sehtable$__onexit        1000b760     MSVCRT:atonexit.obj
 0002:00001780       __sehtable$___DllMainCRTStartup 1000b780     MSVCRT:crtdll.obj
 0002:000017a8       __sehtable$__IsNonwritableInCurrentImage 1000b7a8     MSVCRT:pesect.obj
 0002:00001a98       .idata$6                   1000ba98     memory:Memory.dll
 0002:00001bbc       .idata$6                   1000bbbc     fileio:FileIO.dll
 0002:00001be2       .idata$6                   1000bbe2     debug:Debug.dll
 0002:00001d24       .idata$6                   1000bd24     kernel32:KERNEL32.dll
 0002:00001d3e       .idata$6                   1000bd3e     user32:USER32.dll
 0002:00001e5c       .idata$6                   1000be5c     msvcprt:MSVCP110.dll
 0002:00002038       .idata$6                   1000c038     MSVCRT:MSVCR110.dll
 0002:00002240       .edata                     1000c240     Localizer.exp
 0002:00002268       rgpv                       1000c268     Localizer.exp
 0002:00002314       rgszName                   1000c314     Localizer.exp
 0002:000023c0       rgwOrd                     1000c3c0     Localizer.exp
 0002:00002416       szName                     1000c416     Localizer.exp
 0002:00002424       $N00001                    1000c424     Localizer.exp
 0002:0000244b       $N00002                    1000c44b     Localizer.exp
 0002:0000246c       $N00003                    1000c46c     Localizer.exp
 0002:0000248d       $N00004                    1000c48d     Localizer.exp
 0002:000024b9       $N00005                    1000c4b9     Localizer.exp
 0002:000024d8       $N00006                    1000c4d8     Localizer.exp
 0002:000024fd       $N00007                    1000c4fd     Localizer.exp
 0002:00002561       $N00008                    1000c561     Localizer.exp
 0002:00002586       $N00009                    1000c586     Localizer.exp
 0002:000025e8       $N00010                    1000c5e8     Localizer.exp
 0002:0000260b       $N00011                    1000c60b     Localizer.exp
 0002:00002670       $N00012                    1000c670     Localizer.exp
 0002:00002696       $N00013                    1000c696     Localizer.exp
 0002:000026c7       $N00014                    1000c6c7     Localizer.exp
 0002:000026fa       $N00015                    1000c6fa     Localizer.exp
 0002:0000272e       $N00016                    1000c72e     Localizer.exp
 0002:00002760       $N00017                    1000c760     Localizer.exp
 0002:00002791       $N00018                    1000c791     Localizer.exp
 0002:000027b5       $N00019                    1000c7b5     Localizer.exp
 0002:000027de       $N00020                    1000c7de     Localizer.exp
 0002:00002807       $N00021                    1000c807     Localizer.exp
 0002:00002866       $N00022                    1000c866     Localizer.exp
 0002:000028c7       $N00023                    1000c8c7     Localizer.exp
 0002:000028ea       $N00024                    1000c8ea     Localizer.exp
 0002:00002908       $N00025                    1000c908     Localizer.exp
 0002:000029aa       $N00026                    1000c9aa     Localizer.exp
 0002:00002a10       $N00027                    1000ca10     Localizer.exp
 0002:00002a3b       $N00028                    1000ca3b     Localizer.exp
 0002:00002afb       $N00029                    1000cafb     Localizer.exp
 0002:00002bb5       $N00030                    1000cbb5     Localizer.exp
 0002:00002bd5       $N00031                    1000cbd5     Localizer.exp
 0002:00002bf1       $N00032                    1000cbf1     Localizer.exp
 0002:00002c93       $N00033                    1000cc93     Localizer.exp
 0002:00002cfb       $N00034                    1000ccfb     Localizer.exp
 0002:00002d26       $N00035                    1000cd26     Localizer.exp
 0002:00002d49       $N00036                    1000cd49     Localizer.exp
 0002:00002d71       $N00037                    1000cd71     Localizer.exp
 0002:00002d97       $N00038                    1000cd97     Localizer.exp
 0002:00002db5       $N00039                    1000cdb5     Localizer.exp
 0002:00002ddb       $N00040                    1000cddb     Localizer.exp
 0002:00002df9       $N00041                    1000cdf9     Localizer.exp
 0002:00002e19       $N00042                    1000ce19     Localizer.exp
 0002:00002e37       $N00043                    1000ce37     Localizer.exp
 0003:00000299       ?s_tested@?1??IsNT@@YG_NXZ@4_NA 1000d299     Localizer.obj
 0003:0000029a       ?s_nt@?1??IsNT@@YG_NXZ@4_NA 1000d29a     Localizer.obj
 0003:000002a0       ?tmpL@?6??CompareSort@Localizer@@SGHPB_W0@Z@4PADA 1000d2a0     Localizer.obj
 0003:000012a0       ?tmpR@?6??CompareSort@Localizer@@SGHPB_W0@Z@4PADA 1000e2a0     Localizer.obj
 0003:000022a0       ?tmpL@?6??CompareEqual@Localizer@@SG_NPB_W0@Z@4PADA 1000f2a0     Localizer.obj
 0003:000032a0       ?tmpR@?6??CompareEqual@Localizer@@SG_NPB_W0@Z@4PADA 100102a0     Localizer.obj
 0003:000042ac       _s_instance                100112ac     LocalizerImp.obj
 0003:000042b0       _s_instanceCount           100112b0     LocalizerImp.obj
 0003:000042b4       ?s_pool@?1??Allocator@LocalizerImp@@SGPAU_HMEMPOOL@@XZ@4VMemoryPoolObj@@A 100112b4     LocalizerImp.obj
 0003:000042c0       ?$S1@?1??Allocator@LocalizerImp@@SGPAU_HMEMPOOL@@XZ@4IA 100112c0     LocalizerImp.obj
 0003:000042d4       __Tuple_alloc              100112d4     pch.obj
 0003:000042d5       _ignore                    100112d5     pch.obj
 0003:000042d6       _allocator_arg             100112d6     pch.obj
 0003:000042d7       _piecewise_construct       100112d7     pch.obj
 0003:000042e0       ___proc_attached           100112e0     MSVCRT:crtdll.obj
 0003:000042f0       _GS_ExceptionRecord        100112f0     MSVCRT:gs_report.obj
 0003:00004340       _GS_ContextRecord          10011340     MSVCRT:gs_report.obj
 0003:0000460c       _DebuggerWasPresent        1001160c     MSVCRT:gs_report.obj
 0004:00000060       $R000000                   10012060     * linker generated manifest res *
